:100000000C94650C0C94960C0C94960C0C94960C19
:100010000C94960C0C94723E0C945E6A0C9479715C
:100020000C94960C0C94960C0C94960C0C94960CC8
:100030000C94960C0C94960C0C94960C0C94960CB8
:100040000C94960C0C94C64F0C94F63D0C94960CA4
:100050000C94960C0C94960C0C94960C0C94876F44
:100060000C94960C0C94A0440C9477440C94960C2D
:100070000C94960C0C94960C0C94960C0C94960C78
:100080000C94CA8B0C94960C0C94960C0C94960CB5
:100090000C944E440C9425440C94960C0C94960CA1
:1000A0000C94960C0C94960C0C94960C0C94960C48
:1000B0000C94960C0C94AB4A0C94960C0C94960CE5
:1000C0000C94960C0C94960C0C94960C0C94FC438B
:1000D0000C94D3430C94960C0C94AA430C94814337
:1000E0000C94960C851262123E12A212FA12C112E0
:1000F000F112E012AF138C136813CC135014EB13EE
:1001000047143614E51613174A1781175718901815
:10011000C9180219DE19DE19DE19DE19DE19DE1919
:10012000DE19DE19DE19DE19DE19DE19DE19DE1917
:10013000DE19DE19DE19DE19DE19DE19DE19DE1907
:10014000DE19DE19DE19DE19DE19DE19DE19B8171F
:10015000EF1726183B197419AD19C11BC71BCD1B0E
:10016000D31BD91BDF1BE51BEB1BF11BF71BFD1B77
:10017000031C151C1B1C211C271C2D1C331C391C8B
:100180003F1C451C4B1C511C571C5D1C631C691CEF
:100190006F1C751C7B1C871C8D1C931C991CB11C2F
:1001A000B71CBD1CC31CC91CCF1C1D1D231D291D34
:1001B000351D3B1D411D4D1D531D591D5F1D651DE9
:1001C0006B1D7D1D831D891D8F1D951D9B1DB31DE1
:1001D000B91DBF1DC51DDD1DE11DE51DE91DEF1D7F
:1001E000F31DF71DFB1DFF1D031E071E0D1E131E15
:1001F000191E1F1E251E2B1E311E371E3D1E431E9F
:10020000491E9F1CD51CDB1CE11CE71CED1CF31CCC
:10021000A11DA71DAD1DCB1DD11DD71D4F1E551EE8
:100220005B1E711D771DF91CFF1C051D0B1D111D8B
:10023000171D2F1D471D811C091C0F1CA51CAB1C65
:100240001D311D3137311D3144315D3178319331EC
:100250007A407D406C4070407640B440814085409B
:100260008B408F40934099409D40A140B440A740AF
:10027000AB40AF400A460F4614461E462846A146EC
:1002800032463A4642464C46564660466F467946A6
:10029000A14683468D469746D84AE04AE74AFA4A3D
:1002A0000B4B1C4B264B7E7CB27CE77C077D3C7D58
:1002B000717D817DAB7EF57DFF7D337E687E767EB0
:1002C000F2870988208837884E8865887C889388DB
:1002D000AB88CA88E188F88817892D8921200046D3
:1002E0004143544F52592052455345542120003424
:1002F00000330032004E6F6E650053746F7070658E
:1003000064004E65757472616C205475726E004D98
:100310006F76696E672052657665727365004D6F02
:1003200076696E6720466F7277617264004272610F
:100330006B696E670054414E4B20524553544F52E7
:1003400045440025004865616C7468204C657665FD
:100350006C3A200056454849434C4520524550418F
:10036000495220434F4D504C4554450054414E4B4B
:100370002044455354524F59454400250048656177
:100380006C7468204C6576656C3A200029005645EF
:100390004849434C4520524550414952205354410D
:1003A00052544544202800524550414952204F5054
:1003B00045524154494F4E2043414E43454C4C45D4
:1003C000440029004D414348494E452047554E20A1
:1003D00048495421202800524550414952204F504D
:1003E00045524154494F4E2043414E43454C4C45A4
:1003F0004400290043414E4E4F4E2048495421208D
:10040000280054757272657420726F746174696F1C
:100410006E206973206E6F74206F6620747970652A
:1004200020536572766F2E204E6F20736574757041
:1004300020617661696C61626C652E005475727220
:10044000657420656C65766174696F6E20697320D0
:100450006E6F74206F6620747970652053657276B4
:100460006F2E204E6F207365747570206176616900
:100470006C61626C652E00546F70204C6566740070
:10048000546F702043656E74657200546F70205213
:1004900069676874004D6964646C65204C656674B6
:1004A000004D6964646C652043656E746572004D2F
:1004B0006964646C6520526967687400426F747483
:1004C0006F6D204C65667400426F74746F6D2043CD
:1004D000656E74657200426F74746F6D2052696747
:1004E0006874004649524D57415245205645525373
:1004F000494F4E3A200069427573005342757300AC
:1005000050504D004E6F6E65204465746563746590
:100510006400417A696D7574682020202000456C64
:1005200065766174696F6E2020005475726E2020AC
:100530002020202020005468726F74746C65202085
:100540002000537469636B202020202020204D69F7
:100550006E2020202043656E7465722020204D613E
:1005600078202020204465616462616E64202052FE
:100570006576657273656400524144494F20494E67
:10058000464F202D20004E4F54204445544543549F
:1005900045440049474E4F52454400416E616C6FDF
:1005A00067004469676974616C004175782043682D
:1005B000616E2E2020204D696E20202020204D616C
:1005C00078202020202054797065004368616E6E89
:1005D000656C73207574696C697A65643A200043B0
:1005E00068616E6E656C73206465746563746564C0
:1005F0003A20004D656368616E6963616C207265C5
:10060000636F696C00416972736F6674004D656356
:1006100068616E6963616C2042617272656C3A2038
:100620000020284D31290020284D32290020284261
:10063000290042617272656C20456C65766174694F
:100640006F6E3A20200020284D30290020284D319F
:100650002900202841290054757272657420526F58
:10066000746174696F6E3A20202000447269766567
:10067000204D6F746F72733A202020202020004D8F
:100680004F544F522054595045530054616E6B20C3
:1006900028444B4C4D2074797065290043617200E9
:1006A00048616C66747261636B0054616E6B0055D7
:1006B0004E4B4E4F574E00596573004E6F00290048
:1006C000252C20446563656C65726174696F6E20CA
:1006D000666163746F72200020284B69636B6261EE
:1006E000636B2073706565642000547261636B20D6
:1006F0005265636F696C20456E61626C65643A2077
:100700002020004E2F4120666F7220766568696355
:100710006C652074797065005475726E204D6F643D
:10072000653A20202020202020202020202020206A
:10073000004E2F4120666F722076656869636C6594
:100740002074797065002500202D20004E65757499
:1007500072616C205475726E20416C6C6F776564A9
:100760003A2020200020736563005472616E736D1F
:10077000697373696F6E2044656C61793A2020203B
:100780002020002073656300456E67696E65205008
:10079000617573652054696D653A20202020202002
:1007A00000207365630053686966742054696D6541
:1007B0003A2020202020202020202020202000253A
:1007C00000596573202D200052657665727365208F
:1007D0005370656564204C696D697465643A2020C6
:1007E000002500596573202D2000466F72776172D5
:1007F00064205370656564204C696D697465643A62
:10080000202000206D73290025207468726F747495
:100810006C6520666F7220002028004D6F746F7227
:10082000204E7564676520456E61626C65643A2090
:100830002020200029004E6F6E65004E6F6E65000F
:100840002C205072657365743A20002900202841DD
:10085000646A757374656420746F200020284C6589
:1008600076656C3A2000446563656C2052616D705A
:1008700020456E61626C65643A20202020200029AA
:10088000004E6F6E65004E6F6E65002C20507265D5
:100890007365743A20002900202841646A757374D6
:1008A000656420746F200020284C6576656C3A20C2
:1008B00000416363656C2052616D7020456E61621A
:1008C0006C65643A202020202000416374697665BD
:1008D0002044726976696E672050726F66696C6534
:1008E0003A200056656869636C6520547970653AF2
:1008F0002020202020202020202020004452495663
:10090000452053455454494E4753002073656300B6
:100910005265636F696C2064656C61793A202020B0
:1009200020202020202020202020202020202020C7
:10093000002500596573202D200042617272656C9C
:1009400020456C65766174696F6E205370656564CF
:10095000204C696D697465643A20002500596573FF
:10096000202D200054757272657420526F7461746A
:10097000696F6E205370656564204C696D6974659C
:10098000643A202000545552524554205345545443
:10099000494E475300556E6B6E6F776E0048656128
:1009A0007679004D656469756D004C6967687400FF
:1009B000437573746F6D00556E6B6E6F776E004F7D
:1009C00070656E2050616E7A65720054616D697950
:1009D0006120537065630020736563207265636FE7
:1009E000766572792900207365632072656C6F618A
:1009F000642C2000204D4720686974732C2000204F
:100A000063616E6E6F6E20686974732C200028001D
:100A100057656967687420436C6173733A202020BE
:100A200020200044616D6167652050726F66696CBB
:100A3000653A2020200059657320280041636365D2
:100A40007074204D472044616D6167653A200059FC
:100A5000657320280053656E64204D47204952205D
:100A6000436F64653A2020004E2F4100526570614B
:100A7000697265642062793A202020202020004E8F
:100A80002F41004869742050726F746F636F6C203F
:100A9000323A20202000290020285465616D200072
:100AA000466972652050726F746F636F6C3A2020D4
:100AB000202000466972652050726F746F636F6CFE
:100AC0003A2020202000497320526570616972200D
:100AD00054616E6B3F202020004952202620546133
:100AE0006E6B20426174746C696E67204469736137
:100AF000626C656400424154544C4520494E464F57
:100B000000554E4B4E4F574E004265696572205559
:100B1000534D2D52432D320054616967656E205349
:100B20006F756E642043617264004F70656E205073
:100B3000616E7A657220536F756E642043617264D2
:100B40000042656E6564696E6920544253204D69A8
:100B50006E6900536F756E6420636172643A2000A1
:100B6000534F554E4420434152440048696C6C2019
:100B70005068797369637320456E61626C65643A8D
:100B80002020202020202020200042617272656CED
:100B90002053746162696C697A6174696F6E204573
:100BA0006E61626C65643A200053656E736F7220EB
:100BB00064657465637465643A20202020202020D9
:100BC000202020202020205965730053656E736F0C
:100BD00072206E6F742064657465637465642100AF
:100BE000494E45525449414C204D4541535552457B
:100BF0004D454E5420554E495400556E6B6E6F77DF
:100C00006E00537065656420646563726561736529
:100C1000732062656C6F772000537065656420698E
:100C20006E637265617365732061626F7665200023
:100C300056656869636C652044657374726F796585
:100C4000640043616E6E6F6E204869740042726189
:100C50006B6573204170706C6965640056617269E0
:100C600061626C650020286F6620352900332028DA
:100C70006F66203329003220286F66203329003127
:100C800020286F66203329003220286F6620322901
:100C9000003120286F6620322900506F73200041F8
:100CA0007578204368616E6E656C200056617269CC
:100CB00061626C65004F6E004F6666004200410045
:100CC00045787465726E616C20496E707574200091
:100CD000070809090B0C0C0B0C0C54757272657427
:100CE00020537469636B202D200046756E63746910
:100CF0006F6E202300202D3E20002073656300547A
:100D00007572726574206D6F76656D656E742064A2
:100D1000656C61793A2020004E6F6E6500596573ED
:100D20000054757272657420737469636B20667504
:100D30006E6374696F6E733A200046554E43544992
:100D40004F4E205452494747455253007620637511
:100D5000746F666629002028004C564320456E615A
:100D6000626C65643A202020202020007600566FB7
:100D70006C746167653A20202020202020202020EC
:100D800000596573004E6F0042617474657279207A
:100D900044657465637465643A2000424154544567
:100DA00052590053657269616C2033205478204297
:100DB0006175643A2020004175782053657269613D
:100DC0006C20426175643A202020004D6F746F7270
:100DD0002053657269616C20426175643A20005548
:100DE00053422053657269616C20426175643A20F8
:100DF0002020004241554420524154455300556E35
:100E00006B6E6F776E0044657461636865642F4E26
:100E100041005265636F696C20536572766F0050B4
:100E2000616E20536572766F00536572766F2F4541
:100E30005343004F6E626F617264204D6F746F7226
:100E400020447269766572004F70656E2050616E45
:100E50007A65722053636F75742053657269616C93
:100E600020455343005361626572746F6F7468204C
:100E700053657269616C00506F6C6F6C75205365BF
:100E80007269616C00536572766F20310053657230
:100E9000766F203200536572766F2033005365728F
:100EA000766F203400536572766F2035005365727B
:100EB000766F203600536572766F20370053657267
:100EC000766F20380000002100240027002A002D22
:100ED000003000330001010000040107010A010095
:100EE000002200250028002B002E003100340002D3
:100EF000010000050108010B01000020002300266D
:100F00000029002C002F0032000001000003010620
:100F10000109010505050507050808080802020280
:100F2000020A0A0808040404040101010101010184
:100F3000010303030303030303040707070C0C0C5B
:100F40000C0C0C0C0C020202020606060606060633
:100F5000060B0B0B0B0B0B0B0B01021020200808D0
:100F6000102040102040800201020108040201010B
:100F700002040810204080804020100804020180F4
:100F8000040201804020100804020108040201014B
:100F90000204081020408001020408102040800054
:100FA000000A0B02090C0D0E0807030401000000E3
:100FB0000000000000000000000000000000000031
:100FC00000000000000000000000001211100000EE
:100FD0000000000000000000000000000000000011
:100FE0000000000000536F6E790052435441204DC1
:100FF000616368696E652047756E00436C61726B52
:10100000204D616368696E652047756E00524354D8
:1010100041205265706169720049425520526570E5
:1010200061697200436C61726B2052657061697214
:10103000004F70656E50616E7A6572005673546130
:101040006E6B00464F560054616967656E004865D7
:101050006E67204C6F6E670054616D697961203155
:101060002F33350054616D69796120322D53686FDB
:10107000740054616D69796100556E6B6E6F776EA7
:10108000003A200042697420004761703A20005203
:101090004144494F204641494C5341464500526125
:1010A00064696F205265616479202D200052657655
:1010B00065727365643A2020004D61782050756C2C
:1010C00073653A20004D696E2050756C73653A2047
:1010D00000456E642056616C75657300456E642032
:1010E0005265636F696C20536572766F2053657427
:1010F000757000456E6420526F746174696F6E2064
:10110000536572766F20536574757000456E642068
:10111000456C65766174696F6E20536572766F20D9
:10112000536574757000536572766F20756E2D72FD
:101130006576657273656400536572766F207265BB
:101140007665727365640052657665727365643A9C
:101150002020004D61782050756C73653A20004D59
:10116000696E2050756C73653A2000537461727417
:101170002056616C75657300494E56414C494420B8
:10118000534552564F2E204E4F2053455455502E06
:10119000005365747570205265636F696C205365E8
:1011A00072766F0053657475702054757272657431
:1011B00020526F746174696F6E2050616E205365A8
:1011C00072766F0053657475702054757272657411
:1011D00020456C65766174696F6E2050616E205396
:1011E0006572766F00416972736F6674202D2044BA
:1011F000697361626C6564004D656368616E696303
:10120000616C205265636F696C202D2044697361A5
:10121000626C656400436F6D6D73206368616E6717
:10122000656420746F2055534200436F6D6D7320C9
:101230006368616E67656420746F205365726961CD
:101240006C20310044726976696E672050726F6657
:10125000696C652073657420746F20230054757267
:101260006E20456E67696E65204F6E005475726E14
:1012700020456E67696E65204F666600456E67693A
:101280006E65204175746F2053687574646F776E56
:1012900000456E67616765205472616E736D697396
:1012A00073696F6E00446973656E6761676520548A
:1012B00072616E736D697373696F6E00536574202C
:1012C0005475726E204D6F64653A20310053657419
:1012D000205475726E204D6F64653A20320053655C
:1012E00074205475726E204D6F64653A203300454A
:1012F0006E61626C65204E65757472616C20547508
:10130000726E730044697361626C65204E6575741A
:1013100072616C205475726E730042617272656CFA
:101320002053746162696C697A6174696F6E3A20E6
:101330005475726E6564204F4E0042617272656C26
:101340002053746162696C697A6174696F6E3A20C6
:101350005475726E6564204F46460048696C6C2077
:10136000506879736963733A205475726E656420AE
:101370004F4E0048696C6C20506879736963733A0A
:10138000205475726E6564204F464600494F2050C8
:101390006F72742041204F7574707574202D204F2A
:1013A0006E00494F20506F72742041204F75747049
:1013B0007574202D204F666600417578204F757436
:1013C000707574205072657365742044696D0041B6
:1013D0007578204F757470757420466C61736865FC
:1013E0006400417578204F757470757420496E766D
:1013F0006572736520466C61736865640053746F31
:101400007020417578204F757470757420426C6936
:101410006E6B696E670053746F70205265766F6CE7
:1014200076696E6720417578204C69676874003171
:101430000031202D205374617274205265706561F3
:1014400074696E670031202D2053746F7000320074
:1014500032202D205374617274205265706561745E
:10146000696E670032202D2053746F700033003393
:10147000202D205374617274205265706561746907
:101480006E670033202D2053746F700034003420B9
:101490002D20537461727420526570656174696E99
:1014A000670034202D2053746F7000350035202DD7
:1014B00020537461727420526570656174696E673F
:1014C0000035202D2053746F7000360036202D20FB
:1014D000537461727420526570656174696E67003F
:1014E00036202D2053746F70005573657220467539
:1014F0006E6374696F6E2031005573657220467596
:101500006E6374696F6E203200494F20506F7274A1
:101510002042204F7574707574202D204F6E004945
:101520004F20506F72742042204F75747075742074
:101530002D204F6666004C56432045786974202D57
:1015400020566F6C7461676520526573746F7265A5
:1015500064007629004C5643207468726573686F86
:101560006C642072656163686564212028004C69A1
:101570006768742031204F6E004C696768742031B1
:10158000204F6666004C696768742032204F6E00F9
:101590004C696768742032204F666600326E6420A2
:1015A0004D472053746F7000326E64204D472053B6
:1015B000746172740052756E6E696E67204C696753
:1015C000687473204F6E0052756E6E696E67204CA2
:1015D0006967687473204F666600417578204F759F
:1015E00074707574204F6E00417578204F7574705B
:1015F0007574204F66660053746F70205265766F65
:101600006C76696E6720417578204C696768740054
:1016100053746F7020417578204F75747075742005
:10162000426C696E6B696E6700537461727420411D
:101630007578204F757470757420426C696E6B6993
:101640006E6700536D6F6B657220656E61626C65CD
:101650006400536D6F6B65722064697361626C65C1
:10166000640053657420766F6C756D653A20005583
:1016700073657220536F756E642000466972652031
:1016800043616E6E6F6E00466972652052657061CF
:101690006972205369676E616C00416972736F668D
:1016A00074202D204D616E75616C205472696767DE
:1016B0006572004D656368616E6963616C20526597
:1016C000636F696C202D204D616E75616C205472C2
:1016D000696767657200536572766F205265636F44
:1016E000696C202D204D616E75616C2054726967A4
:1016F000676572004869676820496E74656E736932
:10170000747920466C61736820556E6974202D20B1
:101710004D616E75616C2054726967676572004D2A
:1017200047205374617274004D472053746F7000EA
:10173000401F7017D007A00FA00FDC05D007C40909
:1017400010278813983A10276C023A026C023A026A
:101750006C023A026C02B036384A5C121C255C12EC
:101760005C121C255C12BC7FC7F2C07887A5B7C588
:10177000A00F8813B80B401FB80BB80B7017401F91
:1017800053657420416363656C2052616D70204C19
:101790006576656C3A200053657420446563656C1A
:1017A0002052616D70204C6576656C3A200053655F
:1017B000742042617272656C2053656E736974693E
:1017C000766974793A20005365742048696C6C20FE
:1017D00053656E73697469766974793A2000416E55
:1017E000616C6F6720557365722046756E6374690E
:1017F0006F6E2031202D2000416E616C6F67205587
:101800007365722046756E6374696F6E2032202D89
:1018100020002D00202D2000200054525545004668
:10182000414C534500250057616974696E67206615
:101830006F7220726164696F2E2E2E2000290020A5
:101840002D2041646A757374656420746F200020D4
:101850002853656E7369746976697479200029006C
:10186000202D2041646A757374656420746F2000B4
:10187000202853656E736974697669747920005302
:1018800074617274205265766F6C76696E67204160
:101890007578204C6967687400416972736F66746B
:1018A000202D20456E61626C6564004D6563686142
:1018B0006E6963616C205265636F696C202D2045F1
:1018C0006E61626C65640000B99C11241FBECFEF8D
:1018D000D1E2DEBFCDBF00E00CBF15E0A0E0B2E07A
:1018E000EFE1F5E701E00BBF02C007900D92A23BCC
:1018F000B107D9F722E1A2EBB5E001C01D92AF39E3
:10190000B207E1F71CE0C5E6DCE000E006C0219785
:101910000109802FFE010E949FA7C436D10780E0F5
:101920000807A9F70E94EA8C0C945FAD0C940000A4
:101930002F923F924F925F926F927F928F929F92DF
:10194000AF92BF92CF92DF92EF92FF920F931F93CD
:10195000CF93DF93CDB7DEB7A9970FB6F894DEBF6C
:101960000FBECDBF85EC91E00E94EAAC6A327F44A5
:101970008105910519F00E94AA5608C049EC51E072
:1019800060E070E088E99EE00E94D2AC40E052EC5A
:1019900061E070E080E998E00E94FD8640913E1091
:1019A00050913F10609140107091411083EF97E08B
:1019B0000E94FD8640914210509143106091441066
:1019C0007091451086E597E00E94FD864091461093
:1019D00050914710609148107091491089EB96E042
:1019E0000E94FD868AEC9CE09093B5058093B40537
:1019F0008BE89AE09093B3058093B20580E998E074
:101A000090930C0E80930B0E10920D0E1092CF0C33
:101A10001092CC0C1092CE0C1092CD0C11E01093C1
:101A2000DB0C0E94406380915C1080935D061092F5
:101A30005C061092800082E0809381008FE286BB7A
:101A400010926F0010928500109284009BE2909398
:101A5000A0009AE09093A10089BB109272001092AE
:101A6000A5001092A4001092A9001092A800109254
:101A7000AB001092AA001092AD001092AC0099EA4F
:101A800090932001109321018ABB10927300109251
:101A90002501109224011092290110922801109220
:101AA0002B0110922A0110922D0110922C0180918D
:101AB000350F9091360F8093EE059093EF058130AE
:101AC00071F461E08FE30E94A7458091EF058823C0
:101AD00019F00E94EB5F0FC00E94D45F0CC0809190
:101AE000EF05882311F062E001C060E08FE30E94FF
:101AF000A7450E94FD758091370F9091380F809314
:101B0000F5059093F605813071F461E08EE30E9453
:101B1000A7458091F605882319F00E946A730FC0CB
:101B20000E9453730CC08091F605882311F062E087
:101B300001C060E08EE30E94A7450E94CA7560E084
:101B400085E40E94A74562E08CE30E94A74562E01D
:101B50008BE30E94A74562E080E40E94A74562E013
:101B600081E40E94A74562E082E40E94A74562E00A
:101B700081E20E94A74562E084E40E94A74561E0FB
:101B800089E30E94A74561E08AE30E94A7450E947D
:101B9000D8730E940F7461E085E30E94A74561E05D
:101BA00085E00E94A74561E070E085E00E94E34582
:101BB00061E084E00E94A74561E087E00E94A745BC
:101BC00061E089E20E94784561E089E20E94A745D0
:101BD0006A9A60E085E30E94784560E085E00E94B3
:101BE000784560E084E00E94784560E087E00E94EC
:101BF0007845729861E088E00E94A74580E090E017
:101C00009C012856314FF901ED55FF4F40814F3669
:101C100029F4329720813181232B31F403968837C0
:101C2000910571F760E001C061E088E00E947845AD
:101C300061E08BE20E94A74560E08BE20E9478455C
:101C40000E940F740E94757F80917B0A813009F099
:101C50006CC080917E0A90917F0AA091800AB09119
:101C6000810A4091820A5091830A6091840A70919E
:101C7000850A841B950BA60BB70B84379E40A105E4
:101C8000B10500F30E94AA5680915A0690915B0616
:101C90000E945E4380915A0690915B060E945E43CB
:101CA0000E9413856FED72E080915A0690915B0659
:101CB0000E94004201E010E00E94DC730E940F7459
:101CC0006EEE72E080E090E00E94EE466CED72E015
:101CD00080915A0690915B060E9400420E94D87340
:101CE0000E940B740530110531F064EF71E080E063
:101CF00090E00E94EE460F5F1F4F06301105E1F69F
:101D000080915A0690915B060E945E430E94138563
:101D100080915A0690915B060E945E4380915A061C
:101D200090915B060E945E4302C081118BCF80912F
:101D30006F00826080936F00809184009091850095
:101D40008056904F909389008093880081E0809323
:101D500054128093571280935A1280935D1280938D
:101D6000691280936C129091ED0F9150943040F075
:101D70008093ED0F61E070E085E591E00E94067FC1
:101D80009091ED0F2DEF290F8091B10F223008F0C7
:101D9000AEC18A3079F03CF4883009F45DC08930F6
:101DA00009F45DC153C18B3009F49EC08C3009F435
:101DB000E0C04CC183E290E00E94B9A8FC0188E039
:101DC00090E0938382838824839499249A949582C3
:101DD0008482AA24AA94B12CB782A6821186108686
:101DE000108E53E8752E718E66E5C62E67E0D62EEE
:101DF000D38EC28E79E6E72E72E0F72EF182E08272
:101E000002E410E111A300A312A2F0934D06E093A7
:101E10004C06CF010E94F93983E290E00E94B9A8F4
:101E2000FC0189E090E09383828395828482B7826B
:101E3000A68211861086108E718ED38EC28EF1828C
:101E4000E08211A300A312A2F0934B06E0934A068E
:101E5000CF010E94F939D0C280E290E00E94B9A877
:101E6000FC0188E090E09383828388248394992402
:101E70009A9495828482AA24AA94B12CB782A682CD
:101E800011861086108E9AE0D92ED18E26E5E22E8C
:101E900027E0F22EF38EE28E01E512E0118300833B
:101EA000F0934D06E0934C06CF010E94E53680E2A8
:101EB00090E00E94B9A8FC0189E090E093838283BE
:101EC00095828482B782A68211861086108ED18E6A
:101ED000F38EE28E11830083F0934B06E0934A0663
:101EE000CF010E94E53688C289E190E00E94B9A83E
:101EF000FC0188E090E093838283CC24C394DD24AA
:101F0000DA94D582C482EE24EA94F12CF782E68238
:101F100011861086108E05E412E011830083F09381
:101F20004D06E0934C06CF010E942C3610926912A8
:101F30008091ED0F843009F05FC289E190E00E944A
:101F4000B9A8FC0189E090E093838283D582C482A2
:101F5000F782E68211861086108E11830083F0933B
:101F60004B06E0934A06CF010E942C3610926C1269
:101F700043C289E190E00E94B9A88C0175E8872EE0
:101F800075E0972EDC0111969C928E9287E090E08E
:101F900013969C938E931297AA24A394BB24BA946D
:101FA0001596BC92AE921497CC24CA94D12C179655
:101FB000DC92CE92169719961C921E9218975896FC
:101FC0001C92C8010E949550A5EEEA2EA3E0FA2EBD
:101FD000F801F182E08210934D0600934C06C8018F
:101FE0000E94C734109254128091ED0F843009F092
:101FF00003C289E190E00E94B9A88C01DC0111962E
:102000009C928E9286E090E013969C938E9312970A
:102010001596BC92AE9214971796DC92CE921697B4
:1020200019961C921E92189758961C92C8010E94ED
:102030009550F801F182E08210934B0600934A0616
:10204000C8010E94C73410925712D6C189E080930C
:10205000B10F69E070E089E191E00E94067F80E2C3
:1020600090E00E94B9A8FC0188E090E0938382830D
:102070008824839499249A9495828482AA24AA9489
:10208000B12CB782A68211861086108E50E8D52E0C
:10209000D18E66E5E62E67E0F62EF38EE28E0DE534
:1020A00012E011830083F0934D06E0934C06CF01BC
:1020B0000E94923980E290E00E94B9A8FC0189E078
:1020C00090E09383828395828482B782A682118670
:1020D0001086108ED18EF38EE28E11830083F093E2
:1020E0004B06E0934A06CF010E94923985C18A309F
:1020F00079F03CF4883009F455C0893009F425C1E1
:102100001BC18B3009F471C08C3009F4A8C014C114
:1021100083E290E00E94B9A8FC017090F90F88E07A
:1021200090E0938382838824839499249A9495825F
:102130008482AA24AA94B12CB782A6821186108622
:10214000108E83E8682E618E96E5C92E97E0D92E11
:10215000D38EC28E29E6E22E22E0F22EF182E082B8
:1021600002E410E111A300A372A2F0934F06E093E2
:102170004E0683E290E00E94B9A8FC0189E090E05D
:102180009383828395828482B782A6821186108689
:10219000108E618ED38EC28EF182E08211A300A3D5
:1021A00072A210C180E290E00E94B9A8FC0188E010
:1021B00090E0938382838824839499249A949582CF
:1021C0008482AA24AA94B12CB782A6821186108692
:1021D000108EAAE0DA2ED18EB6E5EB2EB7E0FB2EFC
:1021E000F38EE28E01E512E0D2C089E190E00E9418
:1021F000B9A8FC0188E090E093838283CC24C39447
:10220000DD24DA94D582C482EE24EA94F12CF7829C
:10221000E68211861086108E05E412E01183008399
:10222000F0934F06E0934E0689E190E00E94B9A832
:10223000FC0189E090E093838283D582C482F78297
:10224000E68211861086108E11830083F09351066A
:10225000E09350061092691210926C12B7C092303F
:1022600049F481E08093ED0F61E070E085E591E055
:102270000E94067F89E190E00E94B9A88C0185E860
:10228000882E85E0982ED80111969C928E9287E038
:1022900090E013969C938E931297AA24A394BB2448
:1022A000BA941596BC92AE921497CC24CA94D12CB1
:1022B0001796DC92CE92169719961C921E9218973A
:1022C00058961C92C8010E94955035EEE32E33E0DB
:1022D000F32EF801F182E08210934F0600934E0630
:1022E00089E190E00E94B9A88C01DC0111969C92D2
:1022F0008E9286E090E013969C938E93129715969B
:10230000BC92AE9214971796DC92CE9216971996BD
:102310001C921E92189758961C92C8010E949550C4
:10232000F801F182E082109351060093500610925A
:102330005412109257124AC089E08093B10F69E09D
:1023400070E089E191E00E94067F80E290E00E94C7
:10235000B9A8FC0188E090E0938382838824839469
:1023600099249A9495828482AA24AA94B12CB78243
:10237000A68211861086108EA0E8DA2ED18EB6E5E0
:10238000EB2EB7E0FB2EF38EE28E0DE512E011830B
:102390000083F0934F06E0934E0680E290E00E94A7
:1023A000B9A8FC0189E090E09383828395828482BE
:1023B000B782A68211861086108ED18EF38EE28EA1
:1023C00011830083F0935106E093500680915006EC
:1023D00090915106DC01ED91FC910280F381E02D9A
:1023E000199580914E0690914F06DC01ED91FC917C
:1023F0000280F381E02D19958091ED0F825082309B
:1024000050F589E190E00E94B9A88C0185E895E03B
:10241000F8019183808386E090E09383828381E05A
:102420009FEF958384838FEF90E097838683118657
:102430001086108EC8010E94955085EE93E0D80159
:102440008D939C931093480600934706C8010E9401
:10245000C73410925712E091B20F8E2FEE0F990BE6
:10246000AA0BBB0BFC013897E830F10508F0B9C0A6
:102470008827EE58FF4F8F4F0C949FA783E290E080
:102480000E94B9A8FC0188E090E09383828381E0F8
:102490009FEF958384838FEF90E0978386831186E7
:1024A0001086108E84E8818F86E597E0938F828F67
:1024B00089E692E09183808382E490E191A380A3F6
:1024C00012A21EC080E290E00E94B9A8FC0188E040
:1024D00090E09383828381E09FEF958384838FEFE5
:1024E00090E09783868311861086108E87E8818F0F
:1024F00086E597E0938F828F8DE592E091838083CC
:10250000F0935506E09354069CC080E290E00E9450
:10251000B9A8FC0188E090E09383828381E09FEF7B
:10252000958384838FEF90E097838683118610864E
:10253000108E8DE0818F86E597E0938F828F81E505
:1025400092E0DCCF89E190E00E94B9A8FC0188E02C
:1025500090E09383828381E09FEF958384838FEF64
:1025600090E09783868311861086108E85E492E032
:1025700091838083F0935506E0935406109269127C
:1025800060C08CE190E00E94B9A88C0185E895E0DC
:10259000F8019183808385E090E09383828381E0DA
:1025A0009FEF958384838FEF90E0978386831186D6
:1025B0001086108EC8010E94955089E795E038C0BA
:1025C00089E190E00E94B9A8FC0113821282158271
:1025D00014821782168211861086108E81E292E094
:1025E0008DCF8CE08093B20F6CE070E08AE191E0D7
:1025F0000E94067F89E190E00E94B9A88C0185E8DD
:1026000095E0F8019183808385E090E09383828355
:1026100081E09FEF958384838FEF90E0978386839B
:1026200011861086108EC8010E94955085EE93E0A9
:10263000D8018D939C9310935506009354061092E5
:102640005A128091540690915506DC01ED91FC914F
:102650000280F381E02D19958091BA0F843658F4E9
:10266000853608F084E664E6681B809154069091F4
:1026700055060E94983A8091B20F8C508230A8F48F
:102680006091BB0F7091BC0F85E00E94E04E60919D
:10269000BD0F7091BE0F85E00E94264D8091BF0F47
:1026A000E0915406F0915506808FE091B30F8E2F84
:1026B000EE0F990BAA0BBB0BFC013897E830F10524
:1026C00008F0E5C08827E658FF4F8F4F0C949FA76E
:1026D00083E290E00E94B9A8FC0189E090E0938336
:1026E000828381E09FEF958384838FEF90E09783CF
:1026F000868311861086108E84E8818F86E597E0A8
:10270000938F828F89E692E09183808382E490E1C7
:1027100091A380A312A21EC080E290E00E94B9A8FB
:10272000FC0189E090E09383828381E09FEF9583B1
:1027300084838FEF90E09783868311861086108EB6
:1027400087E8818F86E597E0938F828F8DE592E011
:1027500091838083F0935906E0935806C8C080E2C5
:1027600090E00E94B9A8FC0189E090E09383828305
:1027700081E09FEF958384838FEF90E0978386833A
:1027800011861086108E8DE0818F86E597E0938FFD
:10279000828F81E592E0DCCF89E190E00E94B9A8C8
:1027A000FC0189E090E09383828381E09FEF958331
:1027B00084838FEF90E09783868311861086108E36
:1027C00085E492E091838083F0935906E093580664
:1027D00010926C128CC08CE190E00E94B9A88C0120
:1027E00095E8692E95E0792EF8017182608224E0E7
:1027F000822E912C93828282AA24A394BB24BA9421
:10280000B582A482CC24CA94D12CD782C6821186E8
:102810001086108EC8010E94955059E7E52E55E0AC
:10282000F52ED801ED92FC921093590600935806AC
:102830008CE190E00E94B9A88C01FC017182608259
:1028400093828282B582A482D782C6821186108644
:10285000108E0E949550D801ED92FC921093EB0DD2
:102860000093EA0DC8010E9486353FC089E190E0DF
:102870000E94B9A8FC011382128215821482178269
:10288000168211861086108E81E292E061CF8CE074
:102890008093B30F6CE070E08BE191E00E94067FC3
:1028A00089E190E00E94B9A88C0185E895E0F801E3
:1028B0009183808384E090E09383828381E09FEF23
:1028C000958384838FEF90E09783868311861086AB
:1028D000108EC8010E94955085EE93E0D8018D932B
:1028E0009C93109359060093580610925D128091A4
:1028F000580690915906DC01ED91FC910280F3811C
:10290000E02D19958091B90F843658F4853608F07A
:1029100084E664E6681B80915806909159060E94EF
:10292000983A8091B30F8C50823000F56091B40FCB
:102930007091B50F84E00E94E04E6091B60F7091E7
:10294000B70F84E00E94264D8091B80FE0915806A1
:10295000F0915906808F8091B30F8D3039F48091BA
:10296000B80FE091EA0DF091EB0D808F8EE190E0D1
:102970000E94B9A88C01D090C40FA090C80FB0904D
:10298000C90F8090C60F9090C70F85E895E0F801B9
:102990009183808383E090E09383828381E09FEF43
:1029A00095838483EE24EA94F12CF782E6821186E3
:1029B0001086108EC8010E94955089E392E0D801DC
:1029C00011969C938E935A969C928E9259975C96F0
:1029D000BC92AE925B975D96DC921093910E009341
:1029E000900E6091CA0F7091CB0F83E00E94E04E71
:1029F0006091CC0F7091CD0F83E00E94264D8091A5
:102A0000C40FE091900EF091910E808F8091C40FD1
:102A10000E94D17E8091900E9091910EDC01ED91FB
:102A2000FC910280F381E02D19958091CE0F8823CF
:102A3000D1F083E290E00E94B9A8FC018091D10F0F
:102A40009091D20F2091CF0F3091D00F4091D30FA2
:102A50005091D40F68E070E0738362831582148212
:102A60005783468315C083E290E00E94B9A8FC0119
:102A70008091D10F9091D20F2091CF0F3091D00F34
:102A800048E050E05383428315821482F782E68245
:102A900011861086108E4DE252E051834083328FB2
:102AA000218F948F838FF093E505E093E405809167
:102AB000E4059091E5050E940A3680916912882309
:102AC000F9F089E190E00E94B9A8FC0188E090E06B
:102AD00093838283158214828FEF93E0978386839A
:102AE0008FEF91E091878087108E85E492E091834B
:102AF0008083F0936812E0936712CF010E942C3616
:102B000080916C128823F9F089E190E00E94B9A8C5
:102B1000FC0189E090E093838283158214828FEF19
:102B200093E0978386838FEF91E091878087108E63
:102B300085E492E091838083F0936B12E0936A12B4
:102B4000CF010E942C368CE89AE09093680D809318
:102B5000670D1091FC0F2091FB0F8091EA0F90916F
:102B6000EC0F3091ED0F3093B6059093B90580933B
:102B7000BA0530E0AFEFB0E00E9450AD24E630E09F
:102B800040E050E00E9402AD20938312612F70E07C
:102B900080E090E00E94BDAB23EC34E64AEA5AE3C1
:102BA0000E941EAC2AE939E949E55FE30E94B4A717
:102BB00060937D1270937E1280937F1290938012A7
:102BC0001092950010929400109290008CE08093E7
:102BD000910084EF90E0909399008093980011E029
:102BE00018BB82E080937100809100020E94DB623A
:102BF00080915A0690915B0620915D064091E60F08
:102C00005091E70F5093C10D4093C00D2093F50DE7
:102C10009093F40D8093F30D1092BB051093C60DA5
:102C200080910310843040F01092031060E070E057
:102C30008BE691E00E94067F10910310113081F025
:102C400008F444C0123021F1133009F457C0109237
:102C5000031060E070E08BE691E00E94067F36C0D2
:102C60008BE090E00E94B9A82DE233E0FC013183B3
:102C7000208326E537E0328721879093570680939B
:102C800056061093601210936312109366123CC0A4
:102C900086E090E00E94B9A821ED32E0DC012D939E
:102CA0003C9390935706809356068FB7F8942CED7B
:102CB00035E03093841120938311109289118FBFD6
:102CC00081E080936012809363121CC085E090E0E5
:102CD0000E94B9A88C0129E833E0FC0121933193CB
:102CE000CF016CE87AE00E94434A85E792E0D80180
:102CF0008D939C9310935706009356061092601282
:102D000010926312109266128091560690915706A7
:102D1000DC01ED91FC910190F081E02D19958091FD
:102D2000541281111FC08091571281111BC08091D4
:102D30005A12811117C080915D12811113C08091C8
:102D4000601281110FC08091631281110BC08091BC
:102D50006612811107C081E00E943C63882309F458
:102D60003DC335C3A12CB12C312C812C412C512CCD
:102D7000612C912C712C05E815E0EE24EA94A3E077
:102D8000FA2ECC24CA94DD24D394C5018856914FE1
:102D9000FC01ED55FF4FE081EE2309F40FC3DC0188
:102DA000AF55BF4F8D919C91892B09F407C38E2F8E
:102DB00090E0FC01F797EB32F10508F0FFC288279D
:102DC000EE57FF4F8F4F0C949FA78091541288238A
:102DD00009F4F4C27110F2C289E190E00E94B9A82E
:102DE0009C01FC011183008387E090E09383828340
:102DF00015821482F782E682D186C086108EC901C0
:102E000028A739A70E94955028A539A5E5EEF3E03B
:102E1000D901ED93FC933093451220934412C901DC
:102E20000E94C7347AC180915712882309F4C6C220
:102E30009110C4C289E190E00E94B9A89C01DC0114
:102E400011961C930E93E6E0F0E01396FC93EE933C
:102E5000129715961C921E9214971796FC92EE925A
:102E600016971996DC92CE92189758961C9228A71E
:102E700039A70E94955028A539A5E5EEF3E0D901C0
:102E8000ED93FC933093471220934612C9010E94A0
:102E9000C7347CC180915A12882309F48FC2611013
:102EA0008DC289E190E00E94B9A89C01DC011196D5
:102EB0001C930E93E5E0F0E01396FC93EE931297CB
:102EC00015961C921E9214971796FC92EE921697E6
:102ED0001996DC92CE92189758961C9228A739A77B
:102EE0000E94955028A539A5E5EEF3E0D901ED93B0
:102EF000FC933093491220934812C9010E94C734B1
:102F00007EC180915D12882309F458C2511056C2C7
:102F100089E190E00E94B9A89C01DC0111961C9304
:102F20000E93E4E0F0E01396FC93EE93129715965F
:102F30001C921E9214971796FC92EE921697199671
:102F4000DC92CE92189758961C9228A739A70E9417
:102F5000955028A539A5E5EEF3E0D901ED93FC9352
:102F600030934B1220934A12C9010E94C73480C18A
:102F700080916012882309F421C241101FC289E1A7
:102F800090E00E94B9A89C01DC0111961C930E935D
:102F9000E2E0F0E01396FC93EE93129715961C92E4
:102FA0001E9214971796FC92EE9216971996DC9241
:102FB000CE92189758961C9228A739A70E94955030
:102FC00028A539A5E5EEF3E0D901ED93FC93309304
:102FD0004D1220934C12C9010E94C73482C18091C6
:102FE0006312882309F4EAC18110E8C189E190E005
:102FF0000E94B9A89C01DC0111961C930E93E1E09C
:10300000F0E01396FC93EE93129715961C921E9285
:1030100014971796FC92EE9216971996DC92CE9220
:10302000189758961C9228A739A70E94955028A552
:1030300039A5E5EEF3E0D901ED93FC9330934F12FF
:1030400020934E12C9010E94C73484C18091661238
:10305000882309F4B3C13110B1C189E190E00E9425
:10306000B9A81C01DC0111961C930E9313961C92B7
:103070001E92129715961C921E9214971796FC9208
:10308000EE9216971996DC92CE92189758961C924B
:103090000E94955025EE33E0F10131832083309278
:1030A000511220925012C1010E94C73485C18091F3
:1030B0005412882309F482C1711080C18CE190E020
:1030C0000E94B9A89C01DC0111961C930E93E7E0C5
:1030D000F0E01396FC93EE93129715961C921E92B5
:1030E00014971796FC92EE9216971996DC92CE9250
:1030F000189758961C9228A739A70E94955028A582
:1031000039A5E9E7F5E0D901ED93FC93309353122B
:1031100020935212C9010E948635772473944EC1C0
:1031200080915712882309F449C1911047C18CE15D
:1031300090E00E94B9A89C01DC0111961C930E93AB
:10314000E6E0F0E01396FC93EE93129715961C922E
:103150001E9214971796FC92EE9216971996DC928F
:10316000CE92189758961C9228A739A70E9495507E
:1031700028A539A5E9E7F5E0D901ED93FC93309353
:10318000561220935512C9010E94863599249394B2
:1031900015C180915A12882309F410C161100EC123
:1031A0008CE190E00E94B9A89C01DC0111961C936F
:1031B0000E93E5E0F0E01396FC93EE9312971596CC
:1031C0001C921E9214971796FC92EE9216971996DF
:1031D000DC92CE92189758961C9228A739A70E9485
:1031E000955028A539A5E9E7F5E0D901ED93FC93C1
:1031F0003093591220935812C9010E9486356624D3
:103200006394DCC080915D12882309F4D7C051100B
:10321000D5C08CE190E00E94B9A89C01DC01119618
:103220001C930E93E4E0F0E01396FC93EE93129758
:1032300015961C921E9214971796FC92EE92169772
:103240001996DC92CE92189758961C9228A739A707
:103250000E94955028A539A5E9E7F5E0D901ED933D
:10326000FC9330935C1220935B12C9010E94863557
:1032700055245394A3C080916012882309F49EC002
:1032800041109CC08CE190E00E94B9A89C01DC0137
:1032900011961C930E93E2E0F0E01396FC93EE93EC
:1032A000129715961C921E9214971796FC92EE9206
:1032B00016971996DC92CE92189758961C9228A7CA
:1032C00039A70E94955028A539A5E9E7F5E0D9016D
:1032D000ED93FC9330935F1220935E12C9010E941C
:1032E0008635442443946AC080916312882309F48C
:1032F00065C0811063C08CE190E00E94B9A89C0178
:10330000DC0111961C930E93E1E0F0E01396FC9320
:10331000EE93129715961C921E9214971796FC9294
:10332000EE9216971996DC92CE92189758961C92A8
:1033300028A739A70E94955028A539A5E9E7F5E007
:10334000D901ED93FC933093621220936112C9016D
:103350000E9486358824839431C080916612882328
:1033600069F131102BC08CE190E00E94B9A81C01DA
:10337000DC0111961C930E9313961C921E921297C9
:1033800015961C921E9214971796FC92EE92169721
:103390001996DC92CE92189758961C920E949550DE
:1033A00029E735E0F10131832083309265122092C4
:1033B0006412C1010E9486353324339433E0A30E96
:1033C000B11C88E7A816B10409F0DFCCC4CC82E0B8
:1033D0000E943C63882311F01DA216C081E00E9468
:1033E0003C63882329F082E00E94206381116EC62D
:1033F0008CE30E945045892B09F059C68CE30E944A
:103400005045892B09F059C686E0E0E3F0E1DE0182
:10341000549601900D928A95E1F780912910909031
:103420003910A0902A10B0902B1090912C10709110
:103430002D1060912E1050912F1040913610209138
:10344000371030913810E0915606F0915706FFA3DF
:10345000EEA30091900E1091910E50905710E090B5
:103460005010F090511070905A1060905910C09008
:10347000C20FD090C30F4090C50F3090C00F209066
:10348000C10FFDA1FB8B8A8F9B8EAC8EBD8E9E8F54
:103490007F8F68A359A34AA33CA32BA3F2E18F2EED
:1034A000FE017396DE01119601900D928A94E1F768
:1034B000ECE8FAE0F093C405E093C305ADA1A9835D
:1034C00088879986AA86BB869C877D876E875F875B
:1034D000488B3A8B298B22E1FE013196A0EDB5E0B5
:1034E00001900D922A95E1F720923E0E30923F0E08
:1034F00040923D0ED0928B0EC0928A0E5092920E48
:1035000060928F0E70928E0EF0928D0EE0928C0E65
:1035100010933C0E00933B0E2EA13FA13093C605A5
:103520002093C505911107C01092DC05811103C0DD
:103530001092620AA3C081E08093620A00915D0A42
:1035400010915E0A8091EE0960E00E94A745D801C3
:10355000ED91FC910190F081E02DC80119958091C9
:10356000D005882359F1813071F08330C1F488E2AD
:1035700093E29093D2058093D10589E08093D5059D
:1035800080E197E217C088EB9BE09093D20580938F
:10359000D10583E08093D50588E99AE30BC088E8DC
:1035A00093E19093D2058093D10586E08093D50571
:1035B00080EE9EE29093D4058093D3058091D70549
:1035C0008823E9F18091DB056091D50570E08823BF
:1035D000C9F08091DD058823A9F080E090E00E9489
:1035E000BDAB9B01AC0160E070E088EC92E40E940E
:1035F00018A86093C7057093C8058093C905909378
:10360000CA0525C080E090E00E94BDAB9B01AC01E3
:1036100060E070E088EC92E40E9418A86093C7050F
:103620007093C8058093C9059093CA051092BE0592
:103630001092BF051092C0051092C1051FC01092D4
:10364000C7051092C8051092C9051092CA0560916D
:10365000D60570E080E090E00E94BDAB9B01AC011C
:1036600060E070E088EC92E40E9418A86093BE05C8
:103670007093BF058093C0059093C1051092E30538
:103680001092CF051092C2051092CB051092CC0576
:103690001092CD051092CE050E94BC6C6E98769A61
:1036A000EE9880916A008F7C80936A0080913F0E33
:1036B000882321F080916A00806203C080916A00B3
:1036C000806380936A00EE980E945C6F80E090E0D7
:1036D00040E09C012856314FF901ED55FF4F5081D4
:1036E000552331F0329720813181232B09F04F5F30
:1036F00003968837910569F74093E805A7EFB5E091
:1037000020E030E08DE3282E84E6382E9AE4492E1E
:1037100094E6592E44E7642E44E8742E57E5852E2E
:1037200054E6952E6CE5A62E64E6B62E4EE554E6DC
:1037300000E614E675E6E72E74E6F72EE7E6CE2EF1
:10374000E4E6DE2EC9018856914FFC01ED55FF4F8E
:103750006081662309F4B4C28F559F4FFC018081BC
:103760009181892B09F4ACC270E0FB013197E337FA
:10377000F10508F0A5C28827E355FF4F8F4F0C9441
:103780009FA780E89AE711969C938E9399C28EE743
:103790009AE711969C938E9393C28CE79AE71196C1
:1037A0009C938E938DC285E79AE711969C938E9396
:1037B00087C283E79AE711969C938E9381C287E133
:1037C0009AE711969C938E937BC289E19AE71196B2
:1037D0009C938E9375C28AEF99E711969C938E9372
:1037E0006FC286EE99E711969C938E9369C287ED1E
:1037F00099E711969C938E9363C28BE799E7119694
:103800009C938E935DC282E399E711969C938E936D
:1038100057C286E299E711969C938E9351C28AE132
:1038200099E711969C938E934BC28FE099E711967E
:103830009C938E9345C288E199E711969C938E9351
:103840003FC281E199E711969C938E9339C281E63C
:1038500097E611969C938E9333C28FE597E6119667
:103860009C938E932DC28DE597E611969C938E9333
:1038700027C28DE497E611969C938E9321C28BE428
:1038800097E611969C938E931BC289E497E6119656
:103890009C938E9315C289E397E611969C938E9321
:1038A0000FC287E397E611969C938E9309C285E336
:1038B00097E611969C938E9303C284E194E6119649
:1038C0009C938E93FDC182E194E611969C938E9316
:1038D000F7C180E194E611969C938E93F1C188E63E
:1038E00092E711969C938E93EBC182E297E6119634
:1038F0009C938E93E5C180EB94E611969C938E93F6
:10390000DFC181E994E611969C938E93D9C180E240
:1039100097E611969C938E93D3C181EF96E611960C
:103920009C938E93CDC18AEE96E611969C938E93CE
:10393000C7C189EB96E611969C938E93C1C189E825
:103940009AE711969C938E93BBC187EB96E61196EE
:103950009C938E93B5C185EB96E611969C938E93BE
:10396000AFC18AE996E611969C938E93A9C18FE721
:1039700096E611969C938E93A3C184E696E61196E3
:103980009C938E939DC189E496E611969C938E93A9
:1039900097C18EE296E611969C938E9391C183E136
:1039A00096E611969C938E938BC188EF95E61196BF
:1039B0009C938E9385C18DED95E611969C938E9385
:1039C0007FC182EC95E611969C938E9379C187EA2C
:1039D00095E611969C938E9373C18CE895E61196AB
:1039E0009C938E936DC181E795E611969C938E937F
:1039F00067C186E595E611969C938E9361C18BE332
:103A000095E611969C938E935BC180E295E61196A4
:103A10009C938E9355C185E095E611969C938E9369
:103A20004FC18AEE94E611969C938E9349C18FEC18
:103A300094E611969C938E9343C182E094E611968E
:103A40009C938E933DC181E094E611969C938E9356
:103A500037C180E094E611969C938E9331C18EE736
:103A600094E611969C938E932BC180EF93E611966A
:103A70009C938E9325C18EEE93E611969C938E9324
:103A80001FC18CEE93E611969C938E9319C189E623
:103A900094E611969C938E9313C185E194E8119658
:103AA0009C938E930DC18BEC93E811969C938E930F
:103AB00007C180E690E611969C938E9301C18CE439
:103AC00090E611969C938E93FBC088E390E6119646
:103AD0009C938E93F5C087EE98E711969C938E93F6
:103AE000EFC08AE093E811969C938E93E9C088EF2B
:103AF00092E811969C938E93E3C081E492E811962C
:103B00009C938E93DDC08FE292E811969C938E93E6
:103B1000D7C08FEB93E811969C938E93D1C083EB23
:103B200093E811969C938E93CBC087EA93E8119605
:103B30009C938E93C5C08BE993E811969C938E93CA
:103B4000BFC08FE893E811969C938E93B9C083E829
:103B500093E811969C938E93B3C087E793E81196F0
:103B60009C938E93ADC08FEB92E811969C938E93AD
:103B7000A7C08DEA92E811969C938E93A1C08BE921
:103B800092E811969C938E939BC089E892E81196D7
:103B90009C938E9395C087E792E811969C938E93A1
:103BA0008FC085E692E811969C938E9389C083E539
:103BB00092E811969C938E9383C01196DC92CE92DC
:103BC0007FC01196FC92EE927BC011961C930E93CF
:103BD00077C087EA94E811969C938E9371C01196F2
:103BE0005C934E936DC01196BC92AE9269C01196D3
:103BF0009C928E9265C011967C926E9261C01196D5
:103C00005C924E925DC011963C922E9259C0E2E5B4
:103C1000F3E81196FC93EE9353C08DE293E811966E
:103C20009C938E934DC0EBE3F4E61196FC93EE93D8
:103C300047C086E190E611969C938E9341C0E3E0E5
:103C4000F0E61196FC93EE933BC08EE290E611965F
:103C50009C938E9335C0E9E3F4E61196FC93EE93C2
:103C60002FC087E394E611969C938E9329C0EFE2D0
:103C7000F4E61196FC93EE9323C084E294E6119649
:103C80009C938E931DC0EDE2F4E61196FC93EE93A7
:103C900017C086E294E611969C938E9311C0EBEECA
:103CA000F2E81196FC93EE930BC08EED92E811961C
:103CB0009C938E9305C0E1EDF2E81196FC93EE9390
:103CC0002D5F3F4F12962837310509F03BCD1092FA
:103CD000E9058091EE05811114C080E090E0FC01BF
:103CE000E75CF04F208131812456310924363105BB
:103CF00028F003968837910591F703C081E08093FF
:103D0000E9051092F0058091F505811114C080E05D
:103D100090E0FC01E75CF04F20813181285C3109A3
:103D20002436310528F003968837910591F703C0B2
:103D300081E08093F0058091560690915706DC0152
:103D4000ED91FC91EC5BFF4F209106103091071034
:103D500040910410509105100190F081E02D61E038
:103D600019958091560690915706DC01ED91FC91D2
:103D7000EC5BFF4F20910A1030910B10409108101E
:103D8000509109100190F081E02D62E01995809129
:103D9000560690915706DC01ED91FC91EC5BFF4FCC
:103DA00020910E1030910F1040910C1050910D1079
:103DB0000190F081E02D63E0199580915606909175
:103DC0005706DC01ED91FC91EC5BFF4F209119103F
:103DD00030911A1040911710509118100190F081F5
:103DE000E02D64E019958091560690915706DC010C
:103DF000ED91FC91EC5BFF4F20911D1030911E1056
:103E000040911B1050911C100190F081E02D65E055
:103E100019958091560690915706DC01ED91FC9121
:103E2000EC5BFF4F209121103091221040911F1028
:103E3000509120100190F081E02D66E0199580915D
:103E4000560690915706DC01ED91FC91EA5BFF4F1D
:103E50000190F081E02D4091101061E01995809162
:103E6000560690915706DC01ED91FC91EA5BFF4FFD
:103E70000190F081E02D4091111062E01995809140
:103E8000560690915706DC01ED91FC91EA5BFF4FDD
:103E90000190F081E02D4091121063E0199580911E
:103EA000560690915706DC01ED91FC91EA5BFF4FBD
:103EB0000190F081E02D4091231064E019958091EC
:103EC000560690915706DC01ED91FC91EA5BFF4F9D
:103ED0000190F081E02D4091241065E019958091CA
:103EE000560690915706DC01ED91FC91EA5BFF4F7D
:103EF0000190F081E02D4091251066E019958091A8
:103F0000560690915706DC01ED91FC9106A8F7A9A1
:103F1000E02D6091141019958091560690915706E6
:103F2000DC01ED91FC9104A4F5A5E02D6091151044
:103F300019958091560690915706DC01ED91FC9100
:103F400002A8F3A9E02D60911610199580E090E089
:103F50009C012856314FF901ED55FF4F4081423702
:103F600031F4329720813181232B09F0B5C00396BB
:103F70008837910569F70E94157B809156069091CC
:103F80005706DC01ED91FC91EA5AFF4F0190F08158
:103F9000E02D40E060912610199580915606909191
:103FA0005706DC01ED91FC91EA5AFF4F0190F08138
:103FB000E02D41E06091281019958091560690916E
:103FC0005706DC01ED91FC91EA5AFF4F0190F08118
:103FD000E02D42E06091271019958091FD0F882314
:103FE00031F08091B30F8D3011F01092FD0F1092CF
:103FF000B8061092F60D8091FE0F8093B80580915F
:1040000000108093B70520914E1030E0AFEFB0E084
:104010000E9450AD24E630E040E050E00E9402AD46
:104020002093590E80914D1081110E9455740E9469
:10403000035F0E9426476B017C0110E011110FC045
:1040400080915D06882359F02CE133E840ED57E07C
:1040500060E070E08CE89AE00E943C4C11E00E9425
:104060000C39882351F00E9482730E943B620E94A7
:104070000F740E9499380E949F730E94CC5202973D
:1040800011F00E9471670E94E47B0E94CC5202975B
:10409000A9F60E942647DC01CB018C199D09AE09C7
:1040A000BF098C3B9240A105B10540F218C082E0E7
:1040B0000E943C6381110DC0A1C982E00E9420636F
:1040C000882309F4A1C9B3E0BDA39EC991E09DA3D3
:1040D0009BC9A2E0ADA398C90E94097B4ECF0E9464
:1040E000B35E0E940F748091760A811102C00E9413
:1040F00083800E94A15286E30E94AA46BC01990FC8
:10410000880B990B611571058105910511F00E94CD
:1041100044AB2AE232E848EE53E060E070E08CE81D
:104120009AE0A9960FB6F894DEBF0FBECDBFDF911F
:10413000CF911F910F91FF90EF90DF90CF90BF90A4
:10414000AF909F908F907F906F905F904F903F9037
:104150002F900C943C4C2F923F924F925F926F9213
:104160007F928F929F92AF92BF92CF92DF92EF9207
:10417000FF920F931F93CF93DF93CDB7DEB7E797EF
:104180000FB6F894DEBF0FBECDBF80915A06909156
:104190005B060E945E430E94138563EE74E080918B
:1041A0005A0690915B060E9400426DE875E0CE01D0
:1041B00001960E94C14100915A0610915B06D801F8
:1041C000ED91FC914D815E8169817A810280F3815C
:1041D000E02DC8011995C8010E945E43CE010196E9
:1041E0000E9491410E94E47B80915A0690915B0667
:1041F000DC01ED91FC910284F385E02D199580910D
:104200005A0690915B060E945E430E94138568E700
:1042100075E080915A0690915B060E940042E09101
:10422000770AE4300CF0E0E084E095E09A8389833B
:1042300080E095E09C838B838BEF94E09E838D835D
:1042400086EF94E098878F83EE0FFF0B81E090E07C
:104250008C0F9D1FE80FF91F6081718180915A06B4
:1042600090915B060E9471430E94138562E475E0A1
:1042700080915A0690915B060E9471430E941385BB
:1042800066E375E080915A0690915B060E940042B9
:10429000E0916211F091631181819281883E934097
:1042A00014F40E940385E0916211F0916311618121
:1042B000728180915A0690915B060E94FE7F84E095
:1042C0000E94228CE0916211F091631165817681E8
:1042D00080915A0690915B060E94FE7F85E00E94C5
:1042E000228CE0916211F09163116381748180915D
:1042F0005A0690915B060E94FE7F84E00E94228C09
:10430000E0916211F0916311678180915A0690915A
:104310005B060E94E47F88E00E94228CE09162119B
:10432000F091631180850E94EF846AE275E08091CC
:104330005A0690915B060E940042E0916C11F09148
:104340006D1181819281883E934014F40E9403850F
:10435000E0916C11F0916D116181728180915A062A
:1043600090915B060E94FE7F84E00E94228CE09187
:104370006C11F0916D116581768180915A06909152
:104380005B060E94FE7F85E00E94228CE0916C110A
:10439000F0916D116381748180915A0690915B0652
:1043A0000E94FE7F84E00E94228CE0916C11F091CB
:1043B0006D11678180915A0690915B060E94E47F9F
:1043C00088E00E94228CE0916C11F0916D11808543
:1043D0000E94EF846EE175E080915A0690915B0631
:1043E0000E940042E0917611F091771181819281D3
:1043F000883E934014F40E940385E0917611F09179
:1044000077116181728180915A0690915B060E94BA
:10441000FE7F84E00E94228CE0917611F09177116A
:104420006581768180915A0690915B060E94FE7F9D
:1044300085E00E94228CE0917611F09177116381E2
:10444000748180915A0690915B060E94FE7F84E001
:104450000E94228CE0917611F09177116781809112
:104460005A0690915B060E94E47F88E00E94228CAD
:10447000E0917611F091771180850E94EF8462E1DE
:1044800075E080915A0690915B060E940042E0918F
:104490008011F091811181819281883E934014F4C2
:1044A0000E940385E0918011F091811161817281F8
:1044B00080915A0690915B060E94FE7F84E00E94E4
:1044C000228CE0918011F09181116581768180913B
:1044D0005A0690915B060E94FE7F85E00E94228C26
:1044E000E0918011F09181116381748180915A066D
:1044F00090915B060E94FE7F84E00E94228CE091F6
:104500008011F0918111678180915A0690915B062C
:104510000E94E47F88E00E94228CE0918011F0915B
:10452000811180850E94EF8480915A0690915B06EC
:104530000E945E430E94A152C82E6AEA75E08091F3
:104540005A0690915B060E9471430E94138501E018
:1045500011E1E12CF12CD12C57012FEFA21AB20A54
:10456000B50180915A0690915B060E94FE7F49E05A
:10457000E416F10410F48BE001C08AE00E94228C62
:10458000D8012C9180915A0690915B062223C9F1A3
:104590001596ED91FC911697618172810E94FE7FC4
:1045A000D8011596ED91FC91169781819281883EF4
:1045B000934014F40E94038584E00E94228CD80169
:1045C0001596ED91FC9116976381748180915A063E
:1045D00090915B060E94FE7F84E00E94228CD801AD
:1045E0001596ED91FC911697278180915A0690912E
:1045F0005B06222319F062EA75E00BC06BE975E0F7
:1046000008C0EC14FD041CF463E975E002C066E820
:1046100075E00E947143095F1F4F7501BCE0AB1646
:10462000B10409F099CF0E9413856FED75E0809178
:104630005A0690915B060E9400420E94A152682F88
:1046400080915A0690915B060E94BA7E6BEC75E0F1
:1046500080915A0690915B060E9400426091740A14
:104660007091750A80915A0690915B060E94348081
:104670000E94E47B80915A0690915B06DC01ED91EB
:10468000FC910284F385E02D199580915A06909152
:104690005B060E945E430E9413856FE776E080917F
:1046A0005A0690915B060E9471430E9413856BE647
:1046B00076E080915A0690915B060E9400428091BC
:1046C000B10F0E94C43ABC0180915A0690915B06DA
:1046D0000E94714367E576E080915A0690915B06EF
:1046E0000E9400428091B20F0E94C43ABC018091A6
:1046F0005A0690915B060E9400422091B20F809171
:104700005A0690915B062B303CF4293054F4283043
:1047100069F466E476E007C02B3041F462E576E0A8
:1047200002C06CE476E00E94714302C00E945E43C6
:1047300062E376E080915A0690915B060E94004207
:104740008091B30F0E94C43ABC0180915A069091A7
:104750005B060E9400422091B30F80915A0690910F
:104760005B062B303CF4293054F4283069F461E2C4
:1047700076E007C02B3041F46DE276E002C067E2DC
:1047800076E00E94714302C00E945E436DE076E0D5
:1047900080915A0690915B060E9400422091C00FC2
:1047A00080915A0690915B06222319F065E076E02D
:1047B00002C063EF75E00E94004280915A0690911A
:1047C0005B060E945E430E94E47B80915A069091B2
:1047D0005B06DC01ED91FC910284F385E02D1995D7
:1047E00080910002823011F40C94522CF090D70F7B
:1047F0000091DA0F11E080915A0690915B060E94B9
:104800005E430E9413856CEF78E080915A06909188
:104810005B060E9471430E94138563EE78E08091ED
:104820005A0690915B060E940042E091ED0FE53040
:104830000CF0E0E08FEA96E09A8389838AEA96E0BA
:104840009C838B8380EA96E09E838D838CE996E03F
:1048500098878F838BE896E09A878987EE0FFF0B06
:1048600081E090E08C0F9D1FE80FF91F608171813E
:1048700080915A0690915B060E9471436AEC78E041
:1048800080915A0690915B060E940042609100025E
:1048900080915A0690915B060E94BA7E61EB78E0A7
:1048A00080915A0690915B060E9400428F2D0E94D3
:1048B000DA84FF2009F44AC067EA78E080915A065A
:1048C00090915B060E94004280915A0690915B068F
:1048D000112339F06091D80F0E94E47F9091D80F96
:1048E00006C06091DE0F0E94E47F9091DE0F809100
:1048F0007A129813DEC76BE878E080915A0690919F
:104900005B060E94004280915A0690915B0611233B
:1049100039F06091D90F61110CC066E878E006C0EB
:104920006091DF0F611105C061E878E00E940042EC
:1049300005C0062E000C770B0E94FE7F6FE778E023
:1049400080915A0690915B060E94004280915A061F
:1049500090915B060E945E4366E678E080915A067D
:1049600090915B060E940042802F0E94DA8400230F
:1049700009F44AC06CE578E080915A0690915B0694
:104980000E94004280915A0690915B06112339F0F3
:104990006091DB0F0E94E47F9091DB0F06C0609175
:1049A000E10F0E94E47F9091E10F80917C129813B7
:1049B00099C760E478E080915A0690915B060E9466
:1049C000004280915A0690915B06112339F0609164
:1049D000DC0F61110CC06BE378E006C06091E20F60
:1049E000611105C066E378E00E94004205C0062E12
:1049F000000C770B0E94FE7F64E378E080915A06FA
:104A000090915B060E94004280915A0690915B064D
:104A10000E945E436BE178E080915A0690915B06BC
:104A20000E9400428091F60F811103C00E94E88429
:104A300035C067EB76E080915A0690915B060E9444
:104A4000004268E178E080915A0690915B060E94EE
:104A500000426091F60F80915A0690915B060E9489
:104A6000E47F68E078E080915A0690915B060E94AE
:104A700000424091F70F5091F80F60E070E02AE09B
:104A800080915A0690915B060E94394263E078E07B
:104A900080915A0690915B060E9471436AEE77E01E
:104AA00080915A0690915B060E9400428091EE0F21
:104AB0008436C8F463EE77E080915A0690915B06E5
:104AC0000E9400426091EE0F80915A0690915B0621
:104AD0000E94E47F61EE77E080915A0690915B0638
:104AE0000E94714303C080E00E94E88468EC77E094
:104AF00080915A0690915B060E9400428091EF0FD0
:104B00008436C8F461EC77E080915A0690915B0698
:104B10000E9400426091EF0F80915A0690915B06CF
:104B20000E94E47F6FEB77E080915A0690915B06DC
:104B30000E94714303C080E00E94E88466EA77E047
:104B400080915A0690915B060E9400426091E40FAA
:104B50007091E50F072E000C880B990B0E94BFABDC
:104B600020E030E04AE754E40E9418A8AB01BC0101
:104B700021E080915A0690915B060E94814261EA91
:104B800077E080915A0690915B060E94714368E835
:104B900077E080915A0690915B060E9400426091F6
:104BA000E60F7091E70F072E000C880B990B0E94FF
:104BB000BFAB20E030E04AE754E40E9418A8AB0104
:104BC000BC0121E080915A0690915B060E948142CF
:104BD00063E877E080915A0690915B060E947143EA
:104BE0006AE677E080915A0690915B060E94004247
:104BF0006091E80F7091E90F072E000C880B990B5C
:104C00000E94BFAB20E030E04AE754E40E9418A8BD
:104C1000AB01BC0121E080915A0690915B060E9495
:104C2000814265E677E080915A0690915B060E948A
:104C300071436CE477E080915A0690915B060E9484
:104C400000428091ED0F813011F08430D9F48091D1
:104C5000EA0F0E94DA848091EA0F8823D9F068E491
:104C600077E080915A0690915B060E940042609125
:104C7000EB0F80915A0690915B060E94E47F66E4F8
:104C800077E002C061E377E080915A0690915B067D
:104C90000E94004280915A0690915B060E945E43FA
:104CA00068E177E080915A0690915B060E9400428D
:104CB0009091ED0F2FEF290F80915A0690915B068E
:104CC000223028F46091B9050E94BA7E04C063E0E6
:104CD00077E00E9471436AEE76E080915A069091E7
:104CE0005B060E9400428091FA0F0E94DA84809154
:104CF000FA0F882341F168ED76E080915A06909191
:104D00005B060E9400426091FB0F80915A069091D1
:104D10005B060E94E47F60EC76E080915A069091F9
:104D20005B060E9400426091FC0F80915A069091B0
:104D30005B060E94E47F6EEB76E080915A069091CC
:104D40005B060E94004280915A0690915B060E9489
:104D50005E430E94E47B80915A0690915B06DC01E1
:104D6000ED91FC910284F385E02D199580915A060E
:104D700090915B060E945E430E94138565E879E08E
:104D800080915A0690915B060E9471430E941385A0
:104D900064E679E080915A0690915B060E94004299
:104DA0008091BA0F8436C8F46DE579E080915A0697
:104DB00090915B060E9400426091BA0F80915A0662
:104DC00090915B060E94E47F6BE579E080915A0642
:104DD00090915B060E94714303C080E00E94E884CA
:104DE0006AE379E080915A0690915B060E94004246
:104DF0008091B90F8436C8F463E379E080915A0654
:104E000090915B060E9400426091B90F80915A0612
:104E100090915B060E94E47F61E379E080915A06FD
:104E200090915B060E94714303C080E00E94E88479
:104E300060E179E080915A0690915B060E94004201
:104E40006091C20F7091C30F1616170614F50091EA
:104E50005A0610915B06072E000C880B990B0E94D6
:104E6000BFAB20E030E04AE754E40E9418A8AB0151
:104E7000BC0122E0C8010E948142C8010E945E4339
:104E80006BE079E080915A0690915B060E94714335
:104E900003C080E00E94E8840E94E47B80915A066F
:104EA00090915B06DC01ED91FC910284F385E02D8D
:104EB000199580915A0690915B060E945E430E946C
:104EC000138565EF7AE080915A0690915B060E9407
:104ED00071430E9413852091D70580915A069091C5
:104EE0005B06222309F4BFC166EC7AE00E9400420F
:104EF0000E9440760E94E8840E94407620915A06E3
:104F000030915B06882389F063EB7AE0C9010E9447
:104F100000428091DA050E947155BC0180915A06C9
:104F200090915B060E9471434FC060EA7AE0C9012C
:104F30000E9400428091D7050E947155BC0180916A
:104F40005A0690915B060E9400428091D805882302
:104F5000A9F168E97AE080915A0690915B060E9477
:104F60000042E091D805E4300CF0E0E085EF92E0FB
:104F70009A83898383EF92E09C838B8381EF92E015
:104F80009E838D838FEE92E098878F83EE0FFF0BC9
:104F900081E090E08C0F9D1FE80FF91F6081718107
:104FA00080915A0690915B060E94004266E97AE081
:104FB00080915A0690915B060E94004280915A06A9
:104FC00090915B060E945E4363E87AE080915A0606
:104FD00090915B060E9400428091D90500915A068B
:104FE00010915B06882321F00E947155BC0102C01C
:104FF0006FE77AE0C8010E9471436CE67AE0809125
:105000005A0690915B060E9400428091DA05009159
:105010005A0610915B06882321F00E947155BC014D
:1050200002C068E67AE0C8010E94714365E57AE053
:1050300080915A0690915B060E9400428091DC05A7
:105040008823E1F06FE47AE080915A0690915B0644
:105050000E9400428091DB050E947155BC01809145
:105060005A0690915B060E94004265E975E08091C6
:105070005A0690915B060E94614303C080E00E9443
:10508000E8846CE37AE080915A0690915B060E9476
:1050900000428091DD058823E1F066E37AE08091AB
:1050A0005A0690915B060E9400428091DB050E94A7
:1050B0007155BC0180915A0690915B060E94004296
:1050C00065E975E080915A0690915B060E94614304
:1050D00003C080E00E94E88463E27AE080915A068F
:1050E00090915B060E940042E091DE05E2300CF0F8
:1050F000E2E08BEC99E09A8389838FEB99E09C83C3
:105100008B8387EB99E09E838D83EE0FFF0BA1E0ED
:10511000B0E0AC0FBD1FEA0FFB1F60817181809171
:105120005A0690915B060E94714360E17AE080919B
:105130005A0690915B060E940042E091D005E4304F
:105140000CF0E4E080EB99E09A8389838AEA99E0A5
:105150009C838B8383EA99E09E838D838DE999E01C
:1051600098878F8385E999E09A878987EE0FFF0BEF
:1051700081E090E08C0F9D1FE80FF91F6081718125
:1051800080915A0690915B060E9471436EE07AE02E
:1051900080915A0690915B060E9400426091D5056D
:1051A00080915A0690915B060E94E47F6FEF79E050
:1051B00080915A0690915B060E9400428091D00532
:1051C000811110C06091D60580915A0690915B06BE
:1051D0000E94E47F64EF79E080915A0690915B062B
:1051E0000E9400426091D1057091D205072E000CFB
:1051F000880B990B0E94BFAB20E030E04AE754E4F3
:105200000E9418A8AB01BC0121E080915A06909140
:105210005B060E94814266EE79E080915A06909189
:105220005B060E9400426091D3057091D405072E61
:10523000000C880B990B0E94BFAB20E030E04AE7DE
:1052400054E40E9418A8AB01BC0121E080915A06E9
:1052500090915B060E94814267ED79E080915A0649
:1052600090915B0602C069ED7AE00E9471430E9452
:10527000E47B80915A0690915B06DC01ED91FC91F4
:105280000284F385E02D199580915A0690915B0672
:105290000E945E430E94138560E67BE080915A067F
:1052A00090915B060E9471430E94138563E57BE049
:1052B00080915A0690915B060E940042E091031093
:1052C000E4300CF0E4E081E49BE09A8389838AE295
:1052D0009BE09C838B8388E19BE09E838D8389E0A8
:1052E0009BE098878F8381E09BE09A878987EE0F08
:1052F000FF0B81E090E08C0F9D1FE80FF91F60818C
:10530000718180915A0690915B060E9471430E94C0
:10531000E47B80915A0690915B06DC01ED91FC9153
:105320000284F385E02D199580915A0690915B06D1
:105330000E945E430E94138560EE7BE080915A06D6
:1053400090915B060E9471430E9413852091B806DC
:1053500080915A0690915B062223C9F169EA7BE0AD
:105360000E94004280915A0690915B060E945E4323
:105370006AE87BE080915A0690915B060E940042A9
:105380008091FD0F0E94DA848091FD0F81110E94AF
:10539000A58C80915A0690915B060E945E436BE655
:1053A0007BE080915A0690915B060E9400428091BA
:1053B000FF0F0E94DA848091FF0F81110E94778C89
:1053C00080915A0690915B060E945E4304C06BEC8C
:1053D0007BE00E9471430E94E47B80915A06909189
:1053E0005B06DC01ED91FC910284F385E02D1995BB
:1053F00082E39BE5A1E0BB278BAB9CABADABBEAB27
:1054000080915A0690915B060E945E430E9413852C
:105410006AE37DE080915A0690915B060E94714399
:105420000E94138561E27DE080915A0690915B06AF
:105430000E9400422091720A80915A0690915B0668
:10544000222319F06DE17DE002C068E17DE00E9459
:1054500071438091720A882349F16FEF7CE080915B
:105460005A0690915B060E94004260910110709173
:105470000210072E000C880B990B0E94BFAB20E096
:1054800030E04AE754E40E9418A8AB01BC0122E0D6
:1054900080915A0690915B060E9481426AEF7CE0FF
:1054A00080915A0690915B060E9471439BE3E92E1E
:1054B0009FE0F92E28E1422E2CEF522E3AE0A32E47
:1054C000B12C44E6C42ED12C5EE0252ED7012C91C0
:1054D000222309F4A5C1F70132970081118101153A
:1054E000110509F49DC18EEB9AE5A1E0BB27820F5F
:1054F000911DA11DB11DABBFFC01879133243394D5
:10550000811101C0312C20915A0630915B06C801EF
:105510000197849790F56AED7CE0C9010E940042F2
:1055200009500C3148F4E02FF0E0EE0FFF1FE3517B
:10553000FC4F6081718102C06AEF7BE080915A0666
:1055400090915B060E9400420C3130F4E02FF0E0B5
:10555000EB5DFB4F808101C080E090E08053934F72
:10556000092E000CAA0BBB0BABBFFC018791B22D1F
:10557000B81B8B2F09F0FBC0FCC0C80184569109F1
:105580008438934008F03FC060EC7CE0C9010E9481
:105590000042C801B6010E9478A76130710531F060
:1055A0006230710559F46CEB7CE002C06EEB7CE07C
:1055B00080915A0690915B060E9400420E940B85E2
:1055C00080905A0690905B063320B1F0C8010E948B
:1055D000CC7A811107C068EB7CE0C4010E940042D4
:1055E00087E0C5C0813009F0C4C065EB7CE0C40130
:1055F0000E94004288E0BBC06CEA7CE0C4010E94CB
:10560000004282E0B4C0C801885E93408035964471
:1056100008F069C0C80168EE73E00E9478A74B01EA
:105620006FE97CE0C9010E9400422AE082169104E1
:1056300010F40E940385B40180915A0690915B0694
:105640000E94FE7F0E940B8560905A0670905B0658
:10565000332009F442C0C8010E94CC7A282F6AE99D
:105660007CE0C3012FAB0E940042849CC001859C5A
:10567000900D949C900D1124800F911FB5010E94F4
:105680008CA780915A0690915B062FA9633059F040
:105690006530C9F0623009F06CC0243008F03BC1BD
:1056A00061E97CE03AC1233018F46FE77CE035C152
:1056B000233019F466E77CE030C1243008F459C087
:1056C0006DE67CE02AC1622F0E94E47F65E67CE003
:1056D00080915A0690915B0620C16CE57CE0C30185
:1056E0000E94004243C0C80188539A44883E9340B8
:1056F00000F509338AE4180771F00A339AE41907B0
:1057000089F008331A44A9F56DE47CE0C9010E94D0
:1057100000428FE02CC062E47CE0C9010E9400429C
:1057200083E125C060E37CE0C9010E9400428CE077
:105730001EC0C80180529E44883E934020F400520F
:1057400069E17CE009C0C80188509245883E9340D9
:1057500080F4085062E07CE0C9010E9400420A30F7
:1057600010F40E940385802F0E945F8484E00E94D1
:10577000228C65EF7CE080915A0690915B060E9436
:1057800000426AEE7CE080915A0690915B060E948E
:105790000042D7016C9170E080915A0690915B06AF
:1057A0000E94FE7FF70180818A3010F40E940385F9
:1057B0000E940B85D7014C91B9E2B49FA00111243E
:1057C000052E000C660B770B8BA99CA9ADA9BEA971
:1057D000480F591F6A1F7B1FDE0111968A019B012A
:1057E0000F5F1F4F2F4F3F4F6BBFFA0187918D9374
:1057F000B901A8018111F2CFBE016F5F7F4F809187
:105800005A0690915B060E94614380915A069091DE
:105810005B06DC01ED91FC910284F385E02D199586
:10582000B3E0EB0EF11CE3EBEE16EFE0FE0609F041
:105830004DCE0E94E47B80915A0690915B06DC017C
:10584000ED91FC910284F385E02D199580915A0623
:1058500090915B060E945E430E9413856BE97DE098
:1058600080915A0690915B060E9471430E941385B5
:1058700068E87DE080915A0690915B060E940042A4
:105880000E94F67420E030E040E050E40E94B9ABA2
:1058900020915A0630915B0687FF42C065E87DE0A3
:1058A000C9015CC0F090DD0F0091E00F10E00C9496
:1058B000FB2368E978E080915A0690915B060E948C
:1058C000004260917A1280915A0690915B060E9484
:1058D000E47F66E978E080915A0690915B060E9429
:1058E000004209C86DE478E080915A0690915B0609
:1058F0000E94004260917C1280915A0690915B0652
:105900000E94E47F6BE478E080915A0690915B06F8
:105910000E9400424EC868E87CE00E94004229CF05
:1059200061E87DE0C9010E9471436EE67DE08091EF
:105930005A0690915B060E9400420E94F674AB01E9
:10594000BC0122E080915A0690915B060E94814240
:105950006CE67DE080915A0690915B060E9471434F
:1059600069E57DE080915A0690915B060E940042B5
:1059700080914A100E94DA8420914A1080915A0640
:1059800090915B06222379F066E57DE00E9400425B
:105990000E94608C6CE47DE080915A0690915B06D9
:1059A0000E94714302C00E945E430E94E47B80918A
:1059B0005A0690915B06DC01ED91FC910284F3851F
:1059C000E02D199580915A0690915B060E945E43E6
:1059D0000E94138563EF7DE080915A0690915B06EB
:1059E0000E9471430E9413856FED7DE080915A06FD
:1059F00090915B060E94004240913A1050913B10FA
:105A000060913C1070913D1080915A0690915B0618
:105A10000E94EB7F6BEC7DE080915A0690915B06D3
:105A20000E940042409142105091431060914410F6
:105A30007091451080915A0690915B060E94EB7F11
:105A400067EB7DE080915A0690915B060E940042D0
:105A500040913E1050913F10609140107091411064
:105A600080915A0690915B060E94EB7F63EA7DE08D
:105A700080915A0690915B060E9400424091461028
:105A800050914710609148107091491080915A06CA
:105A900090915B060E94EB7F0E94E47B80915A0606
:105AA00090915B06DC01ED91FC910284F385E02D81
:105AB000199580915A0690915B060E945E430E9460
:105AC0001385E7960FB6F894DEBF0FBECDBFDF910A
:105AD000CF911F910F91FF90EF90DF90CF90BF90EB
:105AE000AF909F908F907F906F905F904F903F907E
:105AF0002F9008952F923F924F925F926F927F92D4
:105B00008F929F92AF92BF92CF92DF92EF92FF92CD
:105B10000F931F93CF93DF93CDB7DEB7C65AD1094A
:105B20000FB6F894DEBF0FBECDBFCDB6DEB6CC55F6
:105B3000DF4F1882C45AD040CD55DF4F1882C35A68
:105B4000D0408091D00C8A3709F447C0C0F4873721
:105B500009F4D9C238F48F3109F435C5863709F410
:105B6000E2C1F7C5883709F4DDC2893709F0F1C50C
:105B70000E948A520E9426472B013C0129C08E3781
:105B800009F42EC338F48B3709F4CAC18C3709F4F1
:105B9000D8C2DFC5813809F407C5823809F4EDC4DD
:105BA000803809F0D6C565C40E942647DC01CB01C8
:105BB00084199509A609B70980329340A105B1055A
:105BC00008F00CC50E9471670E948A520E944A6BBD
:105BD0000E94CC52029741F701C50E94CC52029715
:105BE00029F060E084E80E940D6C8BC18091770AF7
:105BF000823031F0833039F482E08093120E03C09A
:105C000081E08093970D81E08093DA0C8E010C5532
:105C10001F4F2BE0AE0144575F4F68E871E90E94C7
:105C2000876B0E94A152893058F0015011092BE076
:105C3000AE014F575F4F68E872E981E00E94876BC1
:105C40001092D90C772473940E94B752882309F4D8
:105C50003DC1198222961FAE22978091D90C8111E5
:105C60000EC0BE0164577F4FCE018F5B9F4F0E94D5
:105C7000D7AACC55DF4F0881C45AD0400FC07092CC
:105C8000D90CBE016F577F4FCE018F5B9F4F0E9493
:105C9000D7AACD55DF4F0881C35AD0401091D90CF7
:105CA000ADB6BEB68091730AEDB7FEB722E0829F13
:105CB000E019F10911240FB6F894FEBF0FBEEDBF35
:105CC0008DB79EB701967C0161EB75E0CE018356DE
:105CD0009F4F0E94C1418091770A823089F08330C2
:105CE00061F1813009F0A1C04091730A50E0B70121
:105CF0008091700D9091710D0E943F6A10E039C043
:105D00002091730A30E05FB7F89440E0842F90E070
:105D10008217930774F4880F991FF701E80FF91F92
:105D2000DC01AA58B24F8D919C91918380834F5F83
:105D3000EDCF5FBF1092960D1CC02091730A30E02A
:105D40005FB7F89440E0842F90E08217930774F4D3
:105D5000880F991FF701E80FF91FDC01A55BB24F0F
:105D60008D919C91918380834F5FEDCF5FBF1092A7
:105D70006D0D6DE270E0CE0183569F4F0E94F040A2
:105D80002091730A293048F0112321F0113021F4B9
:105D900018E004C028E001C020E010E0121758F518
:105DA000F701E10FF11DE10FF11D608171814AE002
:105DB000CE0189569F4FCB55DF4F2883C55AD0401F
:105DC0000E949641BE0169567F4FCE0183569F4F78
:105DD0000E941741CE0189569F4F0E949141CE01EA
:105DE00083569F4F0E9408871F5FCB55DF4F288146
:105DF000C55AD040D3CF40E450E0BE016F5F7F4F23
:105E0000CE0183569F4F0E940087CF55DF4F1881E8
:105E1000C15AD040CE0183569F4F0E9491410FB688
:105E2000F894BEBE0FBEADBE0BC0CE0183569F4FD1
:105E30000E9491410FB6F894BEBE0FBEADBE10E0F9
:105E4000BE016F5F7F4FCE018F5B9F4F0E94D7AA2D
:105E5000010F10E0E1E4F0E0EC0FFD1FE00FF11F97
:105E60001082BE016F5B7F4F80910B0E90910C0EE4
:105E70000E942442B801CE018F5B9F4F0E94676B46
:105E8000BC0180910B0E90910C0E0E94FE7F6AE087
:105E900080910B0E90910C0E0E94F94180910B0E97
:105EA00090910C0EDC01ED91FC910284F385E02DC4
:105EB00019950E94A152893048F08091D90C811126
:105EC00003C07092D90C02C01092D90C0E948A5261
:105ED0000E944A6B0E94963781110CDE8091CF0C94
:105EE00081110FC08091DA0C882359F080910D0E3A
:105EF000811107C08091CD0C9091CE0C0A970CF4C3
:105F0000A3CE8091770A823039F0833009F021C422
:105F100081E08093120E1DC481E08093970D19C417
:105F20001092DA0C4DC31091D30C8FEF810F853096
:105F300028F060E089E80E940D6C0BC4133079F002
:105F400018F41230F9F004C0143079F0153099F0DB
:105F500040E6442E49E0542E612C712C19C0412C8E
:105F60003BE4532E612C712C13C0412C26E9522E98
:105F7000612C712C0DC0412C92EC592E6624639437
:105F8000712C06C080E8482E85E2582E612C712CB9
:105F900000E0E12EF12C5701BFE8AB0EB11C15015A
:105FA000E89427F83324E6E9EE0EF11CE894E7F8CC
:105FB000FF24023091F018F4013051F004C0033096
:105FC00089F00430A1F040E659E060E070E013C0D1
:105FD00040E855E260E070E00EC040E05BE460E065
:105FE00070E009C040E056E960E070E004C040E0C5
:105FF00052EC61E070E086E597E00E94FD8686E560
:1060000097E00E9415400E9426474B015C01F2E395
:106010008F0E911CA11CB11C0E940A6B0E94264786
:10602000681579058A059B05B8F360E870E086E598
:1060300097E00E948B396FE070E086E597E00E9460
:106040008B39612F86E597E00E94CF3FB10186E54D
:1060500097E00E948B390E9426474B015C012AE0A1
:10606000820E911CA11CB11C0E940A6B0E94264743
:10607000681579058A059B05B8F367E870E086E541
:1060800097E00E948B396FE070E086E597E00E9410
:106090008B39612F86E597E00E94CF3FB70186E5F7
:1060A00097E00E948B3986E597E00E9415400E9498
:1060B00026474B015C013EE5830E31E0931EA11C97
:1060C000B11C0E940A6B0E942647681579058A0553
:1060D0009B05B8F30F5F053009F06BCFB301A20148
:1060E00086E597E00E94FD86409242105092431050
:1060F0006092441070924510B301A2018AEA91E0C7
:106100000E943B875DC283E090E00E94B9A82AE02C
:10611000DC012C9326E537E012963C932E931197E1
:106120006AE00CC083E090E00E94B9A82DE0FC0179
:10613000208326E537E0328321836DE00E949B694E
:106140003FC24091D30C5091D40C0091D50C1091CA
:10615000D60C6091D10C7091D20CCE010196CB552A
:10616000DF4F4883C55AD040CA55DF4F5883C65ABF
:10617000D0400E941B59CB55DF4F4881C55AD040B3
:10618000CA55DF4F5881C65AD040892BE9F08D811E
:10619000873050F4853080F48130B0F0642F8B81EB
:1061A0009C810E9469800DC0893070F4B8018B8198
:1061B0009C810E943B8705C0BA018B819C810E9413
:1061C000067F0E94886C04C061E085E80E940D6C27
:1061D0008091CC0C8111BDC281E08093CC0CB9C2FE
:1061E000B090D10CE090D20CC956DF4F1882C7593D
:1061F000D04061EB75E0CE018F579F4F0E94C141A7
:106200006B2D7E2DCE0184579F4F0E941B59892BE9
:1062100009F4C9C0C057DF4FE881C059D0404E2FA4
:1062200050E0FA013197E830F10508F0BCC088274A
:10623000E05EFE4F8F4F0C949FA7C257DF4F8881BF
:106240009981CE58D0400E94E2AC23961FAE1EAE7C
:10625000239725961FAE1EAE259727961FAE1EAE1E
:1062600027974AE0BE016F5F7F4F90E03EC0C25764
:10627000DF4F88819981CE58D0400E94E2AC682FD0
:10628000880F770B4AE00AC0C257DF4F8881998197
:10629000CE58D0400E94EFAC4AE0BC01CE0101963E
:1062A0000E949641BE016F5F7F4FCE018F579F4F77
:1062B0000E94B740CE01019663C0C257DF4F88816C
:1062C0009981CE58D0400E94EFAC23961FAE1EAEEF
:1062D000239725961FAE1EAE259727961FAE1EAE9E
:1062E00027974AE0BE016F5F7F4F0E9490AB35C099
:1062F000C257DF4F88819981CE58D0400E94EAACC6
:1063000023961FAE1EAE239725961FAE1EAE259771
:1063100027961FAE1EAE27972AE0AE014F5F5F4F54
:106320000E9461AB1AC0C257DF4F88819981CE5855
:10633000D0400E94EAAC23961FAE1EAE239725964E
:106340001FAE1EAE259727961FAE1EAE27972AE0DA
:10635000AE014F5F5F4F0E946FABBE016F5F7F4F1B
:10636000CE018F5B9F4F0E947141BE016F5B7F4FDB
:10637000CE018F579F4F0E94B740CE018F5B9F4F3A
:106380000E9491414BE050E0BE016F5B7F4FCE0118
:106390008F579F4F0E940087CB57DF4FF880C5581B
:1063A000D04011E002C0F12C10E0CE018F579F4F7A
:1063B0000E949141112309F4BCCD8E0109561F4F53
:1063C00020E4AE014F5F5F4F68E87B2D8E2D0E9469
:1063D000876BBE016F5B7F4FCE0101960E94D7AAEB
:1063E000C956DF4F8881C759D040F80E81E08F0D24
:1063F000C956DF4F8883C759D040E1E0F0E0EC0F89
:10640000FD1FEF0DF11D9CE79083E1E0F0E0EC0F44
:10641000FD1FE80FF11D1082BE016F5F7F4F80915D
:106420000B0E90910C0E0E942442C956DF4F6881DA
:10643000C759D04070E0CE0101960E94676BBC0145
:1064400080910B0E90910C0E0E94FE7F6AE080916D
:106450000B0E90910C0E0E94F94180910B0E9091C1
:106460000C0EDC01ED91FC910284F385E02D199571
:1064700070C18091D10C9091D20C8038910509F0B7
:1064800068C18E0104571F4F20E4AE014F5F5F4F7C
:1064900068E870E880E00E94876B6DE875E0CE01E7
:1064A0008F579F4F0E94C141CE018F579F4F0E942F
:1064B0000887C457DF4F2881CC58D040CB57DF4FD7
:1064C00088819981C558D040820F911DC457DF4FF4
:1064D0008883CC58D04022961FAE22974BE050E0E4
:1064E000BE016F5B7F4FCE018F579F4F0E94078287
:1064F000BE016F5B7F4FCE0101960E94D7AAC457A1
:10650000DF4F8881CC58D040E1E0F0E0EC0FFD1F78
:10651000E80FF11D1082BE016F5F7F4F80910B0E5F
:1065200090910C0E0E942442C457DF4F6881CC58D2
:10653000D04070E0CE0101960E94676BBC01809153
:106540000B0E90910C0E0E94FE7F6AE080910B0E64
:1065500090910C0E0E94F94180910B0E90910C0EBF
:10656000DC01ED91FC910284F385E02D1995CE01BB
:106570008F579F4F0E949141ECC08091D10C909118
:10658000D20C8238910509F0E4C08E0104571F4FE8
:1065900020E4AE014F5F5F4F68E872E880E00E9440
:1065A000876B67E975E07BCF8091D10C9091D20C1D
:1065B0008138910509F0CDC08091DA0C8111C9C0F4
:1065C0000E94886CC6C08091D10C9091D20C4F97DC
:1065D00009F0BFC081E08093CF0CBBC00E94CC52B9
:1065E000029719F060E084E8A6CC8091760A8111C8
:1065F00002C00E9483800E94A152F82E61EB75E0D8
:10660000CE0184579F4F0E94C141C956DF4F188267
:10661000C759D0408E0109561F4F20E4AE014F5F8D
:106620005F4F68E879E780E00E94876BCF57DF4FC4
:1066300019821882C158D040CD57DF4F1982188275
:10664000C358D040CB57DF4F19821882C558D0406D
:106650006F2D70E080E090E02AE0AE014F5B5F4F6D
:106660000E9461ABBE016F5B7F4FCE018F579F4F82
:106670000E947141BE016F577F4FCE0184579F4FDB
:106680000E94B740CE018F579F4F0E9491414BE02F
:1066900050E0BE016F5B7F4FCE0184579F4F0E9439
:1066A0000782C057DF4F1881C059D040BE016F5BD1
:1066B0007F4FCE0101960E94D7AAC956DF4F88812D
:1066C000C759D040810F91E0980FC956DF4F98838A
:1066D000C759D040E1E0F0E0EC0FFD1FE80FF11DDD
:1066E0008CE78083E1E0F0E0EC0FFD1FE90FF11D86
:1066F0001082BE016F5F7F4F80910B0E90910C0E48
:106700000E942442C956DF4F6881C759D04070E0CB
:10671000CE0101960E94676BBC0180910B0E909197
:106720000C0E0E94FE7F6AE080910B0E90910C0E81
:106730000E94F94180910B0E90910C0EDC01ED91BD
:10674000FC910284F385E02D1995CE0184579F4F6B
:1067500011CF0FB6F894DEBE0FBECDBECA55DF4FC7
:106760000FB6F894DEBF0FBECDBFDF91CF911F9162
:106770000F91FF90EF90DF90CF90BF90AF909F90E0
:106780008F907F906F905F904F903F902F900895E3
:1067900008950895FC01828193818830910529F440
:1067A00010922B0110922A010895099721F410925A
:1067B0002901109228010895FC01178A168A6CEDB0
:1067C00075E082810C94C24FCF93DF93EC011F8A56
:1067D0001E8A8A810E943B4F8B8D882331F08A81EB
:1067E0000E94B24F9A8F898F1B8EDF91CF910895AF
:1067F000DF92EF92FF920F931F93CF93DF93EC0101
:106800008A81893010F40E94224FDD8C6B8D7C8D43
:10681000098D1A8DEA80FB8089E08E1508F466C028
:106820000F30110538F001369DE6190728F000E613
:106830001DE602C00FE010E06F30710538F06136E0
:106840008DE6780728F060E67DE602C06FE070E034
:1068500080E090E00E94BDAB20E030E04AE754E4E5
:106860000E9418A820E030E04CE852E40E941EACE0
:106870009B01AC0160E070E08AEF94E40E9418A8EC
:106880000E9480A8FF2425E12E9DF0012F9DF00D90
:106890001124EE57FE4EDD2071F023813481AB01CF
:1068A00077FF04C044275527461B570B8827992795
:1068B000841B950B0AC025813681AB0177FF04C08C
:1068C00044275527461B570BCA014FB7F89455E18B
:1068D0005E9DF0015F9DF00D1124EE57FE4E108B72
:1068E0000787328B218B948B838B4FBF9D8D6B8D54
:1068F0007C8D8A819923F9F08A3058F495E1899F3B
:10690000F0011124EE57FE4E05811681169507956C
:1069100002C00EEE12E041E00E94694F61E070E0BB
:1069200080E090E00E94EE468A810E94B24F0817F4
:106930001907A0F31EC08A3058F495E1899FF00131
:106940001124EE57FE4E038114811695079502C05F
:106950000AEC18E040E00E94694F61E070E080E0DE
:1069600090E00E94EE468A810E94B24F8017910704
:10697000A0F38A810E943B4FB8018A81DF91CF91B9
:106980001F910F91FF90EF90DF900C94C24FCF9327
:10699000DF93EC018A81893010F40E94224F48EE87
:1069A00053E05B874A8720ED37E03D872C878CEDED
:1069B00095E09F878E87598B488B3B8B2A8B9D8BCD
:1069C0008C8BDF91CF910895CF93DF93EC017F8B78
:1069D0006E8B888599856817790769F48A810E948A
:1069E0003B4F8B8D882321F18A810E94B24F9A8F71
:1069F000898F1B8E1DC0CE0128D6EA81EA30B0F403
:106A00009C01C39714F022E330E02E3C8FEF38074F
:106A100014F42EEC3FEF8FB7F89495E1E99FF00165
:106A20001124EE57FE4E318720878FBF81E08B8F78
:106A3000DF91CF910895CF93DF93EC0189A19AA1C3
:106A4000892B11F01AA219A29B0177FF03C031957F
:106A500021953109B901CE01F8D590932D0180938C
:106A60002C019F8B8E8B0E9426476D8F7E8F8F8F80
:106A700098A3DF91CF9108950F931F93CF93DF9346
:106A80008C01FC01778B668BE0D5EC01F8018281EB
:106A9000938188309105D1F4D7FF06C060E08AE089
:106AA0000E94784561E005C061E08AE00E94784577
:106AB00060E086E00E947845D7FF03C0D195C1957C
:106AC000D109D0932B01C0932A011BC00997C9F4A7
:106AD000D7FF06C060E08DE00E94784561E005C008
:106AE00061E08DE00E94784560E08BE00E9478458F
:106AF000D7FF03C0D195C195D109D0932901C09387
:106B00002801DF91CF911F910F910895CF93DF93CB
:106B1000EC018A81893010F40E94224F2EEC3FEF65
:106B20003B872A8782E390E09D878C871F861E869D
:106B3000398B288B9B8B8A8B1D8A1C8A6EEE72E0A8
:106B40008A810E94AE4F6AEC78E08A810E94AA4F47
:106B50008CED95E09A8F898F1B8EDF91CF910895F0
:106B6000CF93DF93EC0189A19AA1892B11F01AA28E
:106B700019A2CE010E94EF8610922D0110922C01D5
:106B80001F8A1E8A0E9426476D8F7E8F8F8F98A343
:106B9000DF91CF9108950F931F93CF93DF93FC0163
:106BA00021A132A1232B89F1EC010E9426470D8DF2
:106BB0001E8D2F8D38A1DC01CB01801B910BA20B08
:106BC000B30B4097A105B10500F189A19AA10197E6
:106BD000E1F46E897F89615071097F8B6E8BCE01E4
:106BE000161617062CF0DF91CF911F910F91B8CF99
:106BF0002CD590932D0180932C019F8B8E8B0E941E
:106C000026476D8F7E8F8F8F98A3DF91CF911F9135
:106C10000F910895CF93DF93EC011B861A868FEFB7
:106C200090E09D878C871F861E86198A188A9B8B09
:106C30008A8B1D8A1C8A61E08CE20E94A7458A81AA
:106C40009B81089721F410922D0110922C011AA219
:106C500019A2DF91CF910895CF93DF93EC0121E04A
:106C60003FEF3B872A878FEF90E09D878C871F86B9
:106C70001E86398B288B9B8B8A8B1D8A1C8A61E030
:106C80008AE00E94A74561E086E00E94A74561E096
:106C90008DE20E94A74561E08DE00E94A74561E07A
:106CA0008BE00E94A74561E08EE20E94A7458A81A1
:106CB0009B818830910529F410922B0110922A01B2
:106CC00006C0099721F41092290110922801DF9142
:106CD000CF9108950F931F93CF93DF93EC011F8AF9
:106CE0001E8A8C01075E1F4F40E068E0C8010E94C9
:106CF000256A40E06CE0C8010E94256A0E94264790
:106D00006C8F7D8F8E8F9F8FDF91CF911F910F9111
:106D10000895CF93DF93EC017F8B6E8B96D4AC01FB
:106D20008A819B818830910541F4CE01499657FFB5
:106D300002C06AE009C068E00DC00997D1F4CE0135
:106D4000499657FF06C06EE042382FEF520744F0D5
:106D500001C06CE04F3751052CF04EE750E002C007
:106D600042E85FEF57FF03C05195419551090E94DA
:106D7000256A0E9426476C8F7D8F8E8F9F8FDF91B3
:106D8000CF9108950F931F93CF93DF93EC010E944F
:106D900026470C8D1D8D2E8D3F8DDC01CB01801B78
:106DA000910BA20BB30B853F9140A105B10540F0BB
:106DB0006E897F89CE01DF91CF911F910F91A9CF6D
:106DC000DF91CF911F910F910895CF93DF93EC0145
:106DD0008091DD0C811109C06A8D7B8DCE014996B1
:106DE0000E94447F81E08093DD0C21E83FEF3B87E8
:106DF0002A878FE790E09D878C871F861E86398BB8
:106E0000288B9B8B8A8B1D8A1C8ADF91CF910895DA
:106E10000F931F93CF93DF93EC011F8A1E8A8C017F
:106E2000075E1F4F40E060E0C8010E94505140E003
:106E300064E0C8010E9450510E9426476C8F7D8FEC
:106E40008E8F9F8FDF91CF911F910F910895CF93D8
:106E5000DF93EC017F8B6E8BF8D39C018A819B8141
:106E600088309105C1F437FF06C061E021388FEF0B
:106E700038074CF001C060E0A901203831052CF042
:106E80004FE750E002C041E85FEF57FF1FC0519548
:106E9000419551091BC00997E9F4922F832F20389F
:106EA000310514F09FE780E0492F582F41388FEFCC
:106EB000580714F441E85FEF57FF03C0519541951F
:106EC0005109632F661F6627661F6C5FCE014996C6
:106ED0000E9450510E9426476C8F7D8F8E8F9F8F0E
:106EE000DF91CF9108950F931F93CF93DF93EC0120
:106EF0000E9426470C8D1D8D2E8D3F8DDC01CB0110
:106F0000801B910BA20BB30B853F9140A105B105EE
:106F100040F06E897F89CE01DF91CF911F910F9153
:106F200096CFDF91CF911F910F9108956F927F922D
:106F30008F929F92AF92BF92CF92DF92EF92FF9289
:106F40000F931F93CF93DF9380910B0E90910C0EB4
:106F5000DC01ED91FC910480F581E02D1995B12CB7
:106F6000181619060CF0D5C0AA24A39480910B0E14
:106F700090910C0EDC01ED91FC910480F581E02DE7
:106F80001995892B09F4C5C0C091370D81E08C0F8C
:106F90008093370D80910B0E90910C0EDC01ED91DA
:106FA000FC910680F781E02D1995EC2FF0E0E95077
:106FB000F34F80838A30D1F6E090370DF12C109298
:106FC000D80C1092D70C1092D30C1092D40C1092B3
:106FD000D50C1092D60C1092D20C1092D10C1092AB
:106FE000D00C87EFC82E8CE0D82E00E010E0D0E067
:106FF000C0E00E151F050CF06FC0F60191916F01F6
:107000009D3009F466C09C37A1F19A3009F055C053
:10701000CC2359F16C2E712CC30101970E947D87FE
:107020007093D80C6093D70C0E94264760930E0E85
:1070300070930F0E8093100E9093110E8091DB0CC5
:10704000882309F462C08090D70C9090D80CB801C6
:107050006619770987EF9CE00E94676B881699068E
:1070600009F453C01092F60C52C01092F60CD0E006
:1070700030C08C2F90E0FC01E957FD4E1082D130DA
:1070800099F068F0D230B1F40E947D876093D30C00
:107090007093D40C8093D50C9093D60C0BC00E94A7
:1070A0007D876093D00C06C00E947D877093D20CC0
:1070B0006093D10CDF5FC0E00CC00F3311053CF4CE
:1070C000EC2FF0E0E957FD4E9083CF5F02C01092A5
:1070D000F60C0F5F1F4F8DCF8091F60C81110EC003
:1070E0008091CD0C9091CE0C01969093CE0C809314
:1070F000CD0C60E087E80E940D6C02C0BB24B39405
:107100001092F70C1092370D31CFA092F60CD1E00F
:10711000E0CF8B2DDF91CF911F910F91FF90EF90DA
:10712000DF90CF90BF90AF909F908F907F906F90A7
:107130000895CF931092CF0C1092CC0C1092CE0CDD
:107140001092CD0C61E089E30E9478450E940A6BA1
:1071500080910B0E90910C0EDC01ED91FC9104805E
:10716000F581E02D1995892B61F080910B0E90919E
:107170000C0EDC01ED91FC910680F781E02D199554
:10718000E7CF0E94886C80910B0E90910C0EDC0171
:10719000ED91FC910284F385E02D199510920D0E6E
:1071A0000E94264760930E0E70930F0E8093100E70
:1071B0009093110EC1E0BADE81110E947A2D0E94D7
:1071C0004A6B0E948A528091CD0C9091CE0C0A9706
:1071D00024F480910D0E882331F060E08AE80E944B
:1071E0000D6CC093CF0C8091CF0C882321F380913C
:1071F000CC0C882341F049EC51E060E070E088E974
:107200009EE00E94D2AC60E089E30E94784560E095
:107210008AE3CF910C947845EF92FF920F931F93DE
:10722000CF93DF9300D000D0CDB7DEB76FE975E024
:10723000CE0101960E94C1410D811E81F02EEE24E7
:10724000E39480910B0E90910C0EDC01ED91FC917A
:107250000480F581E02D1995892B21F180910B0E89
:1072600090910C0EDC01ED91FC910680F781E02DF0
:1072700019958F3439F4E092F50C8093EA0CE09282
:10728000E90CDFCF9091F50C9923D9F2E091E90C4C
:1072900091E09E0F9093E90CF0E0E651F34F80836C
:1072A0009F1578F28091E90C8F1510F4F12C21C014
:1072B0004BE050E06EED7CE0CE0101960E9407822B
:1072C000AAEEBCE0EFE9F5E0FF24F3941127CF012B
:1072D0008F5995408017910734F49D9181919817AB
:1072E000B1F3F12CF4CF1092EA0C1092F50C10923D
:1072F000E90CCE0101960E9491418F2D26960FB682
:10730000F894DEBF0FBECDBFDF91CF911F910F91DB
:10731000FF90EF900895DC01ED91FC910190F081D8
:10732000E02D19940F931F93CF93DF93EC0180917D
:10733000DC0C811111C00A8D1B8D6AEA70E0C80156
:10734000EADFD801ED91FC910284F385E02DC801BC
:10735000199581E08093DC0C4AE06EE0CE014996FD
:107360000E94505121E83FEF3B872A878FE790E04A
:107370009D878C871F861E86398B288B9B8B8A8BDB
:107380001D8A1C8ADF91CF911F910F910895CF9391
:10739000DF93EC017F8B6E8B58D1BC018A81DF912A
:1073A000CF910C94C24F08950895089508951092B6
:1073B0005C0A08950F931F93CF93DF93EC011F8A0C
:1073C0001E8A8C01075E1F4F40E060E0C8010E94EA
:1073D000135140E064E0C8010E9413510E94264707
:1073E0006C8F7D8F8E8F9F8FDF91CF911F910F912B
:1073F00008950F931F93CF93DF93EC01E8A1F9A1B8
:1074000080819181A281B3818E01075E1F4F81151A
:107410009649A105B10509F451C040E056E960E084
:1074200070E086E597E00E94FD8664E170E080E010
:1074300090E00E94EE46E8A1F9A180819181A281AD
:10744000B38181152BE49207A105B105E9F068F439
:10745000803629E09207A105B105A1F08038954258
:10746000A105B105C1F442E012C0811521EE9207D9
:10747000A105B10559F08115924CA140B10559F40F
:1074800045E005C041E003C043E001C046E06FE0D5
:10749000C8010E94135186E597E0C7D5E8A1F9A17C
:1074A000408151816281738186E597E00E94FD866B
:1074B00064E170E080E090E00E94EE464AE06EE019
:1074C000C8010E94135141E067E1C8010E941351B5
:1074D0004AA168E1C8010E94135121E83FEF3B87B0
:1074E0002A878FE790E09D878C871F861E86398BC1
:1074F000288B9B8B8A8B1D8A1C8ADF91CF911F91D1
:107500000F91089544CFCF93DF93CEEED9E081E081
:1075100090E09A83898310925C0A0E94C9466C832A
:107520007D838E839F83E49AEC9ADF91CF910895B7
:10753000EF92FF920F931F93CF93DF93EC0166239B
:10754000E1F0262F653608F024E60A891B89E888D1
:10755000F988D801AE19BF0930E00E94ADA728EC28
:1075600030E040E050E00E942EADE20EF31EFB86BC
:10757000EA86021B130B1D870C87DF91CF911F91A9
:107580000F91FF90EF900895CF93DF93CDB7DEB7C3
:10759000A2970FB6F894DEBF0FBECDBF80310CF0BE
:1075A00080E12DEB3EE03A83298325EB3EE03C83EE
:1075B0002B832DEA3EE03E832D8325EA3EE038878B
:1075C0002F832DE93EE03A87298725E93EE03C8775
:1075D0002B872DE83EE03E872D8725E83EE0388B5F
:1075E0002F8727E73EE03A8B298B25E63EE03C8B50
:1075F0002B8B28E43EE03E8B2D8B23E33EE0388F3F
:107600002F8B29E23EE03A8F298F2FE13EE03C8F1D
:107610002B8F22E13EE03E8F2D8F26E03EE038A307
:107620002F8F2EEF3DE03AA329A3E82FEE0FFF0B9B
:10763000EC0FFD1F81819281A2960FB6F894DEBFF8
:107640000FBECDBFDF91CF9108958F929F92AF92E1
:10765000BF92CF92DF92EF92FF920F931F93DC01C4
:1076600018968D919C9119971E96CD90DC901F973E
:107670006817790709F456C05896FC9058974C0142
:10768000092E000CAA08BB088B01072E000C220B48
:10769000330B861797073CF41696ED91FC911797DC
:1076A000FF2039F015C01496ED91FC911597FF203D
:1076B00079F00D2C000CEE08FF08A901980128199B
:1076C00039094A095B091C966D917C911D970EC082
:1076D0000D2C000CEE08FF08A901980128193909A2
:1076E0004A095B091A966D917C911B97CB01770F24
:1076F000AA0BBB0BBC01CD016C197D098E099F093A
:107700000E9469A78F01FF0F220B330BA90198017B
:10771000281939094A095B090E9402ADC20ED31E1D
:10772000E41EF51EC6011F910F91FF90EF90DF90B0
:10773000CF90BF90AF909F908F900895CF93DF939D
:10774000EC017F8B6E8B81DF9C018A819B8188306D
:107750009105C1F437FF06C061E021388FEF38078B
:107760004CF001C060E0A901203831052CF04FE752
:1077700050E002C041E85FEF57FF1FC051954195AF
:1077800051091BC00997E9F4922F832F2038310546
:1077900014F09FE780E0492F582F41388FEF5807AA
:1077A00014F441E85FEF57FF03C05195419551092B
:1077B000632F661F6627661F6C5FCE0149960E9485
:1077C00013510E9426476C8F7D8F8E8F9F8FDF9184
:1077D000CF9108950F931F93CF93DF93EC010E94F5
:1077E00026470C8D1D8D2E8D3F8DDC01CB01801B1E
:1077F000910BA20BB30B853F9140A105B10540F061
:107800006E897F89CE01DF91CF911F910F9196CF25
:10781000DF91CF911F910F910895CF93DF93EC01EA
:1078200061E089E00E94A74560E089E00E94784518
:1078300010929A0987EF94E099838883DF91CF9122
:107840000895CF92DF92EF92FF9280919B0983304F
:1078500009F061C080919C098130D1F488EE93E0F9
:10786000A0E0B0E080932D0990932E09A0932F09FA
:10787000B093300980E797E1A0E0B0E08093310950
:1078800090933209A0933309B093340932E001C0D8
:1078900030E0E0919C09F0E0E356F64F2081A0E152
:1078A000A30F48EE53E060E070E088EBC82E8BE059
:1078B000D82EE12CF12C832F90E0FC01EE0FFF1F5E
:1078C000EE0FFF1FE35DF64F27FF10C0C082D1828D
:1078D000E282F382880F991F880F991FFC01EF5CE9
:1078E000F64F40835183628373830FC0408351837B
:1078F00062837383880F991F880F991FFC01EF5CC7
:10790000F64FC082D182E282F3823E5F220F3A13A9
:10791000D2CF30939609FF90EF90DF90CF900895EB
:10792000CF93DF9380919A09811153C010929809E7
:1079300010929509C1E0C0939A09D091990961E02C
:1079400089E00E94A74560E089E00E9478452D2FDC
:1079500030E040E050E060E47FE180E090E00E94B1
:1079600002ADC093B00089E08093B1002093B300D2
:107970008BEA289F212D112426952093B400809115
:107980006F008B7F80936F008091B0008062809346
:10799000B0002091840030918500E091950981E04C
:1079A0008E0F8093950984E0E89FF0011124E35D38
:1079B000F64F80819181A281B381820F931F9093B2
:1079C0008B0080938A00B29A80916F0084608093CC
:1079D0006F00DF91CF9108954F925F926F927F92E7
:1079E0008F929F92AF92BF92CF92DF92EF92FF92CF
:1079F0008AE1809396092093970988E280939909F8
:107A000081E080939C0980939D098EE080939B097F
:107A100080EC92E1A0E0B0E080932D0990932E09D4
:107A2000A0932F09B093300980EB94E0A0E0B0E080
:107A30008093310990933209A0933309B0933409AC
:107A4000A4E1440F551F661F771FAA95D1F722E0C6
:107A500030E0B0EBCB2EB4E0DB2EE12CF12C80E655
:107A6000482E89E0582E612C712C90E4892E9CE9D7
:107A7000992EA12CB12CC901880F991F880F991F2D
:107A8000FC01E35DF64F77FF05C0408251826282C0
:107A9000738204C0C082D182E282F382C90101965E
:107AA000880F991F880F991FFC01E35DF64F28315D
:107AB00029F0C082D182E282F38204C08082918266
:107AC000A282B382440F551F661F771F2E5F3F4F60
:107AD0002A31310581F6FF90EF90DF90CF90BF9073
:107AE000AF909F908F907F906F905F904F9018CF46
:107AF0008F929F92AF92BF92CF92DF92EF92FF92BE
:107B000082E18093960986E08093970996E29093AC
:107B1000990991E090939C0990939D0980939B090A
:107B200088ED90E4A0E0B0E080932D0990932E09B9
:107B3000A0932F09B09330098CE19CE0A0E0B0E065
:107B40008093310990933209A0933309B09334099B
:107B5000742F66275527442722E030E0ACE1CA2E77
:107B6000ACE0DA2EE12CF12CB8E38B2EB8E19B2EA1
:107B7000A12CB12CC901880F991F880F991FFC01F6
:107B8000E35DF64F77FF05C080829182A282B382C7
:107B900004C0C082D182E282F382F901EE0FFF1F9E
:107BA000EE0FFF1FEF5CF64FC082D182E282F382BC
:107BB000440F551F661F771F2E5F3F4F223131053F
:107BC000C9F68CE199E8A0E0B0E080937109909348
:107BD0007209A0937309B0937409FF90EF90DF903E
:107BE000CF90BF90AF909F908F909ACE1F920F92A0
:107BF0000FB60F9211240BB60F922F933F934F9312
:107C00005F936F937F938F939F93AF93BF93EF9304
:107C1000FF939091950980919609981316C0109240
:107C2000950980919C098F5F80939C0990919C0994
:107C300080919D09891740F481E080939C0980918F
:107C400098098F5F80939809FCDD90919809809145
:107C5000970998130DC08091B0008F7D8093B0007C
:107C600080916F008B7F80936F0010929A0927C0DC
:107C70008091B00085FF04C08091B0008F7D03C06B
:107C80008091B00080628093B00020918400309198
:107C90008500E091950981E08E0F8093950984E03D
:107CA000E89FF0011124E35DF64F80819181A2816C
:107CB000B381820F931F90938B0080938A00FF9172
:107CC000EF91BF91AF919F918F917F916F915F9154
:107CD0004F913F912F910F900BBE0F900FBE0F90C1
:107CE0001F9018951F920F920FB60F9211240BB68A
:107CF0000F921F932F933F934F935F936F937F93B5
:107D00008F939F93AF93BF93EF93FF93CF93DF93A3
:107D100000D01F92CDB7DEB78091EE09C1D611E039
:107D2000892B09F010E00E94C94669837A838B830E
:107D30009C8389819A81AB81BC814091F2095091E9
:107D4000F3096091F4097091F509841B950BA60B5A
:107D5000B70B2091EF093091F0092430310509F477
:107D60004CC02530310521F021303105E9F414C033
:107D70002091F109222339F020915C0A20FF02C0F2
:107D8000289A01C02898112379F0813E2EE29207AB
:107D9000A105B10548F02BC0112379F125E030E0B1
:107DA0003093F0092093EF092091EF093091F00909
:107DB0002530310511F5E0915C0AF0E0EE0FFF1F70
:107DC000EA50F64F9183808389819A81AB81BC818F
:107DD0008093F2099093F309A093F409B093F50905
:107DE00080915C0A8F5F80935C0A833330F084E07B
:107DF00090E09093F0098093EF090F900F900F900F
:107E00000F90DF91CF91FF91EF91BF91AF919F9133
:107E10008F917F916F915F914F913F912F911F9122
:107E20000F900BBE0F900FBE0F901F9018950895E6
:107E3000CF92DF92EF92FF920F931F93CF93DF9336
:107E40006C017A018B01C0E0D0E0CE15DF0589F02E
:107E5000D8016D918D01D601ED91FC910190F081D9
:107E6000E02DC6011995892B11F47E0102C02196DF
:107E7000ECCFC701DF91CF911F910F91FF90EF9051
:107E8000DF90CF900895FC01A089B1898C91A689DB
:107E9000B78982FD0FC09C91818D8F5F8F73228D7A
:107EA000821749F0218DDF01A20FB11D5D969C93D1
:107EB000818F08958C910895FC01918D828D981782
:107EC00061F0828DDF01A80FB11D5D968C91928DBE
:107ED0009F5F9F73928F90E008958FEF9FEF0895BB
:107EE000FC01918D828D981731F0828DE80FF11D84
:107EF000858D90E008958FEF9FEF0895FC01918D9F
:107F0000228D892F90E0805C9F4F821B91098F7397
:107F10009927089589EB96E0F1DF21E0892B09F498
:107F200020E0822F089586E597E0E8DF21E0892BA5
:107F300009F420E0822F089583EF97E0DFDF21E04E
:107F4000892B09F420E0822F089580E998E0D6DF9C
:107F500021E0892B09F420E0822F0895FC01848D13
:107F6000DF01A80FB11DA35ABF4F2C91848D90E063
:107F700001968F739927848FA689B7892C93A0893E
:107F8000B1898C9180648C93938D848D981306C0F5
:107F90000288F389E02D80818F7D80830895EF92A0
:107FA000FF920F931F93CF93DF93EC0181E0888FB3
:107FB0009B8D8C8D981305C0E889F989808185FD9A
:107FC00023C0F62E0B8D10E00F5F1F4F0F7311278C
:107FD000E02E8C8DE8120BC00FB607FCFACFE889B3
:107FE000F989808185FFF5CFCE01B8DFF2CF8B8D87
:107FF000FE01E80FF11DE35AFF4FF0820B8FEA8973
:10800000FB898081806207C0EE89FF896083E889EF
:10801000F98980818064808381E090E0DF91CF9155
:108020001F910F91FF90EF900895CF93DF93EC0194
:10803000888D8823C1F0EA89FB89808185FD05C090
:10804000A889B9898C9186FD0EC00FB607FCF5CFC3
:10805000808185FFF2CFA889B9898C9185FFEDCF0A
:10806000CE017CDFE8CFDF91CF91089580E090E0F2
:10807000892B19F06ADF811116C080E090E0892B0E
:1080800019F05ADF811112C080E090E0892B19F0BD
:108090004ADF81110EC080E090E0892B79F03ADF51
:1080A00081110AC008950E940000E7CF0E940000DD
:1080B000EBCF0E940000EFCF0C940000089590E0F9
:1080C000FC013197E231F10508F04EC08827E85DE8
:1080D000FE4F8F4F0C949FA7809180008F7703C035
:1080E000809180008F7D8093800008958091800032
:1080F000877FF9CF84B58F7702C084B58F7D84BD2B
:1081000008958091B0008F7703C08091B0008F7D7B
:108110008093B0000895809190008F7707C0809180
:1081200090008F7D03C080919000877F80939000A6
:1081300008958091A0008F7707C08091A0008F7D67
:1081400003C08091A000877F8093A0000895809154
:1081500020018F7707C0809120018F7D03C080911F
:108160002001877F8093200108950E94CAAA0F935F
:108170001F93CF93DF938C01EB01FC0180819181F0
:108180000097B1F0688179816115710579F04281BC
:1081900053812C813D814217530740F00E94E2AA8F
:1081A0008C819D81F8019583848313C00E944EA920
:1081B00088819981F801918380838A819B8193834F
:1081C00082838C819D8195838483198218821B828E
:1081D0001A821D821C82DF91CF911F910F91089509
:1081E0000F931F93CF93DF93EC01888199810097C0
:1081F00029F02A813B812617370788F48B016F5FAE
:108200007F4F0E94E6A9009761F0998388831B83C2
:108210000A832C813D81232B11F4FC01108281E023
:1082200001C080E0DF91CF911F910F910895EF92EF
:10823000FF920F931F93CF93DF93FB01248135812E
:10824000E080F180FC0104811581E114F10411F456
:1082500080E016C02115310591F0EC01020F131FCB
:10826000B801BEDF8823A1F3288139818C819D81EB
:10827000B701820F931F0E94E2AA1D830C8381E045
:10828000DF91CF911F910F91FF90EF900895EF92A2
:10829000FF920F931F93CF93DF93EC017B018A0131
:1082A000BA019EDF2881398181110DC02115310568
:1082B00019F0C9010E944EA9198218821D821C82E0
:1082C0001B821A8206C01D830C83B701C9010E945C
:1082D000E2AACE01DF91CF911F910F91FF90EF9015
:1082E0000895CF93DF93EC016115710551F0FB0107
:1082F00001900020E9F73197AF01461B570BC7DF0C
:108300000CC088819981009711F00E944EA91982B2
:1083100018821D821C821B821A82CE01DF91CF91AE
:108320000895FC01808191810C944EA90F931F93B5
:10833000CF93DF93CDB7DEB762970FB6F894DEBF69
:108340000FBECDBF8C01CB01F801118210821382C8
:1083500012821582148250E0BE016F5F7F4F0E942F
:108360004DABBE016F5F7F4FC801BBDF62960FB69A
:10837000F894DEBF0FBECDBFDF91CF911F910F915B
:108380000895FC01118210821382128215821482D8
:108390006115710549F0FB0101900020E9F7319763
:1083A000AF01461B570B73CF0895CF93DF9300D0D7
:1083B0001F92CDB7DEB7611571058105910579F082
:1083C0009B01AC0169833A834B835C830E9441AB80
:1083D00029813A814B815C810E9402AD03C060E03B
:1083E00070E0CB010F900F900F900F90DF91CF9125
:1083F0000895DC01ED91FC910190F081E02D19943C
:10840000EF92FF920F931F93CF93DF938C017B0129
:10841000C0E0D0E0F701EC0FFD1F6491662361F02E
:10842000D801ED91FC910190F081E02DC8011995E2
:10843000892B11F02196EECFCE01DF91CF911F91C4
:108440000F91FF90EF9008956115710579F0FB0190
:1084500001900020E9F73197AF01461B570BDC0173
:10846000ED91FC910280F381E02D199480E090E081
:1084700008954F925F926F927F92EF92FF920F93C7
:108480001F93CF93DF93CDB7DEB7A1970FB6F894C4
:10849000DEBF0FBECDBF7C01FA01CB0119A2223095
:1084A00008F42AE08E010F5D1F4F422E512C612CE3
:1084B000712CBF01A30192010E942EADF901CA01E6
:1084C000015011096A3014F4605D01C0695CD80183
:1084D0006C93232B242B252B61F7B801C701B4DF44
:1084E000A1960FB6F894DEBF0FBECDBFDF91CF913E
:1084F0001F910F91FF90EF907F906F905F904F9042
:1085000008954F925F926F927F928F929F92AF9257
:10851000BF92CF92DF92EF92FF92CF93DF93EC0165
:108520006A017B01B22E9A01AB01C701B6010E941C
:10853000B5A8882319F063EA75E027C02601370142
:10854000E89477F82FEF3FEF4FE75FE7C301B20101
:108550000E94B5A881110DC02FEF3FEF4FE75FE7F5
:10856000C301B2010E94B9AB18161CF467EA75E0AA
:108570000CC02FEF3FEF4FE75FE4C701B6010E9449
:10858000B1A8181694F46BEA75E0CE01DF91CF9193
:10859000FF90EF90DF90CF90BF90AF909F908F9023
:1085A0007F906F905F904F904FCF2FEF3FEF4FE74F
:1085B0005FECC701B6010E94B9AB87FDE4CF20E0B4
:1085C00030E0A901C701B6010E94B9AB87FF09C01D
:1085D0006DE2CE010EDF4C01F7FAF094F7F8F0945B
:1085E00002C0812C912CA12C60E070E080E09FE320
:1085F000AB1441F020E030E040E251E40E9418A8C2
:10860000A394F6CF9B01AC01C701B6010E94B4A7A9
:108610002B013C010E9485A86B017C010E94BDAB2F
:108620009B01AC01C301B2010E94B3A72B013C0125
:108630002AE0B701A601CE011CDF7C01E80CF91C81
:10864000BB2029F06EE2CE01D4DEE80EF91EDB2C51
:10865000DD2021F120E030E040E251E4C301B2012D
:108660000E941EAC2B013C010E9485A84B01A12C4D
:10867000B12C2AE0B501A401CE01FBDEE80EF91E03
:10868000C501B4010E94BDAB9B01AC01C301B201A5
:108690000E94B3A72B013C01DA94DACFC701DF9126
:1086A000CF91FF90EF90DF90CF90BF90AF909F90D1
:1086B0008F907F906F905F904F9008956FEA75E074
:1086C000C3CE0F931F93CF93DF93EC01BDDE8C01DC
:1086D000CE01F4DF800F911FDF91CF911F910F9199
:1086E00008950F931F93CF93DF93EC0189DE8C01E4
:1086F000CE01E4DF800F911FDF91CF911F910F9189
:1087000008951F920F920FB60F9211240BB60F927D
:108710002F933F934F935F936F937F938F939F9389
:10872000AF93BF93EF93FF9389EB96E017DCFF9134
:10873000EF91BF91AF919F918F917F916F915F91D9
:108740004F913F912F910F900BBE0F900FBE0F9046
:108750001F9018951F920F920FB60F9211240BB60F
:108760000F922F933F934F935F936F937F938F93CA
:108770009F93AF93BF93EF93FF9389EB96E083DBD7
:10878000FF91EF91BF91AF919F918F917F916F91E9
:108790005F914F913F912F910F900BBE0F900FBEA5
:1087A0000F901F9018951F920F920FB60F921124E1
:1087B0000BB60F922F933F934F935F936F937F93DB
:1087C0008F939F93AF93BF93EF93FF9386E597E0CB
:1087D000C5DBFF91EF91BF91AF919F918F917F91F9
:1087E0006F915F914F913F912F910F900BBE0F9022
:1087F0000FBE0F901F9018951F920F920FB60F92F9
:1088000011240BB60F922F933F934F935F936F9367
:108810007F938F939F93AF93BF93EF93FF9386E5DF
:1088200097E031DBFF91EF91BF91AF919F918F91D5
:108830007F916F915F914F913F912F910F900BBE60
:108840000F900FBE0F901F9018951F920F920FB6AA
:108850000F9211240BB60F922F933F934F935F9378
:108860006F937F938F939F93AF93BF93EF93FF93F8
:1088700083EF97E073DBFF91EF91BF91AF919F91F1
:108880008F917F916F915F914F913F912F910F90B9
:108890000BBE0F900FBE0F901F9018951F920F9256
:1088A0000FB60F9211240BB60F922F933F934F9355
:1088B0005F936F937F938F939F93AF93BF93EF9348
:1088C000FF9383EF97E0DFDAFF91EF91BF91AF91D4
:1088D0009F918F917F916F915F914F913F912F91D8
:1088E0000F900BBE0F900FBE0F901F9018951F9208
:1088F0000F920FB60F9211240BB60F922F933F9346
:108900004F935F936F937F938F939F93AF93BF9397
:10891000EF93FF9380E998E021DBFF91EF91BF9106
:10892000AF919F918F917F916F915F914F913F9107
:108930002F910F900BBE0F900FBE0F901F901895A8
:108940001F920F920FB60F9211240BB60F922F9316
:108950003F934F935F936F937F938F939F93AF93C7
:10896000BF93EF93FF9380E998E08DDAFF91EF9149
:10897000BF91AF919F918F917F916F915F914F9137
:108980003F912F910F900BBE0F900FBE0F901F9035
:108990001895CF93DF93EC01E881F9810284F38588
:1089A000E02D1995EA89FB8980818F7E8083EA8991
:1089B000FB898081877F8083EA89FB8980818F772B
:1089C0008083EA89FB8980818F7D80838A8D898F6E
:1089D000DF91CF910895CF92DF92EF92FF921F9394
:1089E000CF93DF93EC016A017B01122FE889F989AB
:1089F00082E080834115514E61057105B1F060E060
:108A000079E08DE390E0A70196010E942EADDA0196
:108A1000C9010197A109B109B695A79597958795C1
:108A2000AC01411580E15807A8F0E889F989108266
:108A300060E874E88EE190E0A70196010E942EADF7
:108A4000BA01A901415051096109710976956795EB
:108A500057954795EC85FD855083EE85FF854083CE
:108A6000188EEC89FD891083EA89FB8980818061F9
:108A70008083EA89FB89808188608083EA89FB8919
:108A8000808180688083EA89FB8980818F7D8083F3
:108A9000DF91CF911F91FF90EF90DF90CF900895DD
:108AA000CF93DF93282F30E0F901E156F04F849106
:108AB000F901E75AF04FD491F901ED5EF04FC491FE
:108AC000CC2389F08111FBDAEC2FF0E0EE0FFF1FD1
:108AD000E750F14FA591B491EC91ED2381E090E046
:108AE00021F480E002C080E090E0DF91CF91089512
:108AF0001F93CF93DF93282F30E0F901E156F04F19
:108B00008491F901E75AF04FD491F901ED5EF04FED
:108B1000C491CC23C1F0162F8111D1DAEC2FF0E0F3
:108B2000EE0FFF1FE152F14FA591B4918FB7F8946A
:108B3000111105C09C91ED2FE095E92302C0EC9145
:108B4000ED2BEC938FBFDF91CF911F910895CF93C1
:108B5000DF9390E0FC01E75AF04F2491FC01ED5EB9
:108B6000F04F8491882361F190E0880F991FFC01F8
:108B7000EB53F14FC591D491FC01E152F14FA59116
:108B8000B491611109C09FB7F89488812095822320
:108B90008883EC912E230BC0623061F49FB7F89468
:108BA0003881822F809583238883EC912E2B2C9300
:108BB0009FBF06C08FB7F894E8812E2B28838FBF04
:108BC000DF91CF9108951F93CF93DF93182FEB017F
:108BD00061E0BDDF209711F460E004C0CF3FD10514
:108BE00031F461E0812FDF91CF911F9181CFE12F8F
:108BF000F0E0E156F04FE4914E2F50E0FA0131974A
:108C0000E231F10508F09DC08827E65CFE4F8F4FEA
:108C10000C949FA784B5806884BDC7BD97C084B5F8
:108C2000806284BDC8BD92C08091800080688093BE
:108C30008000D0938900C093880088C08091800014
:108C4000806280938000D0938B00C0938A007EC0A6
:108C500080918000886080938000D0938D00C093C5
:108C60008C0074C08091B00080688093B000C09385
:108C7000B3006CC08091B00080628093B000C0935C
:108C8000B40064C080919000806880939000D0937D
:108C90009900C09398005AC08091900080628093A0
:108CA0009000D0939B00C0939A0050C08091900098
:108CB000886080939000D0939D00C0939C0046C034
:108CC0008091A00080688093A0008091A0008F7B9D
:108CD0008093A000D093A900C093A80037C08091D2
:108CE000A00080628093A000D093AB00C093AA0044
:108CF0002DC08091A00088608093A000D093AD002B
:108D0000C093AC0023C08091200180688093200133
:108D1000D0932901C093280119C08091200180625D
:108D200080932001D0932B01C0932A010FC0809122
:108D30002001886080932001D0932D01C0932C01E5
:108D400005C0C038D1050CF04CCF46CFDF91CF9194
:108D50001F910895863308F0865390917B00282F49
:108D60002870977F922B90937B008770806480930C
:108D70007C0080917A00806480937A0080917A00F0
:108D800086FDFCCF809178002091790090E0922BB5
:108D900008953FB7F89480913C0D90913D0DA091BE
:108DA0003E0DB0913F0D26B5A89B05C02F3F19F091
:108DB0000196A11DB11D3FBFBA2FA92F982F88275B
:108DC000820F911DA11DB11DBC01CD0142E0660FB6
:108DD000771F881F991F4A95D1F708958F929F9208
:108DE000AF92BF92CF92DF92EF92FF926B017C0124
:108DF000D0DF4B015C01C114D104E104F104E9F0BE
:108E0000C8DFDC01CB0188199909AA09BB09883E92
:108E10009340A105B10578F321E0C21AD108E10819
:108E2000F10888EE880E83E0981EA11CB11CC114C5
:108E3000D104E104F10421F7DECFFF90EF90DF9041
:108E4000CF90BF90AF909F908F9008952FB7F894D8
:108E50006091380D7091390D80913A0D90913B0DD4
:108E60002FBF08958091470D9091480D9160909388
:108E7000480D8093470D08958091470D9091480DBE
:108E800080689093480D8093470D08958091470D19
:108E90009091480D80619093480D8093470D0895FF
:108EA000FC018281882371F08381882359F0138229
:108EB0008091470D9091480D24E082279093480DB2
:108EC0008093470D0895FC018281882371F083818E
:108ED00081110BC081E083838091470D9091480DF3
:108EE00084609093480D8093470D0895FC01848120
:108EF000882371F08581882359F015828091470D70
:108F00009091480D28E082279093480D8093470D5B
:108F10000895FC018481882371F0858181110BC043
:108F200081E085838091470D9091480D88609093F2
:108F3000480D8093470D08958091470D9091480DFD
:108F400020E282279093480D8093470D08958091E9
:108F5000470D9091480D80629093480D8093470D86
:108F60000895DC01ED91FC910680F781E02D60E031
:108F700070E0199477FF03C07195619571096F3F97
:108F8000710519F014F06FEF70E08091470D90912A
:108F9000480D8C7B91709093480D8093470D809184
:108FA000470D9091480D6F30710514F480641FC017
:108FB0006733710514F481641AC06F3571051CF4B0
:108FC0008164906114C0673871051CF481649063FA
:108FD0000EC06F3A71051CF48164906408C0673D4F
:108FE00071051CF48164906502C081649066909361
:108FF000480D8093470D089580E094E09093480DCC
:109000008093470D08958091470D9091480D92608F
:109010009093480D8093470D8091470D9091480D96
:1090200080649093480D8093470D089508950895A6
:109030000895089508950895089508950895089548
:1090400080E0089508950895089508950895089575
:109050000895089508950895089508950895089528
:1090600080E0089508950895FC0164830895FC014B
:1090700062830895FC01138214821582168217827E
:1090800010860895089508950895FC018381089538
:10909000FC0164830895FC0167830895FC016583E6
:1090A0000895FC018281089588EE94E7A1E0BB2732
:1090B000ABBFFC016791769182E09DD681E0809301
:1090C000680E10926C0E1092690E089581E08093E4
:1090D000890E6CED75E08FC6FC011282138214823A
:1090E000158261E086E133DD61E086E101DDE2E7E2
:1090F000F0E08081816080831092480D1092470DCE
:109100000895FF920F931F93CF93DF938C01C62F87
:10911000F42ED22F6AED70E0DC0119968D919C91AE
:109120001A970E948B39F80181859285DC01ED91B7
:10913000FC910190F081E02D6C2F1995F80181854B
:109140009285DC01ED91FC910190F081E02D6F2D75
:109150001995F80181859285DC01ED91FC910190D2
:10916000F081E02D6D2F1995EC2FF0E0BF016652D4
:109170007F4F6F0D711D6D0F711D6F777727F80190
:1091800081859285DF91CF911F910F91FF900C9473
:109190008B3920E040E0B5CF65E4FBCF68E4F9CF40
:1091A000CF93DF93FC012381222321F0EC0161E4C2
:1091B000F0DF1B82DF91CF910895CF93DF93FC0105
:1091C0002381211105C0EC0160E4E3DF81E08B83A2
:1091D000DF91CF910895FC012481222311F06CE3EB
:1091E000D8CF0895FC012781222331F02085222346
:1091F00019F010866BE3CDCF0895FC01278122235F
:1092000039F02085211104C021E020876AE3C1CF15
:109210000895FC012581222331F02681222319F0B3
:10922000168269E3B6CF0895FC012581222339F027
:109230002681211104C021E0268368E3AACF089586
:1092400067E3A7CF6AE4A5CF69E4A3CF66E3A1CF24
:1092500065E39FCF6EE49DCF64E39BCF63E399CF3B
:1092600062E397CF61E395CF60E393CF6FE291CF55
:109270006DE28FCF6CE28DCF242F462F6CE441CF6F
:1092800077FF03C071956195710920E0462F6EE26A
:1092900038CF462F20E067E434CF462F20E066E445
:1092A00030CF262F64E42DCFCF92DF92FF920F9321
:1092B0001F93CF93DF938C01F62E443F81E0580734
:1092C00038F0413187E2580728F040E157E202C008
:1092D00044EF51E0243F81E0380738F0E9012131C3
:1092E000374228F0C0E1D7E202C0C4EFD1E0CA01A2
:1092F000845F914022E3C22ED12CB6010E9478A750
:10930000462F2F2D62E4C801FCDECE01845F914020
:10931000B6010E9478A7462F2F2D63E4C801DF9184
:10932000CF911F910F91FF90DF90CF90EACE262F23
:1093300040E06FE3E6CE262F40E06EE3E2CE262F3C
:1093400040E06DE3DECE462F20E06DE4DACEFC0196
:109350006283611104C020E040E06BE4D2CE089546
:1093600077FF03C071956195710920E0462F6BE48A
:10937000C8CE4F925F926F927F928F929F92AF92E0
:10938000BF92CF92DF92EF92FF920F931F93CF93F2
:10939000DF936C01A4ECCA1AADEFDA0AD601ED91A5
:1093A000FC917E970CF05CC0FC01E858FF4F812CCB
:1093B000912CA191B191AB2B21F42115310549F4E8
:1093C0004FC0BFEF8B1A9B0AAEE18A16910489F752
:1093D00047C0EC015401AA0CBB1CAA0CBB1CAC0E70
:1093E000BD1EF501EC54FF4F4083518362837383AC
:1093F0007401EE0CFF1CEC0EFD1EF701E858FF4F48
:1094000031832083EC54FF4F11830083BE01680D2C
:10941000791DFB01EC55FE4F81E0808317DDF501DE
:109420006083718382839383C65CDD4F88819981D9
:10943000F701E250FE4F91838083D6012D913C913C
:1094400011972F5F3F4F2D933C939C012F5F3F4F10
:109450001216130614F021E030E03983288302C08D
:109460008FEF9FEFDF91CF911F910F91FF90EF90C2
:10947000DF90CF90BF90AF909F908F907F906F9034
:109480005F904F9008950F931F93CF93DF93EC015C
:109490007093880E6093870E81E090E00E94B9A8D7
:1094A0008C0143D610934A0D0093490D91E090939F
:1094B000890E9093680E1092860E1092850E10926F
:1094C0006B0E10926A0E10926C0E1092690E24EFC1
:1094D00031E03093730E2093720E28EB3BE0309313
:1094E000750E2093740E20E233E030937A0E2093B1
:1094F000790E2CEA3DE030937C0E20937B0E28E021
:1095000037E03093810E2093800E24E931E13093CF
:10951000830E2093820E10926F0E10926E0E109298
:109520006D0E1092760E10927D0E1092840E109297
:10953000710E1092700E1092780E1092770E10929B
:109540007F0E10927E0E988399839A83DF91CF913C
:109550001F910F9108951F920F920FB60F92112431
:109560000BB60F922F933F934F935F936F937F931D
:109570008F939F93AF93BF93EF93FF938091460D8B
:109580008F5F8093460D9091450D891708F4FAC0BE
:109590001092460D8091440D90E08730910508F0BF
:1095A000F1C0FC018827E45BFE4F8F4F0C949FA70E
:1095B00060E086E19DDA88E08093450D81E043C05C
:1095C00061E086E195DA81E08093450D33C060E08B
:1095D00086E18EDA8091420D9091430D97FF05C090
:1095E00083E08093450D84E02EC081E08093450D9B
:1095F00083E029C061E086E17BDA83E08093450D5A
:109600008091410D8F5F8093410D803148F0109221
:10961000410D85E018C061E086E16ADA81E0EECFB5
:109620008091420D9091430D880F991F9093430DA7
:109630008093420D82E007C060E086E159DA81E064
:109640008093450D86E08093440D9CC061E086E1E7
:109650004FDA88E18093450D8091470D9091480D38
:109660009093430D8093420D8091470D9091480D4A
:1096700091FF1DC08091400D8823B1F08091470D6E
:109680009091480D22E092279093480D8093470DCA
:109690008091470D9091480D80649093480D809380
:1096A000470D1092400D03C081E08093400D8091E2
:1096B000470D9091480D92FF0EC08091400D882378
:1096C00039F01092480D1092470D1092400D03C0D2
:1096D00081E08093400D8091470D9091480D84FF6B
:1096E00014C08091400D882369F08091470D9091BE
:1096F000480D20E182279093480D8093470D1092EA
:10970000400D03C081E08093400D8091470D909102
:10971000480D87FF13C08091400D882361F0809130
:10972000470D9091480D80589093480D8093470DB8
:109730001092400D03C081E08093400D8091470D51
:109740009091480D90FF14C08091400D882369F0DE
:109750008091470D9091480D21E092279093480DFC
:109760008093470D1092400D03C081E08093400D1F
:109770008091470D9091480D9093430D8093420D39
:109780001092440DFF91EF91BF91AF919F918F91F6
:109790007F916F915F914F913F912F910F900BBEF1
:1097A0000F900FBE0F901F901895DC01A250BE4F76
:1097B00020E030E04D915D914617570739F4280FAE
:1097C000391FF901EC55FE4F808108952F5F3F4FFF
:1097D0002E31310579F780E00895CF93DF93EC01C6
:1097E000C45CDD4FA881B981109709F442C0FC0127
:1097F000E250FE4F20E030E041915191461757076B
:1098000099F5A901440F551F480F591FFA01E8584F
:10981000FF4F60817181672B61F111821082FC0121
:10982000E20FF31FEC55FE4F1082FA01EE53FE4F8C
:1098300011821082235D3F4F220F331F220F331FEF
:10984000FC01E20FF31F1082118212821382FA01CF
:10985000E859FE4F11821082EA56FF4F11821082A2
:109860001197B983A88305C02F5F3F4F2E31310573
:1098700019F6DF91CF9108950F931F9301E010E047
:1098800078DD1F910F9108950F931F9300E010E072
:1098900070DD1F910F9108952F923F924F925F922A
:1098A0006F927F928F929F92AF92BF92CF92DF92F0
:1098B000EF92FF920F931F93CF93DF9300D000D0CE
:1098C000CDB7DEB78C01C2DA98012E533E4F3C83F0
:1098D0002B831E830D83D801AC55BE4FBA83A98359
:1098E0001801B2E02B1ABEEF3B0AF901AA24A39497
:1098F000B12C32E0832E912C118210829F012A54C8
:109900003140D9012D913C91232B09F44DC0AD81FB
:10991000BE812D913D914D915C9113977D01B4EBEA
:10992000EB0EF11CD701CD90DD90ED90FC902B015A
:109930003C01421A530A640A750A4C145D046E0411
:109940007F0490F1C20ED31EE41EF51EAD81BE81D0
:10995000CD92DD92ED92FC921397A981BA812C9160
:10996000222311F19F0126593109D9012D913C91F2
:109970002115310519F4B182A08216C07F01BAE524
:10998000EB1AF108D7014D915C91119742175307DB
:109990005CF4B182A0824F5F5F4F4D935C9342179E
:1099A000530714F09182808232962D813E812C5F84
:1099B0003F4F3E832D83A981BA811196BA83A98333
:1099C000E215F30509F098CFEB81FC81819191912B
:1099D000FC83EB838130910599F00297C9F4EB8108
:1099E000FC81EC54F1400190F081E02D1995AB81A0
:1099F000BC81DA966D917C91DB97C801EEDE08C0E0
:109A0000EB81FC81EC54F1400190F081E02D19953F
:109A10002B813C8122153305B9F626960FB6F894B2
:109A2000DEBF0FBECDBFDF91CF911F910F91FF9091
:109A3000EF90DF90CF90BF90AF909F908F907F90EE
:109A40006F905F904F903F902F9008956E3E22E070
:109A5000720738F06B3C98E0790728F06AEC78E000
:109A600002C06EEE72E0660F771F9FB7F89425E193
:109A7000829FF0011124EE57FE4E748363839FBFD3
:109A80000895482F50E095E1899FF0011124EE5789
:109A9000FE4E2181328180859185280F391F838177
:109AA00094818217930728F08581968128173907BA
:109AB000E8F485E1849FF001859FF00D1124EE57B5
:109AC000FE4E858196812817390728F52581368134
:109AD00085E1849FF001859FF00D1124EE57FE4E25
:109AE0008285823019F411861086128685E1849F62
:109AF000F001859FF00D1124EE57FE4E3283218335
:109B00008091840090918500280F391F309389003F
:109B10002093880008958381948182179307C0F66B
:109B200023813481D5CF8091710A811157C0E09192
:109B30006211F09163118581968190935F118093FA
:109B40005E111092611110926011E0916C11F09110
:109B50006D1185819681909369118093681110929F
:109B60006B1110926A11E0917611F0917711858155
:109B700096819093731180937211109275111092C7
:109B80007411E0918011F0918111858196819093FB
:109B90007D1180937C1110927F1110927E1182E1D1
:109BA00090E0909356118093551181E080935B1162
:109BB0008093651180936F11809379118093571171
:109BC00080E090E021E0FC01EF5FFE4E21830796EC
:109BD00084359105C1F781E08093710A0895109250
:109BE0007B1108951092711108958F929F92AF92F8
:109BF000BF92CF92DF92EF92FF921F93CF93DF93AA
:109C0000EC0111E08E819F81892B09F410E02C81F9
:109C10003D81E885F985C580D680878190E0A601E1
:109C2000480F591F2417350764F180850D2C000C4F
:109C3000EE08FF08A901330F660B770B0380F48150
:109C4000E02D9A01AB012C193D094E095F098823CB
:109C500029F0A1E0BFEF0E942AAD04C0AFEFB0E051
:109C60000E941EAD4F01FF0FAA08BB08A501940179
:109C70002C193D094E095F090E9402AD3F832E83D6
:109C80004BC0A601481B590B421753070CF43FC0A9
:109C900080850D2C000CEE08FF08A901330F660B20
:109CA000770B81809280092C000CAA08BB089A01CE
:109CB000AB01281939094A095B09882399F0A1E009
:109CC000BFEF0E942AADA7019601281939094A0958
:109CD0005B090E9402ADDA01C90181509F4FAF4F6D
:109CE000BF4F12C0AFEFB0E00E941EADA7019601BA
:109CF000281939094A095B090E9402ADDA01C90134
:109D00008F5F9109A109B1099F838E8305C01F82CE
:109D10001E82111101C019828E819F81009789F0E6
:109D20008F3F910519F014F08FEF90E081305FEFD5
:109D3000950714F481E09FEF9F838E8381E01827BD
:109D40001A83DF91CF911F91FF90EF90DF90CF901A
:109D5000BF90AF909F908F90089581E080936E0A9E
:109D6000089581E080936F0A089581E08093700ADE
:109D700008958091770A833029F48091740D909131
:109D8000750D08C70895CF93DF93C091670DD091EB
:109D9000680D6091A20D7091A30DCE0106DD8111B9
:109DA0000CC023E93DE44CE251E060E070E0CE01FC
:109DB00063DD9093A30D8093A20DDF91CF91089561
:109DC0006E3E22E0720738F06B3C98E0790728F08D
:109DD0006AEC78E002C06EEE72E0660F771F9FB704
:109DE000F89425E1829FF0011124EE57FE4E768310
:109DF00065839FBF0895660F771F282F30E095E198
:109E0000899FF0011124EE57FE4E858196816817D7
:109E1000790718F46581768107C08381948186175C
:109E2000970710F4638174818FB7F89495E1929F3E
:109E3000F001939FF00D1124EE57FE4E7283618363
:109E40008FBF0895982F8FB7F89425E1929FF00166
:109E50001124EE57FE4E21E027838FBF41B121E050
:109E600030E0B90102C0660F771F9A95E2F7CB0187
:109E7000842B81B908958A3058F49FB7F89425E16E
:109E8000829FF0011124EE57FE4E118610869FBF6F
:109E900008951F93CF93DF9325E1829FC001112482
:109EA000EC01CE57DE4E8A8581110FC01FB7F894A2
:109EB00081E08A8789899A899A8389830E942647C3
:109EC0006B877C878D879E871FBFDF91CF911F9106
:109ED0000895CF93DF938A30D0F56233710538F05F
:109EE00061369DE6790728F060E67DE602C062E310
:109EF00070E0D42FC82F80E090E00E94BDAB20E03E
:109F000030E04AE754E40E9418A820E030E04CE832
:109F100052E40E941EAC9B01AC0160E070E08AEF4D
:109F200094E40E9418A80E9480A89B01DD2321F0E0
:109F300022273327261B370B8FB7F89495E1C99F4B
:109F4000F0011124EE57FE4E318720878FBFDF913D
:109F5000CF9108958A3008F479CD08958A3008F4B5
:109F60002FCF08958A3058F495E1899FF00111248C
:109F7000EE57FE4E8181928196958795089580E0F7
:109F800090E008958A3008F436CF08951F920F921A
:109F90000FB60F9211240BB60F920F931F932F93AE
:109FA0003F934F935F936F937F938F939F93AF9361
:109FB000BF93CF93EF93FF938091BF0D893048F00B
:109FC0001092BF0D80913112882399F080912A124E
:109FD0000DC0E091BF0DE15025E1E29FF001112499
:109FE000EE57FE4E8781882321F0808192B1892728
:109FF00082B9E091BF0D85E1E89FF0011124EE5791
:10A00000FE4E8781882321F0808192B1892B82B90D
:10A01000E091BF0DC5E1CE9FF0011124EE57FE4E39
:10A0200080859185892B09F04DC0E091BF0DCE9FB1
:10A03000F0011124EE57FE4E8285813009F060C098
:10A040000E942647E091BF0DCE9FF0011124EE57EC
:10A05000FE4E0385148525853685E091BF0DCE9F84
:10A06000F0011124EE57FE4E0784F089E02DAB017C
:10A07000BC01401B510B620B730BCF01A0E0B0E0A1
:10A0800084179507A607B707D8F5E091BF0DA091F3
:10A09000BF0DCA9FD0011124AE57BE4E53968D916D
:10A0A0009C915497CE9FF0011124EE57FE4E91875C
:10A0B0008087E091BF0DCE9FF0011124EE57FE4E38
:10A0C00082E082878091BF0DDCDC8091BF0D8F5FC5
:10A0D0008093BF0DFF91EF91CF91BF91AF919F9171
:10A0E0008F917F916F915F914F913F912F911F9130
:10A0F0000F910F900BBE0F900FBE0F901F901895F1
:10A10000E091BF0D809184009091850025E1E29F50
:10A11000F0011124EE57FE4E21813281820F931FF0
:10A120009093890080938800D0CF1F93CF93DF93C3
:10A130008091BE0D811173C01092BF0D9FB7F8942E
:10A1400085E128EB3BE04CED55E064E971E1A1E0ED
:10A15000B0E0E091BF0DE93008F052C0E091BF0DD2
:10A160008E9FF0011124EE57FE4E32832183E09141
:10A17000BF0D8E9FF0011124EE57FE4E568345838E
:10A18000E091BF0D8E9FF0011124EE57FE4E7483B7
:10A190006383E091BF0DF091BF0DED0101C0CC0FC5
:10A1A000FA95EAF78E9FF0011124EE57FE4EC08318
:10A1B000E091BF0D8E9FF0011124EE57FE4E1782E5
:10A1C000E091BF0D8E9FF0011124EE57FE4E1186D7
:10A1D0001086E091BF0D8E9FF0011124EE57FE4EC8
:10A1E0001286E091BF0D8E9FF0011124EE57FE4EB6
:10A1F000148A138AE091BF0DEF5FE093BF0DA9CFE2
:10A200009FBF8FB7F89420EA3FE030932C12209341
:10A210002B1210922A128FBF81E08093BE0DDF9126
:10A22000CF911F9108950F931F93CF93DF938C01CC
:10A23000C62FD42FDC0111968D919C911297DC01D1
:10A24000ED91FC910190F081E02DD8016C91199570
:10A25000F80181819281DC01ED91FC910190F08106
:10A26000E02D6C2F1995F80181819281DC01ED912F
:10A27000FC910190F081E02D6D2F1995F8018081FE
:10A280006C2F70E0680F711D6D0F711D6F77772750
:10A2900081819281DF91CF911F910F910C948B3925
:10A2A0000F931F93CF93DF938C01C62FD42FDC0124
:10A2B00011968D919C911297DC01ED91FC9101908A
:10A2C000F081E02DD8016C911995F801818192817E
:10A2D000DC01ED91FC910190F081E02D6C2F19953E
:10A2E000F80181819281DC01ED91FC910190F08176
:10A2F000E02D6D2F1995F80180816C2F70E0680FAB
:10A30000711D6D0F711D6F77772781819281DF91AC
:10A31000CF911F910F910C948B394F925F926F9256
:10A320007F92AF92BF92CF92DF92EF92FF921F93F4
:10A33000CF93DF93DD24D39445E0C42E52E0A52EC5
:10A34000B12CC3E0D0E0EE24E394F12C80919C0D7D
:10A3500090919D0DDC01ED91FC910480F581E02D43
:10A360001995892B09F4BEC01091300180919C0D84
:10A3700090919D0DDC01ED91FC910680F781E02D1F
:10A38000199596B3B39A2091840030918500205995
:10A39000384E30938D0020938C00212F2C7139F092
:10A3A0001092BD0DD0939B0DC0939A0DCFCF93FB10
:10A3B000992790F9E091BD0DE11116C0992331F272
:10A3C0008F3021F6D092BD0D8093A40D80919A0D0F
:10A3D00090919B0D892B09F0B9CFF0929B0DE092E3
:10A3E0009A0D1092990DB2CF9111DACF91E09E0F94
:10A3F0009093BD0DF0E0EC55F24F8083993109F058
:10A40000A5CF81116CC08091BB0D82FF05C0D09398
:10A410009B0DC0939A0D63C083FDF9CF80919A0D77
:10A4200090919B0D019739F48091990D8F5F8093E6
:10A43000990D843020F0B0929B0DA0929A0D8091DE
:10A44000980D8F5F8093980D9091970D981708F055
:10A4500044C0D092960DA6E7BDE0E5EAFDE040E0FD
:10A4600050E0BA0110E0CF01FC011B3098F40196D6
:10A470004080512C612C712C012E04C0440C551CC1
:10A48000661C771C0A94D2F7442955296629772936
:10A49000185FEACF9A013770205E3340C29EC00138
:10A4A000C39E900D112497FD079623E095958795FF
:10A4B0002A95E1F784529A4F8D939D931B503BE070
:10A4C00076956795579547953A95D1F78DE0A639DA
:10A4D000B80749F61092980D02C01092960D10928E
:10A4E000BD0D34CFDF91CF911F91FF90EF90DF90A2
:10A4F000CF90BF90AF907F906F905F904F900895F6
:10A500008091770A823029F48091720D9091730DB9
:10A5100004CF0895F5DF2DCC10925B1110926511D8
:10A5200010926F11109279111092571180E090E003
:10A53000FC01EF5FFE4E1182079684359105C1F74D
:10A5400008958091770A823039F0833049F0813064
:10A5500049F480916F0D01C080E18093730A04C0BB
:10A560008EE0FBCF1092730A8091730A0895809158
:10A57000770A823039F0833049F0813059F4809184
:10A580006E0D0895BDDF8091960D0895F2DB8091E8
:10A590006D0D089580E008958091770A823049F02A
:10A5A000833069F0813089F48091690D90916A0D52
:10A5B0000895A6DF80919A0D90919B0D0895D9DBA7
:10A5C00080916B0D90916C0D089581E090E008955D
:10A5D000AF92BF92CF92DF92EF92FF920F931F93B1
:10A5E000CF93DF93CDB7DEB7EDB6FEB689DFC1DB23
:10A5F000D3DF029709F0B4C1BADF882309F4ACC1F4
:10A60000A090A20DB090A30DC090670DD090680DE2
:10A61000B501C601CAD88823F1F0F601E250FE4F19
:10A6200000E010E0819191918A159B0571F40E94E0
:10A630002647000F111F000F111FF601E00FF11F39
:10A64000608371838283938307C00F5F1F4F0E3136
:10A65000110541F701C097DB1092710ACDB6DEB645
:10A660004091740A5091750ACA01880F991F2DB73D
:10A670003EB7281B390B0FB6F8943EBF0FBE2DBF57
:10A680000DB71EB70F5F1F4F8091770A823069F0B8
:10A69000833029F1813009F071C0B8018091700DCB
:10A6A0009091710D0E943F6A33C03FB7F89420E04B
:10A6B000822F90E08417950774F4880F991FF80192
:10A6C000E80FF91FDC01AA58B24F8D919C9191833C
:10A6D00080832F5FEDCF3FBF1092960D19C03FB71B
:10A6E000F89420E0822F90E08417950774F4880F87
:10A6F000991FF801E80FF91FDC01A55BB24F8D919E
:10A700009C91918380832F5FEDCF3FBF10926D0DA1
:10A7100020E06AE071E0822F90E04091740A50914D
:10A72000750A8417950754F5689FF001699FF00D2D
:10A730001124EF59FF4EA085B1858C918823E1F05B
:10A74000A081B1813C91C801830F911D830F911DA0
:10A75000DC0112978D919C91A281B3814D915C9106
:10A7600011970480F581E02D4817590711F41082E4
:10A7700003C070838D939C932F5FCDCF0FB6F89459
:10A78000DEBE0FBECDBE80915B11882319F08AE535
:10A7900091E12BDA80916511882319F084E691E12B
:10A7A00024DA80916F11882319F08EE691E11DDA89
:10A7B00080917911882319F088E791E116DA809168
:10A7C000720A882309F465C080916F11811105C058
:10A7D00080917911882309F450C080917211909171
:10A7E0007311E0917611F09177112381348128174C
:10A7F000390724F48085811109C00EC0218132817E
:10A800008217930734F48085811106C088E090E0B8
:10A8100005C080E190E002C080E290E020917C11D0
:10A8200030917D11E0918011F0918111438154812B
:10A830004217530724F42085222349F00AC041819E
:10A840005281241735073CF42085222311F08160C2
:10A8500003C0846001C0826020915511309156116F
:10A860002817390719F41092571107C09093561101
:10A870008093551181E080935711809155119091EB
:10A880005611429709F46FC081E080937B11809349
:10A890007111E1E0F1E182E0C82E81E1D82E25E0DE
:10A8A00031E141E08081882309F44AC065817681E5
:10A8B000DB0117968C91882309F442C0D6018C9154
:10A8C0008823F1F18281938140838A33B7E09B072B
:10A8D00094F48C0101541640093F110570F00753A0
:10A8E0001F4F093C110558F08F579440893F91053F
:10A8F00040F081E007C085E005C084E003C083E04C
:10A9000001C082E0DB0119969C91992379F0813096
:10A9100041F0823041F0843041F0853039F481E0FB
:10A9200005C085E003C084E001C082E0D9019C91AC
:10A93000D601981302C01C9203C04C93D9018C938A
:10A940003796B7E0CB0ED11C295F3F4F51E1E5357B
:10A95000F50709F0A7CF02C0DFDD15DA81E065C099
:10A96000DBDD80E062C0C0905811D09059111C14FA
:10A970001D040CF055C0809170110091670D10916D
:10A98000680D6091A00D7091A10D8823B1F081E058
:10A9900080937111C8010E94D54B811115C0A60189
:10A9A000DD0C660B770B22EF3DE4C8010E943C4CA6
:10A9B0009093A10D8093A00D07C0C8010E94D54BB4
:10A9C000811102C01092711180917A110091670D6E
:10A9D0001091680D60919E0D70919F0D8823D1F0AC
:10A9E00081E080937B11C8010E94D54B811151CF2A
:10A9F0004091581150915911052E000C660B770BA0
:10AA00002FEE3DE4C8010E943C4C90939F0D809333
:10AA10009E0D3FCFC8010E94D54B81113ACF02C095
:10AA20001092711110927B1134CF0FB6F894FEBEC4
:10AA30000FBEEDBEDF91CF911F910F91FF90EF9070
:10AA4000DF90CF90BF90AF900895FC0112821382E7
:10AA500014821582168217821286089580E0089566
:10AA60000F931F93CF938C0169E870E180E998E020
:10AA70000E940042D8011896ED91FC9119976081CF
:10AA8000718180E998E00E94477CC1E0D8011A9664
:10AA90008C91C81710F564E870E180E998E00E9495
:10AAA00000426C2F80E998E00E94E47F61E870E149
:10AAB00080E998E00E940042F80190858185E92FA5
:10AAC000F82FEC0FF11DEC0FF11D6081718180E911
:10AAD00098E00E94477CCF5FD9CFCF911F910F9113
:10AAE0000895CF93DF93CDB7DEB76E970FB6F89486
:10AAF000DEBF0FBECDBF8F300CF080E029E730E124
:10AB00003A83298322E730E13C832B8324E630E13A
:10AB10003E832D8328E530E138872F832EE430E112
:10AB20003A87298727E430E13C872B8723E430E10B
:10AB30003E872D872CE330E1388B2F8721E330E1EE
:10AB40003A8B298B24E230E13C8B2B8B29E130E1DD
:10AB50003E8B2D8B2DE030E1388F2F8B2BEF3FE09C
:10AB60003A8F298F2AEE3FE03C8F2B8F25EE3FE076
:10AB70003E8F2D8FE82FEE0FFF0BEC0FFD1F818115
:10AB800092816E960FB6F894DEBF0FBECDBFDF91F7
:10AB9000CF910895AF92BF92CF92DF92EF92FF9242
:10ABA0000F931F93CF93DF9389EC9DE07EE1D72E27
:10ABB000D80ECC24C39402E010E0C3E0D0E0E2E081
:10ABC000BE2EEE24E394F12C8091160E9091170E78
:10ABD000DC01ED91FC910480F581E02D1995892B24
:10ABE00009F4ADC0A09030018091160E9091170E1F
:10ABF000DC01ED91FC910680F781E02D199596B36B
:10AC0000B39A2091840030918500285A344E3093B5
:10AC10008D0020938C002A2D2C7119F01092130EA8
:10AC20004BC093FB992790F9E091130EE11116C0E8
:10AC3000992351F2803241F6C092130E8093C90DD0
:10AC400080916B0D90916C0D892B09F0BDCFF09226
:10AC50006C0DE0926B0D1092150EB6CF9111DECFF8
:10AC6000E13041F4803409F0AFCFB092130E8093FD
:10AC7000CA0DE6CF91E09E0F9093130EF0E0E753DC
:10AC8000F24F8083903209F09FCF1092130EE9ECBF
:10AC9000FDE02FEF3FEF8191281B3109DE12FBCF42
:10ACA0004091E70D8091E80D90E0982F8827840F60
:10ACB000911D2817390729F0D0936C0DC0936B0DA7
:10ACC00083CF80916B0D90916C0D019739F4809139
:10ACD000150E8F5F8093150E843020F010936C0D4D
:10ACE00000936B0D8091140E8F5F8093140E9091E2
:10ACF000120E981708F5C0926D0D20E030E0F901B2
:10AD0000E753F24F4281838190E0982F8827840F88
:10AD1000911DAC014F5E52404B3D554028F4F90166
:10AD2000E55BF24F918380832E5F3F4F2C313105DD
:10AD300031F71092140E48CF10926D0D45CFDF9170
:10AD4000CF911F910F91FF90EF90DF90CF90BF9028
:10AD5000AF900895EF92FF920F931F93CF93DF93DD
:10AD60001092980E82E08093990E68EE73E07093D3
:10AD70009B0E60939A0E40ED57E050939D0E4093CA
:10AD80009C0E2CED35E030939F0E20939E0E8FE0AD
:10AD90008093A00E1092A10E94E09093A20E709357
:10ADA000A40E6093A30E5093A60E4093A50E30936D
:10ADB000A80E2093A70E8093A90E1092AA0E93E0DE
:10ADC0009093AB0E7093AD0E6093AC0E5093AF0E9C
:10ADD0004093AE0E3093B10E2093B00E8093B20E1E
:10ADE0001092B30E91E09093B40E7093B60E6093F0
:10ADF000B50E5093B80E4093B70E3093BA0E209311
:10AE0000B90E8093BB0E1092BC0EEDEBFEE0A6ECEB
:10AE1000BEE080E008EE13E060ED77E04CED55E039
:10AE200031E022E095E0980F9083128301837483D0
:10AE3000638356834583ED01229791E03883219601
:10AE400028831C928F5F3A961A968C3059F710928D
:10AE5000350F9093360F1092370F9093380F80E094
:10AE600090E09C012856314FF901EF55FF4F1182B8
:10AE700010823296108203968837910591F784E20A
:10AE800090E090933A0F8093390F81E080933B0FCD
:10AE90002CE030E030933D0F20933C0F94E09093F2
:10AEA0003E0F21E230E03093400F20933F0F27E028
:10AEB0002093410F29E030E03093430F2093420F5D
:10AEC00020E12093440F7AE07093B10F2BE02093A0
:10AED000B20F2093B30F48EE53E05093B50F409359
:10AEE000B40F20ED37E03093B70F2093B60F1092D8
:10AEF000B80F64E66093B90F6093BA0F5093BC0F1C
:10AF00004093BB0F3093BE0F2093BD0F1092BF0F25
:10AF10001092C00F8093C10F1092C30F1092C20FF6
:10AF20008093C40F8093C50FE8ECF0E0F093C70F57
:10AF3000E093C60FE0E2F3E0F093C90FE093C80F8F
:10AF40005093CB0F4093CA0F3093CD0F2093CC0F6B
:10AF50008093CE0FE9E5F0E0F093D00FE093CF0FB0
:10AF6000E0E8F0E0F093D20FE093D10FEFEFF0E0E4
:10AF7000F093D40FE093D30FF093D60FE093D50F57
:10AF80008093D70F9093D80F1092D90F8093DA0F38
:10AF90009093DB0F1092DC0F1092DD0F8093DE0F89
:10AFA0001092DF0F1092E00F8093E10F1092E20FEA
:10AFB00098E29093E30F5093E50F4093E40F509382
:10AFC000E70F4093E60F3093E90F2093E80F80934B
:10AFD000EA0F92E39093EB0FE2E0E093EC0F8093A3
:10AFE000ED0F6093EE0FE6E4E093EF0F9093F00F18
:10AFF0001092F10F1092F20F1092F30F1092F40FC3
:10B000001092F50F1092F60FEAEFF0E0F093F80FC0
:10B01000E093F70F1092F90F1092FA0F6093FB0F65
:10B0200061E46093FC0F1092FD0F9093FE0F10925D
:10B03000FF0F90930010EEE5F1E0F0930210E09323
:10B04000011010920310ACEDB5E0B0930510A09381
:10B05000041000EA1FE010930710009306103093CD
:10B06000091020930810C8E8D3E1D0930B10C093C7
:10B070000A1068EBE62E6BE0F62EF0920D10E092CF
:10B080000C10E0E4FFE1F0930F10E0930E1010922B
:10B090001010109211101092121069E160931310A9
:10B0A00080931410809315108093161050931810ED
:10B0B0004093171030931A1020931910F0921C101F
:10B0C000E0921B1010931E1000931D10D0932010BF
:10B0D000C0931F1020E737E13093221020932110F6
:10B0E0001092231010922410109225109093261085
:10B0F0009093271090932810809329101092391064
:10B1000010922A1099E090932B1010922C1010920C
:10B110002D1010922E1010922F10B0933110A0937A
:10B120003010F0933310E09332108093341070930A
:10B1300035101092361021E030E030933810209313
:10B14000371040E052EC61E070E040933A105093C9
:10B150003B1060933C1070933D1040933E10509311
:10B160003F10609340107093411040E056E960E05A
:10B1700070E04093421050934310609344107093DA
:10B1800045104093461050934710609348107093B9
:10B19000491010924A1020E039E130934C1020936E
:10B1A0004B1010924D109EE190934E1010924F1044
:10B1B0002EE130E030935110209350103093531013
:10B1C00020935210309355102093541090935610A2
:10B1D00090935710809358108093591010925A10E2
:10B1E00090935B1080935C108AE29FE4A0E0B0E053
:10B1F00080935D1090935E10A0935F10B0936010E9
:10B2000008E91EE0C0E0D0E0CE010E94E2ACF80107
:10B2100061918F01861719F0CE010E94F4AC21963E
:10B22000C93CF1E0DF0781F7DF91CF911F910F91CA
:10B23000FF90EF9008954F925F926F927F928F925E
:10B240009F92AF92BF92CF92DF92EF92FF92CF93F5
:10B25000DF93EB01A091C70DB091C80D9D012F5F49
:10B260003F4F45E0429F2001439F500C1124052C85
:10B27000000C66087708812C912C54012A33E1E0F8
:10B280003E07ECF446EC5DE661E07727750164016A
:10B29000C40CD51CE61CF71C4C0D5D1D6E1D7F1DDE
:10B2A0006BBFFA014791569165E0860E911CA11C77
:10B2B000B11CC417D50729F12F5F3F4FDFCF25E021
:10B2C000822E912CA12CB12C21E030E0A217B307E3
:10B2D00008F44CC046EC5DE661E07727480D591D47
:10B2E0006A1D7B1D6BBFFA0147915691F5E08F0EE9
:10B2F000911CA11CB11CC417D50719F02F5F3F4F3B
:10B30000E5CF46EC5DE661E07727E5E0E29F60018E
:10B31000E39FD00C11240D2C000CEE08FF084E5FAB
:10B320005F4F6F4F7F4F4C0D5D1D6E1D7F1D6BBFBF
:10B33000FA0147915691FC015383428346EC5DE646
:10B3400061E077274C5F5F4F6F4F7F4FC40ED51E74
:10B35000E61EF71EEBBEF601C790FC01C4823093D7
:10B36000C80D2093C70DC901019606C01092C80DE3
:10B370001092C70D80E090E0DF91CF91FF90EF90A9
:10B38000DF90CF90BF90AF909F908F907F906F9005
:10B390005F904F9008950F931F938091C60D811178
:10B3A0001EC00E9426470091C20D1091C30D20912E
:10B3B000C40D3091C50DAB01BC01401B510B620B9C
:10B3C000730B8091C00D9091C10DA0E0B0E0841787
:10B3D0009507A607B70718F481E08093C60D1F9163
:10B3E0000F9108952F923F924F925F926F927F92AA
:10B3F0008F929F92AF92BF92CF92DF92EF92FF9285
:10B400000F931F93CF93DF9300D0CDB7DEB75C01CE
:10B410000E943B620E94D8730E940F7480915A066A
:10B4200090915B060E945E430E94138524E0A21661
:10B43000B10409F448C085E0A816B10409F479C044
:10B44000A3E0AA16B10409F0B1C08CE190E00E941B
:10B45000B9A89B838A8385E895E0EA81FB81918383
:10B460008083B382A28281E09FEF958384838FEFF4
:10B4700090E09783868311861086108ECF010E94FC
:10B48000955089E795E0AA81BB818D939C93E091CB
:10B49000900EF091910ED08C0091C6111091C711B1
:10B4A00016950795E090C411F090C511F694E794B5
:10B4B00061E971E180915A0690915B060E947143A7
:10B4C0002224239490C08CE190E00E94B9A89B8331
:10B4D0008A8385E895E0EA81FB8191838083B3824A
:10B4E000A28281E09FEF958384838FEF90E0978322
:10B4F000868311861086108ECF010E94955089E7B1
:10B5000095E0AA81BB818D939C93E0915806F091C0
:10B510005906D08C0091DB111091DC11169507951E
:10B52000E090D911F090DA11F694E79464EC71E1AF
:10B5300035C08CE190E00E94B9A89B838A8385E89E
:10B5400095E0EA81FB8191838083B382A28281E0CE
:10B550009FEF958384838FEF90E097838683118696
:10B560001086108ECF010E94955089E795E0AA8140
:10B57000BB818D939C93E0915406F0915506D08C3D
:10B580000091F0111091F11116950795E090EE11D0
:10B59000F090EF11F694E79464EA71E180915A0615
:10B5A00090915B060E947143212C1DC068E771E1F8
:10B5B00080915A0690915B060F900F900F90DF914B
:10B5C000CF911F910F91FF90EF90DF90CF90BF90A0
:10B5D000AF909F908F907F906F905F904F903F9033
:10B5E0002F900C9471430E9413856BE671E180915A
:10B5F0005A0690915B060E9471436FE571E180915C
:10B600005A0690915B060E940042B80180915A064A
:10B6100090915B060E94348063E571E180915A0647
:10B6200090915B060E940042B70180915A0690916A
:10B630005B060E94348067E471E180915A06909124
:10B640005B060E9400428D2D0E94EF8480915A0675
:10B6500090915B060E945E43AA81BB81ED91FC91B3
:10B6600011970280F381E02DCD011995CA2C8A2D06
:10B670000E94B24F8D3D9540A8F464E378E08A2D96
:10B680000E94AA4FEA81FB81F78AE68AB70182818C
:10B690000E94C24F6CED75E08A2D0E94AE4FDD20F6
:10B6A000C1F01AC064E873E08A2D0E94AE4FAA81EF
:10B6B000BB8157961C930E935697B80112968C91A6
:10B6C0000E94C24F6CED75E08A2D0E94AA4FDD20CA
:10B6D00019F09924939401C0912C33243394812C34
:10B6E00021E029830E94E85280916F11882359F14B
:10B6F000AA81BB81ED91FC911197609174117091B9
:10B7000075110190F081E02DCD0119958C2D0E94CD
:10B71000B24F8D3DB5E09B075CF48438E3E09E07B3
:10B7200084F08C018D3D954074F00CED15E00BC05C
:10B730007C01853398403CF064E3E62E68E0F62E09
:10B7400002C004E813E0298121111FC08091651116
:10B750008823C9F1E0916C11F0916D11858196817A
:10B7600040916811509169119C0121533109421790
:10B7700053074CF1C196841795072CF10E94264778
:10B780006415750586059705F0F08091651188238D
:10B79000C1F04091681150916911E0916C11F091E4
:10B7A0006D11858196819C01285C310942175307F0
:10B7B0002CF088539F4F841795071CF481E098263E
:10B7C00005C021E02983882009F47CC0992009F470
:10B7D00045C0DD20F9F064E873E08C2D0E94AE4F87
:10B7E000222009F458C06091C80F7091C90F41E040
:10B7F0008C2D0E94694F0E94E47BAA81BB81129626
:10B800008C910E94B24F08171907ACF38C2D0E943F
:10B810003B4F41C064E378E08C2D0E94AA4F222068
:10B82000B1F06091C80F7091C90F40E08C2D0E945B
:10B83000694F0E94E47BAA81BB8112968C910E9481
:10B84000B24F8E159F05ACF38C2D0E943B4FEA81C1
:10B85000FB81F78AE68AB701828110C0DD20B1F052
:10B8600064E378E08C2D0E94AA4FAA81BB81579691
:10B87000FC92EE925697B70112968C910E94C24F9D
:10B880006CED75E08C2D0E94AE4F12C064E873E041
:10B890008C2D0E94AE4FEA81FB81178B068BB8017D
:10B8A00082810E94C24F6CED75E08C2D0E94AA4FE0
:10B8B0000E9426472B013C01F8EC4F0E511C611CE5
:10B8C000711C19823320D9F180915B118823A9F171
:10B8D00040915E1150915F11E0916211F0916311FE
:10B8E000858196819C01285C3109421753072CF011
:10B8F00088539F4F8417950704F581E0D8268091DF
:10B900005A0690915B06DD2039F068E371E10E94F0
:10B91000714382E090E006C066E271E10E947143EB
:10B9200081E090E00E94E0730E942647AA81BB81DB
:10B930005896DC928824839403C0812C1EC0812CED
:10B9400080915B11882309F409C2E0916211F091A2
:10B9500063118581968140915E1150915F119C0128
:10B9600021533109421753070CF4F8C1C19633240F
:10B970003394841795070CF4F1C10E948A520E94F7
:10B98000757F8CE89AE00E944C4C80917B0A88235A
:10B9900009F4A8CE80917D0A882309F4A3CE0E94E1
:10B9A000757F0E94C8878823D1F3B4E0AB16B10439
:10B9B00059F0E5E0AE16B10409F465C0F3E0AF1646
:10B9C000B10409F059C1CBC01093B50F0093B40F67
:10B9D000F092B70FE092B60FD092B80FB8018CE199
:10B9E00091E00E94067FB7018EE191E00E94067F00
:10B9F0006D2D80E291E00E946980B80184E00E9490
:10BA0000E04EB70184E00E94264DE0915806F09187
:10BA10005906D08E8091B30F8D3029F4E091EA0D54
:10BA2000F091EB0DD08E6CED75E084E00E94C24F7A
:10BA300066E970E080E090E00E94EE468091B30FEE
:10BA40008D30E1F484E00E94B24FA0915806B0918D
:10BA50005906ED91FC9111970190F081E02D8D3DFB
:10BA600095401CF06FEF7FEF02C061E070E0CD0108
:10BA7000199580915806909159065BC0809158069F
:10BA80009091590664C01093BC0F0093BB0FF092C5
:10BA9000BE0FE092BD0FD092BF0FB80183E291E0DC
:10BAA0000E94067FB70185E291E00E94067F6D2D1E
:10BAB00087E291E00E946980B80185E00E94E04E33
:10BAC000B70185E00E94264DE0915406F09155069D
:10BAD000D08E6CED75E085E00E94C24F66E970E0A3
:10BAE00080E090E00E94EE468091B20F8D3059F5D3
:10BAF00085E00E94B24FA0915406B09155068D3D4D
:10BB000095404CF0ED91FC9111970190F081E02D62
:10BB10006FEF7FEF08C0ED91FC9111970190F081DC
:10BB2000E02D61E070E0CD0119958091540690916F
:10BB30005506DC01ED91FC910190F081E02D60E073
:10BB400070E0199599C08091540690915506DC01DA
:10BB5000ED91FC910480F581E02D19958DC0109335
:10BB6000CB0F0093CA0FF092CD0FE092CC0FD09282
:10BB7000C40FB80182E391E00E94067FB70184E31D
:10BB800091E00E94067F6D2D8CE291E00E94698019
:10BB9000B80183E00E94E04EB70183E00E94264D89
:10BBA0008091C40FE091900EF091910E808F809162
:10BBB000C40F0E94D17E83E00E94B24F2091C40F37
:10BBC000222369F1B9E0BC1538F02091C6113091FB
:10BBD000C7113695279502C02EEE32E082179307E3
:10BBE00009F44AC06091C80F7091C90F41E083E029
:10BBF0000E94694F0E94E47BEA81FB8182810E945E
:10BC0000B24F08171907B4F383E00E943B4FAA8193
:10BC1000BB8157961C930E935697B80129C029E013
:10BC20002C1508F49DC02091C4113091C511369592
:10BC300027958217930701F16091C80F7091C90F82
:10BC400040E083E00E94694F0E94E47BEA81FB812F
:10BC500082810E94B24F8E159F05B4F383E00E944B
:10BC60003B4FAA81BB815796FC92EE925697B70143
:10BC700012968C910E94C24F80915A0690915B0659
:10BC80000E945E430E941385B4E0AB16B10459F0E4
:10BC9000E5E0AE16B10451F0F3E0AF16B10471F473
:10BCA0006CED70E105C06CE071E102C063EF70E122
:10BCB00080915A0690915B060E9471430E94138501
:10BCC00061ED70E180915A0690915B060E9471438C
:10BCD00065EC70E180915A0690915B060E940042EB
:10BCE000B80180915A0690915B060E94348069EBFE
:10BCF00070E180915A0690915B060E940042B70164
:10BD000080915A0690915B060E9434806DEA70E142
:10BD100080915A0690915B060E9400428D2D0E94F0
:10BD2000EF8480915A0690915B060E945E430F90CB
:10BD30000F900F90DF91CF911F910F91FF90EF9097
:10BD4000DF90CF90BF90AF909F908F907F906F903B
:10BD50005F904F903F902F900C940B74312C0DCE30
:10BD60002AEC38E066CFCF93DF93CDB7DEB72897C4
:10BD70000FB6F894DEBF0FBECDBF8091E90D8823CA
:10BD8000C9F11092E90D0E94827380915D068823AB
:10BD900089F16EE970E180915A0690915B060E94EC
:10BDA0000042E091770AE4300CF0E0E084E095E0B6
:10BDB0009A83898380E095E09C838B838BEF94E06A
:10BDC0009E838D8386EF94E098878F83EE0FFF0B21
:10BDD000EC0FFD1F6181728180915A0690915B0684
:10BDE00028960FB6F894DEBF0FBECDBFDF91CF917E
:10BDF0000C94714328960FB6F894DEBF0FBECDBFEA
:10BE0000DF91CF9108958091E90D811112C033D354
:10BE100081E08093E90D0E949F7380915C068823E6
:10BE200041F06FE870E180915A0690915B060C94A6
:10BE30007143089560E089E30E94784560E08AE3F9
:10BE40000E94784560E085E30E94784560E085E0E7
:10BE50000E94784560E084E00E94784560E087E0D9
:10BE60000E94784572980895CF93DF938091F20DE8
:10BE700081110DC01092F10D1092F00D81E090E053
:10BE80009093EF0D8093EE0D8093F20D36C080916C
:10BE9000F00D9091F10D863191057CF18F3891056F
:10BEA00034F48091EE0D9091EF0D019609C08D351F
:10BEB00021E0920754F48091EE0D9091EF0D0296DF
:10BEC0009093EF0D8093EE0D18C0863222E092071A
:10BED00034F48091EE0D9091EF0D0496F1CF883EF1
:10BEE00093403CF48091EE0D9091EF0D8A5B9F4F53
:10BEF000E7CF1092EF0D1092EE0D0E94F971C091F4
:10BF0000F00DD091F10DC93E83E0D80754F01092A6
:10BF1000F20D90DF2DEA3FE548EE53E060E070E07F
:10BF200007C024E33FE5AE010D2E000C660B770B36
:10BF30008CE89AE00E943C4C9093ED0D8093EC0DC0
:10BF40008091EE0D9091EF0D8C0F9D1F9093F10D50
:10BF50008093F00DDF91CF910895CF93DF9380917F
:10BF60005F06882319F0DF91CF917ECFC091EC0D51
:10BF7000D091ED0DBE018CE89AE00E94D54B88234C
:10BF800029F0BE018CE89AE00E94ED4BDF91CF9141
:10BF900051CF80910602813019F485E0809306022A
:10BFA00008951092520608958091070181FF12C0F2
:10BFB00060E08FE30E9478451092ED0580915C0669
:10BFC000882341F062EA73E180915A0690915B0602
:10BFD0000C94714308958091070181FF13C061E0C3
:10BFE0008FE30E94784581E08093ED0580915C06A7
:10BFF000882341F06CE873E180915A0690915B06CA
:10C000000C94714308958091BA05882371F01092C1
:10C01000BA0580915C06882341F064E073E1809169
:10C020005A0690915B060C94714308958091ED0F30
:10C03000833099F08091BA0581110FC081E080931F
:10C04000BA0580915C06882341F06FEE72E1809121
:10C050005A0690915B060C94714308958091BA053D
:10C06000882319F080E090E0CECF80E090E0DECF32
:10C070008091B905833079F083E08093B905809190
:10C080005C06882341F06EED72E180915A06909132
:10C090005B060C94714308958091B905823079F064
:10C0A00082E08093B90580915C06882341F06DECB5
:10C0B00072E180915A0690915B060C947143089549
:10C0C0008091B905813079F081E08093B905809144
:10C0D0005C06882341F06CEB72E180915A069091E6
:10C0E0005B060C947143089556D98091BB05882353
:10C0F00061F18091610A811128C0809153068111FC
:10C1000024C081E0809353060E94537B8091E60512
:10C11000882319F01092E6050CC080915606909184
:10C120005706DC01ED91FC910088F189E02D61E07A
:10C13000199580915C06882341F061E972E1809154
:10C140005A0690915B060C947143089590915C0699
:10C150008823D9F08091B8068823B9F081E08093D4
:10C16000FF0F8093F60D992311F16BE573E1809138
:10C170005A0690915B060E9400420E94778C809143
:10C180005A0690915B060C945E431092FF0F992320
:10C1900041F063E773E180915A0690915B060E943B
:10C1A00071438091FD0F811102C01092F60D089528
:10C1B00090915C068823F9F08091B8068823D9F025
:10C1C0008091B30F8D30B9F481E08093FD0F80939F
:10C1D000F60D992311F16AE173E180915A0690916D
:10C1E0005B060E9400420E94A58C80915A069091A5
:10C1F0005B060C945E431092FD0F992341F06AE3B5
:10C2000073E180915A0690915B060E947143809180
:10C21000FF0F811102C01092F60D08958091ED0F6D
:10C220008230C1F01CF48130A9F02FC0833011F1AD
:10C23000843059F580914C0690914D06DC01ED91CA
:10C24000FC910480F581E02D199580914A0690912A
:10C250004B0614C08091500690915106DC01ED917F
:10C26000FC910480F581E02D199580914E06909106
:10C270004F0604C080914C0690914D06DC01ED9173
:10C28000FC910480F581E02D1995809156069091DE
:10C290005706DC01ED91FC91E05CFF4F0190F081CD
:10C2A000E02D19958091560690915706DC01ED918D
:10C2B000FC910284F385E02D60E070E019946BD866
:10C2C0008091BB05882341F180915306811101C003
:10C2D0000895109253060E94217B8091E6058823E1
:10C2E00019F01092E6050CC0809156069091570601
:10C2F000DC01ED91FC910088F189E02D60E0199559
:10C3000080915C06882341F065EA72E180915A06CB
:10C3100090915B060C9471430895CF93DF93C09185
:10C32000030ED091040EBE018CE89AE00E94D54B1A
:10C33000882329F0BE018CE89AE00E94ED4B109210
:10C34000040E1092030EDF91CF9108950F931F9367
:10C35000CF93DF938091F20F9091F30FA091F40FA0
:10C36000B091F50F181619061A061B060CF043C0FB
:10C3700012D88091BB058823C9F10091030E10915A
:10C38000040EB8018CE89AE00E94D54B8823D9F0BE
:10C39000EAE8FCE0C0E0D0E081919191801791073C
:10C3A00069F40E942647CC0FDD1FCC0FDD1FC45758
:10C3B000D54F688379838A839B831DC02196CE31B4
:10C3C000D10551F718C04091F20F5091F30F6091D1
:10C3D000F40F7091F50F20E832E68CE89AE00E94A5
:10C3E0003C4C9093040E8093030E05C0DF91CF91D7
:10C3F0001F910F9192CFDF91CF911F910F910895CF
:10C400008091610A811136C00E94CB598091C60D7E
:10C410008823B1F08091BB05882391F01092BB0571
:10C420001092C60D0E94AF8B8091F50D882341F0CC
:10C430006CE672E18091F30D9091F40D0E947143CE
:10C4400080915306882311F081E001C080E00E94B2
:10C45000857B81E08093E60532DF809156069091DE
:10C460005706DC01ED91FC910480F581E02D1995D2
:10C47000D5DE6CCF0895D2DE809156069091570696
:10C48000DC01ED91FC910084F185E02D19958091FE
:10C49000560690915706DC01ED91FC910480F581E0
:10C4A000E02D19950E9443710E94CB598091BB05E4
:10C4B0008111A6DF8091580690915906DC01ED911B
:10C4C000FC910480F581E02D19958091540690919E
:10C4D0005506DC01ED91FC910480F581E02D199564
:10C4E0008091CE0F882359F08091E4059091E50565
:10C4F000DC01ED91FC910480F581E02D1994089503
:10C500000E94CB598091BB05882369F079DF809127
:10C510005C06882341F06CE772E180915A069091A5
:10C520005B060C94714308958091610A811142C0A9
:10C530000E94CB598091C60D8823E1F18091BB0503
:10C54000811138C081E08093BB051092C60D0E9416
:10C55000AF8B8091F50D882341F06DE572E18091FC
:10C56000F30D9091F40D0E947143809156069091C5
:10C570005706DC01ED91FC910280F381E02D1995C5
:10C580004091E80F5091E90F4115510571F081E09C
:10C590008093E60560E070E024E730E68CE89AE0FE
:10C5A0000E943C4C0E94217B04C081E08093E60500
:10C5B0009BDDCCCE0895CF93823069F49091E10F4A
:10C5C0002091DE0F3091E20F4091DF0F5091E00F8C
:10C5D0006091DD0F0CC09091DB0F2091D80F30914E
:10C5E000DC0F4091D90F5091DA0F6091D70F609313
:10C5F0007B125093781240937912309377122093E4
:10C600007A1290937C12909100028917B9F080936E
:10C61000000290915C06992389F0C82F64E472E1CE
:10C6200080915A0690915B060E9400426C2F809187
:10C630005A0690915B06CF910C94BA7ECF910895E3
:10C64000833079F030F4813051F0823091F48BE313
:10C650000BC0843041F0853061F482E405C08CE386
:10C6600003C080E401C081E40E94504521E0892B91
:10C6700009F420E0822F0895E3DF91E089270895EF
:10C680000F931F938091FB0D81110DC00E942647CF
:10C690006093F70D7093F80D8093F90D9093FA0D58
:10C6A00081E08093FB0D809109028A3AF1F485E0E4
:10C6B000C7DF882371F083EF97E090930C0E80938F
:10C6C0000B0E90935B0680935A068FEF80930902BE
:10C6D0000CC080E998E090930C0E80930B0E909321
:10C6E0005B0680935A06109209020E942647009129
:10C6F000F70D1091F80D2091F90D3091FA0DDC0134
:10C70000CB01801B910BA20BB30BC397A105B10505
:10C7100008F449C00E9426476093F70D7093F80D06
:10C720008093F90D9093FA0D85E08ADF882321F03C
:10C7300080910902882349F085E082DF811133C0AE
:10C74000809109028F3F79F518C083EF97E09093AD
:10C750000C0E80930B0E90935B0680935A0680918B
:10C760005C06882331F06AE272E183EF97E00E9471
:10C7700071438FEF8093090216C080E998E090938F
:10C780000C0E80930B0E90935B0680935A0680915B
:10C790005C06882331F065E172E180E998E00E944F
:10C7A0007143109209021F910F91089510923E0E4D
:10C7B00080915C06882379F02091C00F80915A0601
:10C7C00090915B06222319F065EE71E102C068EFDB
:10C7D00071E10C94714308950C9453730C946A7333
:10C7E00080910A0E882319F00E94537302C00E94A0
:10C7F0006A7390910A0E81E0892780930A0E08954A
:10C80000D3CBE9CB8091090E882311F0CDDB01C099
:10C81000E2DB9091090E81E089278093090E08954B
:10C820000C9497720C94D2728091080E882319F0A0
:10C830000E94977202C00E94D2729091080E81E00D
:10C8400089278093080E08950C94C57B809101027E
:10C8500081110C94A97B0C94C57B0C94A97B8091CD
:10C860000002813011F482E001C081E0A4CE82E0B8
:10C87000A2CE81E0A0CE0C94AB2080915C068823F0
:10C8800041F069EF74E180915A0690915B060C9437
:10C890007143089580915C06882341F069EE74E14C
:10C8A00080915A0690915B060C9471430895909183
:10C8B000FF0F81E089274ACC80E048CC81E046CC5C
:10C8C0009091FD0F81E0892773CC80E071CC81E0ED
:10C8D0006FCC8091F605882329F00E9453732AE6D5
:10C8E00033E704C00E946A7323E533E74CE251E06A
:10C8F00060E070E08CE89AE00C943C4C8091EF058D
:10C90000882321F051DB2BEE3FE503C064DB24EDEF
:10C910003FE54CE251E060E070E08CE89AE00C9476
:10C920003C4C0E949772409150105091511060E021
:10C9300070E022ED32E78CE89AE00E943C4C909344
:10C9400099128093981280915C06882341F062EEE0
:10C9500073E180915A0690915B060C94714308959F
:10C960000E94D272409150105091511060E070E0DE
:10C9700027E932E78CE89AE00E943C4C90939912A8
:10C980008093981280915C06882341F06FEC73E1EC
:10C9900080915A0690915B060C94714308958091A2
:10C9A000560690915706DC01ED91FC9104ACF5AD73
:10C9B000E02D66E0199580915C06882351F00E9475
:10C9C000017B60EE74E180915A0690915B060C94B5
:10C9D000714308958091560690915706DC01ED91C0
:10C9E000FC9102ACF3ADE02D66E0199580915C06F8
:10C9F000882351F00E94017B6CEC74E180915A060F
:10CA000090915B060C947143089580915606909125
:10CA10005706DC01ED91FC9100ACF1ADE02D66E034
:10CA2000199580915C06882351F00E94017B6AEC85
:10CA300074E180915A0690915B060C9471430895BD
:10CA40008091560690915706DC01ED91FC9104AC63
:10CA5000F5ADE02D65E0199580915C06882351F0D5
:10CA60000E94017B61EC74E180915A0690915B0613
:10CA70000C94714308958091560690915706DC01FD
:10CA8000ED91FC9102ACF3ADE02D65E0199580913C
:10CA90005C06882351F00E94017B6DEA74E180916D
:10CAA0005A0690915B060C94714308958091560646
:10CAB00090915706DC01ED91FC9100ACF1ADE02DB9
:10CAC00065E0199580915C06882351F00E94017BF6
:10CAD0006BEA74E180915A0690915B060C94714365
:10CAE00008958091560690915706DC01ED91FC91D6
:10CAF00004ACF5ADE02D64E0199580915C068823C7
:10CB000051F00E94017B62EA74E180915A06909193
:10CB10005B060C94714308958091560690915706D8
:10CB2000DC01ED91FC9102ACF3ADE02D64E01995D0
:10CB300080915C06882351F00E94017B6EE874E1CD
:10CB400080915A0690915B060C94714308958091F0
:10CB5000560690915706DC01ED91FC9100ACF1ADC9
:10CB6000E02D64E0199580915C06882351F00E94C5
:10CB7000017B6CE874E180915A0690915B060C94FD
:10CB8000714308958091560690915706DC01ED910E
:10CB9000FC9104ACF5ADE02D63E0199580915C0645
:10CBA000882351F00E94017B63E874E180915A066A
:10CBB00090915B060C947143089580915606909174
:10CBC0005706DC01ED91FC9102ACF3ADE02D63E082
:10CBD000199580915C06882351F00E94017B6FE6D5
:10CBE00074E180915A0690915B060C94714308950C
:10CBF0008091560690915706DC01ED91FC9100ACB6
:10CC0000F1ADE02D63E0199580915C06882351F029
:10CC10000E94017B6DE674E180915A0690915B065B
:10CC20000C94714308958091560690915706DC014B
:10CC3000ED91FC9104ACF5ADE02D62E01995809189
:10CC40005C06882351F00E94017B64E674E18091C8
:10CC50005A0690915B060C94714308958091560694
:10CC600090915706DC01ED91FC9102ACF3ADE02D03
:10CC700062E0199580915C06882351F00E94017B47
:10CC800060E574E180915A0690915B060C947143C3
:10CC900008958091560690915706DC01ED91FC9124
:10CCA00000ACF1ADE02D62E0199580915C0688231F
:10CCB00051F00E94017B6EE474E180915A069091DC
:10CCC0005B060C9471430895809156069091570627
:10CCD000DC01ED91FC9104ACF5ADE02D61E019951E
:10CCE00080915C06882351F00E94017B65E474E129
:10CCF00080915A0690915B060C947143089580913F
:10CD0000560690915706DC01ED91FC9102ACF3AD13
:10CD1000E02D61E0199580915C06882351F00E9416
:10CD2000017B61E374E180915A0690915B060C945B
:10CD3000714308958091560690915706DC01ED915C
:10CD4000FC9100ACF1ADE02D61E0199580915C069D
:10CD5000882351F00E94017B6FE274E180915A06B2
:10CD600090915B060C94714308950C94097B0C948C
:10CD7000157BCF93DF9380919712882321F1109236
:10CD8000971260E088E00E947845C0919812D09197
:10CD90009912BE018CE89AE00E94D54B882329F0B5
:10CDA000BE018CE89AE00E94ED4B80915C068823DE
:10CDB00071F066E174E180915A0690915B06DF9113
:10CDC000CF910C947143DF91CF910C94358CDF910E
:10CDD000CF91089580919712811102C00C94358CE7
:10CDE0000895CF93DF9380919A12882311F10E94C6
:10CDF000977210929A12C0919812D0919912BE0116
:10CE00008CE89AE00E94D54B882329F0BE018CE87B
:10CE10009AE00E94ED4B80915C06882371F06DEFE3
:10CE200073E180915A0690915B06DF91CF910C944B
:10CE30007143DF91CF910C94E772DF91CF91089508
:10CE40000C94E7726091561070E088E00E94E34510
:10CE500080915C06882341F069EB73E180915A066A
:10CE600090915B060C94714308950C943E740C945D
:10CE700055748091070E882319F00E943E7402C0F9
:10CE80000E9455749091070E81E089278093070EC8
:10CE900008950C947F740C94AD748091060E8823D1
:10CEA00019F00E947F7402C00E94AD749091060E2A
:10CEB00081E089278093060E08950C94BE740C942B
:10CEC000DA748091050E882319F00E94BE7402C0A6
:10CED0000E94DA749091050E81E089278093050EF7
:10CEE0000895CF9380913A0EC0910A02811101C139
:10CEF000C23009F450C0C33009F49DC0C13009F0FC
:10CF000028C18091700A811124C181E090E00E94C3
:10CF1000B9A89093710D8093700D62E083E00E9438
:10CF2000A7451092390E10926A0D1092690D109259
:10CF30006E0D80E090E0FC01EE0FFF1FE95DF14F08
:10CF400011821082019688309105A9F71092380E4F
:10CF50001092370E80916A008C6080936A00ED9A7F
:10CF60008FB7F89420918400309185003093260E7D
:10CF70002093250E8FBF25EB3EE44AEF50E060E0A2
:10CF800070E08091670D9091680D0E943C4C81E0AB
:10CF900080933A0EDEC080916F0A8111DAC081E081
:10CFA00090E00E94B9A89093730D8093720D8091C8
:10CFB00004018E7F8093040180910501816080933C
:10CFC000050189EB96E090939D0D80939C0D2EE2D8
:10CFD00040EA56E861E070E00E94EB448091650011
:10CFE0008B7F809365001092350189E08093340136
:10CFF0008EE2809332018CEF8093300180E9809340
:10D00000310110929B0D10929A0D1092990D109271
:10D01000980D1092960DE6E7FDE08CED95E081937A
:10D0200091932DE0E639F207D1F7C1E0C093970D57
:10D0300021EB3EE451C080916E0A81118AC081E0EB
:10D0400090E00E94B9A89093750D8093740D809123
:10D0500004018E7F8093040180910501816080939B
:10D06000050189EB96E09093170E8093160E26E04B
:10D0700040E052EC61E070E00E94EB44809165007A
:10D080008B7F809365001092350180E1809334019D
:10D0900086E0809332018EEF8093300180E98093A7
:10D0A000310110926C0D10926B0D1092150E1092B2
:10D0B000140E10926D0DEBE4FDE08CED95E0819384
:10D0C00091932DE0E736F207D1F71092130EC1E0ED
:10D0D000C093120E2DEA3EE44AEF50E060E070E0AB
:10D0E0008091670D9091680D0E943C4CC0933A0E60
:10D0F00030C0C23069F0C330D1F0C13051F58091F9
:10D10000700A811126C08091690D90916A0D1DC031
:10D1100080916F0A81111DC08091720D9091730DE5
:10D120000E948D5180919A0D90919B0D0EC080911F
:10D130006E0A81110EC08091740D9091750D0E9440
:10D14000CA5580916B0D90916C0D029711F4C093AC
:10D15000770A80910A028230A1F1833009F454C029
:10D16000813009F074C08091700A882309F46FC07F
:10D17000ED98E59A1092390E10926F0D10926A0D8B
:10D180001092690D10926E0D80E090E0FC01EE0FA0
:10D19000FF1FE95DF14F11821082019688309105E1
:10D1A000A9F71092380E1092370E8091700D909161
:10D1B000710D0E944EA910923A0E10926F0A82E0F1
:10D1C00044C080916F0A882309F441C080919C0D6E
:10D1D00090919D0D0E94C944809131018F77809379
:10D1E0003101809131018F7E8093310110923001A5
:10D1F0008091720D9091730D0E944EA910923A0E7B
:10D2000010926E0A83E021C080916E0A8823F9F0A3
:10D210008091160E9091170E0E94C94480913101A1
:10D220008F7780933101809131018F7E809331011E
:10D23000109230018091740D9091750D0E944EA94D
:10D2400010923A0E1092700A81E080930A02809147
:10D25000670D9091680DCF910C944C4CAF92BF929A
:10D26000CF92DF92EF92FF920F931F93CF93DF93B2
:10D270007C016B015A01D0E0C0E08D2F90E0F701F6
:10D28000A181B2818A159B05D0F4F601E80FF91F40
:10D29000608108EE13E721E03327C6270C0F111D2C
:10D2A000211D311D2BBFF801C791ED91FC91119704
:10D2B0000190F081E02DCD011995DF5FDECFED917A
:10D2C000FC9111970190F081E02D6C2FCD01DF9141
:10D2D000CF911F910F91FF90EF90DF90CF90BF9073
:10D2E000AF901994CF93DF9300D01F921F92CDB7C8
:10D2F000DEB7FE01319625E0DF011D922A95E9F7A0
:10D3000024E8298325E52C832AE22D836A834B8335
:10D3100045E050E0BF01A2DF65E070E080E090E012
:10D320000E94EE4680E00F900F900F900F900F90AC
:10D33000DF91CF910895EF92FF921F93CF93DF93E8
:10D340001F92CDB7DEB77C01162FFC01618172817F
:10D350000E94447F65E070E080E090E00E94EE462D
:10D3600042E462E4C701BEDF412F60E0C701BADFDB
:10D37000811163C040E061E0C701B4DF81115DC08D
:10D3800040E062E0C701AEDF811157C046E062E0D5
:10D39000C701A8DF811151C040E063E0C701A2DFEF
:10D3A00081114BC040E064E0C7019CDF11E08111B6
:10D3B00010E040E065E0C70195DF811101C01F5F0B
:10D3C00040E066E0C7018EDF811101C01F5F40E0D1
:10D3D00067E0C70187DF811101C01F5F40E068E09F
:10D3E000C70180DF811101C01F5F40E069E0C70114
:10D3F00079DF811101C01F5F44E06AE0C70172DF7D
:10D40000811101C01F5F44E06AE0C7016BDF811139
:10D4100001C01F5F62E370E080E090E00E94EE4692
:10D4200082E8898341E050E0BE016F5F7F4FC70112
:10D4300015DF81E0183011F0111180E00F90DF91BD
:10D44000CF911F91FF90EF900895CF93DF9300D07D
:10D450001F92CDB7DEB72AEA2983FC0120812A83F7
:10D460006B834C8344E050E0BE016F5F7F4FF6DE7C
:10D470000F900F900F900F90DF91CF9108953FB7CD
:10D48000F89420E0822F90E0841795079CF4FC012B
:10D49000EE0FFF1FE75DF14FA081B181880F991F4B
:10D4A000FB01E80FF91FCD01969587959183808345
:10D4B0002F5FE8CF3FBF10926E0D08951F920F921D
:10D4C0000FB60F9211240BB60F922F933F934F93E9
:10D4D0008F939F93EF93FF938091840090918500A9
:10D4E0002091250E3091260E821B930B20918400F3
:10D4F000309185003093260E2093250E803727E14A
:10D50000920770F19093280E8093270E8091690DF9
:10D5100090916A0D029751F49091390E80916F0DA0
:10D5200098133CC081E080936E0D3EC08091690DE0
:10D5300090916A0D892B49F481E090E090936A0DF7
:10D540008093690D1092240E2FC08091690D9091E7
:10D550006A0D019761F58091390E8430D8F527C0A6
:10D560002091390E283008F047C09C012C5D3540D1
:10D57000293B3B4068F4E091390EEF5FE093390EB0
:10D58000F0E0EE0FFF1FE95DF14F9183808334C01F
:10D590008091690D90916A0D029771F583E090E09A
:10D5A00090936A0D8093690D1092390E25C0809179
:10D5B000690D90916A0D0397B9F79091390E80919A
:10D5C0006F0D9813F1CF80916F0D843068F382E076
:10D5D00090E0E6CF8091240E8F5F8093240E8630FA
:10D5E00018F382E090E090936A0D8093690D80912A
:10D5F000390E80936F0DD8CFFF91EF919F918F914E
:10D600004F913F912F910F900BBE0F900FBE0F9037
:10D610001F9018950F931F9380911C0E81110DC0C0
:10D620000E9426476093180E7093190E80931A0E6D
:10D6300090931B0E81E080931C0E0E942647009160
:10D64000180E1091190E20911A0E30911B0EDC014C
:10D65000CB01801B910BA20BB30B893E9340A1051C
:10D66000B105A8F08AE30E945045892B11F060E0D3
:10D6700001C061E08AE30E9478450E9426476093DA
:10D68000180E7093190E80931A0E90931B0E1F9113
:10D690000F9108950F931F930E94264700910E0E3D
:10D6A00010910F0E2091100E3091110EDC01CB0164
:10D6B000801B910BA20BB30B85339142A105B105E1
:10D6C00018F081E080930D0E1F910F91A3CFFC0104
:10D6D00080E090E06150710977FD18C02191022E21
:10D6E000000C330B322F22278227932728E0AC012E
:10D6F000440F551F97FF06C0CA0131E2832730E16E
:10D70000932701C0CA01215091F7E4CF0895BF9239
:10D71000CF92DF92EF92FF920F931F93CF93DF93FD
:10D72000CDB7DEB76E970FB6F894DEBF0FBECDBF94
:10D73000B62EC72ED82E7A01FA011082F801108277
:10D7400061EB75E0CE0142962E8F0E94C141198E89
:10D75000188E1B8E1A8E1D8E1C8E4AE0BE016F5FC6
:10D760007F4F8B2D90E00E9490ABBE016F5F7F4F8B
:10D77000CE0148960E947141BE01685E7F4FCE0186
:10D7800042960E94B740CE0148960E949141CE0138
:10D7900042960E940887198E188E1B8E1A8E1D8E37
:10D7A0001C8E4AE0BE016F5F7F4FC6010E9490ABA6
:10D7B000BE016F5F7F4FCE0148960E947141BE014E
:10D7C000685E7F4FCE0142960E941741CE01489677
:10D7D0000E949141CE0142960E9408878E89F801ED
:10D7E00080832E8D422F50E0B701CE0142960E94D9
:10D7F0000087CE0142960E9491416E960FB6F89432
:10D80000DEBF0FBECDBFDF91CF911F910F91FF9073
:10D81000EF90DF90CF90BF900895FF920F931F93EA
:10D82000CF93DF93CDB7DEB7C154D1090FB6F894CB
:10D83000DEBF0FBECDBFF62E8E010F5B1F4F20E463
:10D84000AE014F5F5F4F682F782F80E060DF229638
:10D850008FAD229791E0980F22969FAF2297E1E03B
:10D86000F0E0EC0FFD1FE80FF11DFF2011F081E348
:10D8700001C080E3808322969FAD229781E0890FCB
:10D8800022968FAF2297E1E0F0E0EC0FFD1FE90F49
:10D89000F11D9CE79083E1E0F0E0EC0FFD1FE80F45
:10D8A000F11D1082BE016F5F7F4F80910B0E909132
:10D8B0000C0E0E94244222966FAD229770E0CE019A
:10D8C000019605DFBC0180910B0E90910C0E0E9419
:10D8D000FE7F6AE080910B0E90910C0E0E94F94140
:10D8E00080910B0E90910C0EDC01ED91FC91028465
:10D8F000F385E02D1995CF5BDF4F0FB6F894DEBFAF
:10D900000FBECDBFDF91CF911F910F91FF90089572
:10D9100060E085E882CF80910B02882311F0729835
:10D9200001C0729A90910B0281E0892780930B02CB
:10D93000089581E08093630A08951092E3051092A0
:10D94000CF051092C2051092CB051092CC05109213
:10D95000CD051092CE0581E080935F0A4091D305FA
:10D960005091D40560E070E02CEB3CE68091C3055B
:10D970009091C4050C943C4C80919A0981111CC073
:10D980001092AB091092AC091092AD091092AE0939
:10D990001092AF091092B0091092B30980915D0AFC
:10D9A00090915E0ADC01ED91FC910190F081E02DF7
:10D9B000199510925F0A08952CEB3CE645E050E083
:10D9C00060E070E08091C3059091C4050C943C4CDC
:10D9D00060914A0E70914B0E8091C3059091C405E1
:10D9E0000E94D54B882319F081E08093490E089559
:10D9F00060E087E00E9478451092600A089561E037
:10DA000087E00E94784581E08093600A0895CF9373
:10DA1000DF938091570E811110C084EF91E09093B5
:10DA2000560E8093550E8BE290E09093540E8093A7
:10DA3000530E81E08093570E20C08091530E909139
:10DA4000540E8532910514F0049709C08331910575
:10DA500014F0029704C0823091052CF00197909346
:10DA6000540E8093530E8091530E9091540E97FF55
:10DA700004C01092540E1092530EC091520ECC233B
:10DA800011F0B6DF01C0BBDF81E08C278093520E1E
:10DA9000C091550ED091560E1C161D0654F01092D2
:10DAA000570EA6DF27E73DE64AEF50E060E070E062
:10DAB00007C027E03DE6AE010D2E000C660B770B8C
:10DAC0008091C3059091C4050E943C4C9093510EE7
:10DAD0008093500E8091530E9091540EC81BD90B19
:10DAE000D093560EC093550EDF91CF9108950F93AA
:10DAF0001F93CF93DF938091610A882329F0DF91F0
:10DB0000CF911F910F9183CF0091500E1091510E24
:10DB1000C091C305D091C405B801CE010E94D54B78
:10DB2000882321F0B801CE010E94ED4BDF91CF9107
:10DB30001F910F915DCFCF92DF92EF92FF921092E3
:10DB4000610A2091C7053091C8054091C9055091DF
:10DB5000CA056091CB057091CC058091CD0590915F
:10DB6000CE050E94B3A76B017C0120E030E0A90143
:10DB70000E94B9AB87FD09C0C092CB05D092CC05FD
:10DB8000E092CD05F092CE0508C01092CB05109220
:10DB9000CC051092CD051092CE05FF90EF90DF904E
:10DBA000CF90A5CF0F931F93CF93DF9380914F0E0C
:10DBB0009091E30581112AC0992309F456C0009180
:10DBC0004D0E10914E0EC091C305D091C405B80101
:10DBD000CE010E94D54B882321F0B801CE010E94CE
:10DBE000ED4B0DDF22ED3DE642EC51E060E070E0F0
:10DBF0008091C3059091C4050E94444C90934E0EB1
:10DC000080934D0E81E080934F0E5AC08091600A40
:10DC1000992361F0882329F0DF91CF911F910F9113
:10DC2000E7CEDF91CF911F910F91E9CE8823C9F301
:10DC300060914D0E70914E0E8091C3059091C40578
:10DC40000E94ED4B22ED3DE644E150E060E070E0E3
:10DC50008091C3059091C4050E94444C90934E0E50
:10DC600080934D0E10924F0E2BC0C0910C02D0919C
:10DC70000D022297D0930D02C0930C021C161D06B4
:10DC800074F4BE01772787E00E94E345CC2321F09E
:10DC900081E08093600A14C01092600A11C0609104
:10DCA0004D0E70914E0E8091C3059091C4050E9457
:10DCB000ED4B9EDE8FEF90E090930D0280930C026F
:10DCC000DF91CF911F910F9108950F931F93CF93E1
:10DCD000DF930091450E1091460EC091470ED091F2
:10DCE000480EC00FD11FD093480EC093470EBE01FF
:10DCF000772787E00E94E345CC2321F081E08093E1
:10DD0000600A02C01092600A10161106ECF58091AC
:10DD1000430E9091440EC817D9070CF485C080912A
:10DD2000490E882371F01092440E1092430E8CEF2E
:10DD30009FEF9093460E8093450E81E08093420EB4
:10DD400073C068E770E080E090E00E94D541DC019C
:10DD5000CB010A96A11DB11D9093440E8093430EF2
:10DD600068E270E080E090E00E94D541DC01CB01E8
:10DD70000A96A11DB11D66277727681B790B709342
:10DD8000460E6093450E50C0012B09F44DC08091A2
:10DD9000430E9091440E8C179D070CF445C0809162
:10DDA000420E882311F100914A0E10914B0EC09142
:10DDB000C305D091C405B801CE010E94D54B88237C
:10DDC00099F1B801CE010E94ED4B12DE1092480E7F
:10DDD0001092470E1092420E8091E305882321F1A4
:10DDE000DF91CF911F910F91DDCE69E670E080E069
:10DDF00090E00E94D541DC01CB018A569F4FAF4F86
:10DE0000BF4F9093440E8093430E68E270E080E031
:10DE100090E00E94D541DC01CB010A96A11DB11D05
:10DE20009093460E8093450EDF91CF911F910F91F5
:10DE30000895EF92FF921F93CF93DF9300D0CDB759
:10DE4000DEB784E689838CE38A8388E28B83109132
:10DE50004C0E1330E8F4E12EF12C10FF02C0C8DDA7
:10DE600001C0CDDDE1E0F0E0EC0FFD1FEE0DFF1D88
:10DE7000408150E060E070E029E13FE68091C30519
:10DE80009091C4050E943C4C1F5F10934C0E03C040
:10DE9000AFDD10924C0E0F900F900F90DF91CF914D
:10DEA0001F91FF90EF90089560E088E00C94784512
:10DEB00061E089E20C9478450F931F93CF93DF9331
:10DEC00060E08BE20E9478450091400E1091410E77
:10DED000C091C305D091C405B801CE010E94D54BB5
:10DEE000882341F0B801CE01DF91CF911F910F91AE
:10DEF0000C94ED4BDF91CF911F910F91089581E02C
:10DF000080935F0A8091DB050E945D7C35CD1F9276
:10DF10000F920FB60F9211242F933F938F939F93DD
:10DF2000AF93BF938091380D9091390DA0913A0D28
:10DF3000B0913B0D3091580E23E0230F2D3720F484
:10DF40000196A11DB11D05C026E8230F0296A11D53
:10DF5000B11D2093580E8093380D9093390DA093E6
:10DF60003A0DB0933B0D80913C0D90913D0DA091E9
:10DF70003E0DB0913F0D0196A11DB11D80933C0D4A
:10DF800090933D0DA0933E0DB0933F0DBF91AF9187
:10DF90009F918F913F912F910F900FBE0F901F90E7
:10DFA00018950F931F93CF93DF930091500E10910C
:10DFB000510EC091C305D091C405B801CE010E9495
:10DFC000D54B8823A1F0B801CE010E94ED4B28EE7D
:10DFD0003CE648EB5BE060E070E08091C305909127
:10DFE000C4050E943C4C9093510E8093500E60915A
:10DFF0004A0E70914B0E8091C3059091C4050E940A
:10E00000D54B81114BC01092490E8FEF90E0909349
:10E01000480E8093470EF3DC68E770E080E090E004
:10E020000E94D541DC01CB010A96A11DB11D909340
:10E03000440E8093430E68E270E080E090E00E941E
:10E04000D541DC01CB010A96A11DB11D66277727BA
:10E05000681B790B7093460E6093450E25E63EE6ED
:10E0600044E150E060E070E08091C3059091C40508
:10E070000E94444C90934B0E80934A0E28EE3CE64F
:10E0800048EB5BE060E070E08091C3059091C405CF
:10E090000E943C4C9093510E8093500EDF91CF9193
:10E0A0001F910F9108958F929F92AF92BF92CF923E
:10E0B000EF92FF920F931F93CF93DF932091DE0592
:10E0C000223008F07AC07B018C018090CB059090C3
:10E0D000CC05A090CD05B090CE0520E030E0A901A0
:10E0E000C501B4010E94B9AB181654F520E030E028
:10E0F000A901C501B4010E94B1A8181654F420E08A
:10E1000030E048E452E4C501B4010E94B9AB1816EE
:10E11000D4F420E030E048E452E4C501B4010E94A8
:10E12000B1A818169CF420E030E048EC52E4C50198
:10E13000B4010E94B9AB87FF09C0CBE4D0E008C0AE
:10E14000C0E0D0E005C0C2E3D0E002C0C4E6D0E049
:10E150008FEF8C0D823070F4209739F06C2FC8014E
:10E160000E94983A6C2FC7010DC0C8010E94EF862B
:10E17000C70116C08DEF8C0D8230F8F4209779F02E
:10E180006C2FC801DF91CF911F910F91FF90EF90FD
:10E19000CF90BF90AF909F908F900C94983AC80109
:10E1A000DF91CF911F910F91FF90EF90CF90BF9093
:10E1B000AF909F908F900C94EF86DF91CF911F913D
:10E1C0000F91FF90EF90CF90BF90AF909F908F9066
:10E1D00008958F929F92AF92BF92CF92DF92EF926B
:10E1E000FF92C090CB05D090CC05E090CD05F0908B
:10E1F000CE0520E030E0A901C701B6010E94B1A818
:10E2000020E030E040E05FE387FD0BC0C701B601CE
:10E210000E94B4A74B015C010E9480A897FD27C013
:10E2200010C0C701B6010E94B3A70E9480A897FD45
:10E230001EC06536710581059105DCF424E6822F48
:10E2400014C0C501B4010E9480A86536710581051E
:10E2500091057CF420E030E040E05FE3C701B601C7
:10E260000E94B4A70E9480A884E6861B03C084E6AF
:10E2700001C080E0FF90EF90DF90CF90BF90AF9013
:10E280009F908F9008950F931F93CF93DF930091EA
:10E29000BC051091BD05C091C305D091C405B8015E
:10E2A000CE010E94D54B882321F0B801CE010E94F7
:10E2B000ED4B8091610A882339F01092610ADF9159
:10E2C000CF911F910F9113CCDF91CF911F910F919F
:10E2D000089560E089E20E94784528E53FE642E340
:10E2E00050E060E070E08091C3059091C4050C940B
:10E2F0003C4C1F920F920FB60F9211240BB60F9247
:10E300002F933F934F935F936F937F938F939F933D
:10E31000AF93BF93EF93FF9380913F0E8823A9F0B3
:10E32000669917C0EE98C8DD80913E0E882389F06B
:10E3300080913D0E882339F0E0913B0EF0913C0E28
:10E3400082810E94494FF1D404C0669B02C0EE98BE
:10E35000B3DDFF91EF91BF91AF919F918F917F912D
:10E360006F915F914F913F912F910F900BBE0F9046
:10E370000FBE0F901F90189561E08BE20E947845C8
:10E38000EE9A2CE53FE648E853E160E070E08091CA
:10E39000C3059091C4050E943C4C9093410E80931C
:10E3A000400E089561E08BE20E947845EE9A2CE5DC
:10E3B0003FE648E853E160E070E08091C30590914A
:10E3C000C4050E943C4C9093410E8093400E0895EA
:10E3D000CF93C09112026C2F89E30E94784581E0AF
:10E3E000C8276C2F8AE30E947845C0931202CF9110
:10E3F0000895CF93DF93C09111026C2F89E30E949F
:10E400007845D1E0DC276D2F8AE30E9478456C2F98
:10E4100085E30E9478456D2F85E00E9478456D2F39
:10E4200084E00E9478456C2F87E00E947845CC23D9
:10E4300011F0729801C0729A9091110281E08927BF
:10E4400080931102DF91CF910895CF93C091650E13
:10E450006C2F70E088E00E94E34589E18093640EB0
:10E4600090911002992311F0CD5F01C0C350C09369
:10E47000650E8091650E873970F0992321F08FEF3A
:10E480008093650E08C08D3D30F086E98093650E5F
:10E4900088E78093640E8091650E8F3F19F4109287
:10E4A000100205C08A3118F481E080931002409177
:10E4B000640E50E060E070E025E232E78CE89AE01C
:10E4C0000E943C4C9093991280939812CF9108959A
:10E4D000CF92DF92EF92FF92CF93DF93EC019C01FA
:10E4E000AFEFB0E00E9450ADCC24CA9423E0D22E0E
:10E4F000E12CF12CA70196010E9402ADB90188E040
:10E500000E94E3459E01A4E6B0E00E9450ADA70141
:10E5100096010E9402AD80915610821320935610EE
:10E52000DF91CF91FF90EF90DF90CF900895CF9340
:10E53000DF93C0919812D0919912BE018CE89AE0B5
:10E540000E94D54B882329F0BE018CE89AE00E94F6
:10E55000ED4B60E088E00E94784580915C0688235E
:10E56000D1F080919A12882319F060E176E10DC014
:10E5700080919712882319F067EF75E106C08091AA
:10E58000E90D811108C068EE75E180915A069091FD
:10E590005B060E94714310929A1210929712DF91BB
:10E5A000CF91089561E088E00E94784580915C06F3
:10E5B000882361F080919A12811108C06AED75E19B
:10E5C00080915A0690915B060C9471430895809156
:10E5D0009A12811110C0ABDF81E080939A12809172
:10E5E0005C06882341F069E276E180915A069091B9
:10E5F0005B060E9471438091630E882329F060E0DE
:10E6000088E00E94784501C0CDDF9091630E81E0E3
:10E6100089278093630E882329F0409152105091EE
:10E62000531004C0409154105091551060E070E0B8
:10E6300027EE32E78CE89AE00E943C4C90939912C6
:10E64000809398120895CF938091610E81110FC02D
:10E6500081E08093610E80915C06882341F068EA36
:10E6600075E180915A0690915B060E947143C091BA
:10E67000600E6C2F85E00E94784540915B1050E061
:10E6800060E070E023E233E78CE89AE00E943C4CC3
:10E6900090935F0E80935E0E81E06C2F68276093ED
:10E6A000600ECF9108958091070180FF12C060E055
:10E6B0008EE30E9478451092F40580915C068823D1
:10E6C00041F06FE175E180915A0690915B060C94E0
:10E6D000714308958091070180FF13C061E08EE3CC
:10E6E0000E94784581E08093F40580915C06882340
:10E6F00041F069E075E180915A0690915B060C94B7
:10E7000071430895CF93DF93C091660ED091670E49
:10E71000BE018CE89AE00E94D54B882369F0BE01C7
:10E720008CE89AE00E94ED4B1092670E1092660EF4
:10E73000DF91CF910C941A5FDF91CF910895609192
:10E74000660E7091670E8CE89AE00E94D54B81119D
:10E750002EC060E089E30E94784560E08AE30E9471
:10E76000784560E085E30E94784560E085E00E949E
:10E77000784560E084E00E94784560E087E00E9490
:10E780007845729880915810882319F029EF31E765
:10E7900002C028EE31E742E350E060E070E08CE830
:10E7A0009AE00E94444C9093670E8093660E089501
:10E7B00060E08AE30C94784561E08AE30C94784544
:10E7C0000F931F93CF93DF938C01C1E0D0E00C1720
:10E7D0001D079CF0F1DF64E670E080E090E00E94AD
:10E7E000EE46E6DFC017D10734F46AE570E080E05A
:10E7F00090E00E94EE462196EACFDF91CF911F91E3
:10E800000F91089583E090E0DBCF82E090E0D8CFD5
:10E8100081E090E0D5CF60E089E30C94784561E039
:10E8200089E30C9478450F931F93CF93DF938C016A
:10E83000C1E0D0E00C171D079CF0F1DF64E670E04A
:10E8400080E090E00E94EE46E6DFC017D10734F486
:10E850006AE570E080E090E00E94EE462196EACF03
:10E86000DF91CF911F910F91089583E090E0DBCF6E
:10E8700082E090E0D8CF81E090E0D5CF1092620E98
:10E8800080914906811104C060E084E00E947845CF
:10E8900080915C06882341F067EC75E180915A060F
:10E8A00090915B060C947143089581E08093620E11
:10E8B00080914906811106C06091590E70E084E094
:10E8C0000E94E34580915C06882341F065EB75E189
:10E8D00080915A0690915B060C94714308951092B2
:10E8E00049068091620E811104C060E084E00C94BE
:10E8F00078456091590E70E084E00C94E345CF9325
:10E90000DF9360E085E00E947845C0915E0ED09173
:10E910005F0EBE018CE89AE00E94D54B882329F057
:10E92000BE018CE89AE00E94ED4B80915C06882342
:10E9300079F02091610E80915A0690915B06222316
:10E9400019F06CE975E102C060E975E10E9471435C
:10E950001092610EDF91CF91089561E085E00E94F1
:10E96000784580915C06882341F065E875E18091E7
:10E970005A0690915B060C947143089560E085E31C
:10E980000E9478458091560690915706DC01ED91E2
:10E99000FC9104A8F5A9E02D199580915C068823C7
:10E9A00041F069E775E180915A0690915B060C94FD
:10E9B0007143089561E085E30E9478458091560691
:10E9C00090915706DC01ED91FC9104A8F5A9E02D8A
:10E9D000199580915C06882341F06EE675E180917F
:10E9E0005A0690915B060C94714308958F929F9202
:10E9F000AF92BF92CF92DF92EF92FF9285E40E9496
:10EA0000AA46BC01990F880B990B0E94BFAB20E06E
:10EA100030E040E85AE30E941EAC20E030E040EADB
:10EA200050E40E941EAC6B017C0180910F02882390
:10EA300051F0C0925A0ED0925B0EE0925C0EF092B2
:10EA40005D0E10920F0226E636E646E65FE3609121
:10EA50005A0E70915B0E80915C0E90915D0E0E943B
:10EA60001EAC4B015C0120ED3CEC4CEC5DE3C701BE
:10EA7000B6010E941EAC9B01AC01C501B4010E940D
:10EA8000B4A760935A0E70935B0E80935C0E9093C4
:10EA90005D0E2DE33CE248E450E40E941EAC2AE9FE
:10EAA00039E949E95EE30E94B4A7FF90EF90DF9057
:10EAB000CF90BF90AF909F908F90089580910E025D
:10EAC000882351F093DF20E030E040E050E40E94E2
:10EAD000B9AB87FF39C0089589DF20E030E04AE70D
:10EAE00054E40E941EAC0E9485A820914B103091E6
:10EAF0004C1040915F066217730710F4442351F1E4
:10EB0000442309F446C072DF20E030E04AE754E4D1
:10EB10000E941EAC0E9485A820914B1030914C1091
:10EB200062177307B0F110925F0681E080935E0672
:10EB300080915C06882369F166E375E180915A064D
:10EB400090915B060C94714310920E0281E08093C9
:10EB50005E06089581E080935F0610925E068091C4
:10EB60005C06882391F065E575E180915A069091E5
:10EB70005B060E9400420E94608C62E575E1809114
:10EB80005A0690915B060E9471430E943B620C946E
:10EB9000AD5F0895CF93DF938091070180FD2AC078
:10EBA000C091F105D091F2058091F605882371F0AE
:10EBB0008EE30E94AA46813092402CF01092F2051A
:10EBC0001092F1050AC081E090E003C08EE30E943C
:10EBD000AA469093F2058093F1058091F1059091FA
:10EBE000F2058C179D0719F41092F30503C081E01C
:10EBF0008093F305DF91CF910895CF93DF938091B8
:10EC0000070181FD2AC0C091EA05D091EB058091F2
:10EC1000EF05882371F08FE30E94AA46813092406D
:10EC20002CF01092EB051092EA050AC081E090E00A
:10EC300003C08FE30E94AA469093EB058093EA05F8
:10EC40008091EA059091EB058C179D0719F41092BD
:10EC5000EC0503C081E08093EC05DF91CF9108952E
:10EC60001092630A4091D1055091D20560E070E0A6
:10EC700029E93CE68091C3059091C4050C943C4C75
:10EC800081E20E94504521E0892B09F420E0822F87
:10EC900008958091D705882309F446C081E08093C8
:10ECA0005F0AEEDF882329F08091DA058823D1F10D
:10ECB00006C08091D805811104C08091D705FDD58B
:10ECC00031C09091D705963069F5823081F083305C
:10ECD000D1F0813039F5E091CE09F091CF097297EA
:10ECE0008081918145E550E060E070E017C0E091DF
:10ECF000CE09F091CF097297808191814AE550E069
:10ED000060E070E00BC0E091CE09F091CF097297FE
:10ED1000808191814FE550E060E070E08253964F32
:10ED20000E94783D0C94BC6C08958091C50590912B
:10ED3000C605DC01ED91FC910688F789E02D199557
:10ED400080918F0E8111C5DA80918E0E882391F00B
:10ED500061E088E00E94784540918C0E50918D0EC4
:10ED600060E070E024E53FE68091C3059091C40522
:10ED70000E943C4C80913F0E882321F080913E0EF2
:10ED8000811101C086DF80913E0E882379F0809149
:10ED90003F0E882359F080913D0E882339F0E09191
:10EDA0003B0EF0913C0E82810E94494F59CF8091D9
:10EDB000610A811156C064DF8823F1F081E08093FD
:10EDC000610A8091C5059091C605DC01ED91FC9129
:10EDD0000288F389E02D19950E94776D2BE93DE6B5
:10EDE00048E95AE360E070E08091C3059091C40562
:10EDF0000E943C4C35DF09C080913E0E882329F1EA
:10EE000080913F0E882311F0CDDA43CFB5DA80919F
:10EE10003D0E882339F0E0913B0EF0913C0E82814B
:10EE20000E94494F40918A0E50918B0E1416150680
:10EE3000BCF4052E000C660B770B25E936E78091B4
:10EE4000C3059091C4050C943C4C80913D0E8823E1
:10EE500039F0E0913B0EF0913C0E82810E94494FC7
:10EE600064CF089560ED77E081E00E94FB4E109240
:10EE7000890E26E638E444EF51E060E070E08091CE
:10EE8000870E9091880E0E943C4C9093860E809342
:10EE9000850E08950F931F9348EE54E761E077279E
:10EEA0009C01220F331F820F931F092E000CAA0B07
:10EEB000BB0B0296A11DB11D840F951FA61FB71F86
:10EEC000ABBFFC01879108EE14E721E033274091A6
:10EED0006C0E93E0499FA0011124052E000C660BD7
:10EEE000770B4E5F5F4F6F4F7F4F040F151F261F2D
:10EEF000371F2BBFF8010791801720F01F910F914A
:10EF00000C9454481F910F9108958F929F92AF9245
:10EF1000BF92CF92DF92EF92FF920F931F93CF9306
:10EF2000DF93EC01A62E48EE54E761E077276C01F1
:10EF3000CC0CDD1CCC0EDD1E0D2C000CEE08FF08E9
:10EF4000D701C6010296A11DB11D480F591F6A1FA6
:10EF50007B1F6BBFFA01879148EE54E761E077278A
:10EF6000B0906C0E93E0B99E80011124012E000C2C
:10EF7000220B330B0E5F1F4F2F4F3F4F400F511F80
:10EF8000621F731F6BBFFA014791481708F036C024
:10EF900080906A0E90906B0E0091870E1091880EF3
:10EFA000B401C8010E94D54B882321F0B401C801E7
:10EFB0000E94ED4B88EE94E7A1E0BB278C0D9D1DD0
:10EFC000AE1DBF1DABBFFC016791769182E00E9430
:10EFD000FB4EB092690EC0936C0EAA2079F010928D
:10EFE000680E24E538E442E350E060E070E0C801D8
:10EFF0000E943C4C90936B0E80936A0EDF91CF91F0
:10F000001F910F91FF90EF90DF90CF90BF90AF9046
:10F010009F908F900895CF92DF92EF92FF92809110
:10F02000840E882381F161E08EE090E06EDF6091D4
:10F03000820E7091830ECB01A0E0B0E0C090800EF4
:10F04000D090810EE12CF12CC816D906EA06FB06F9
:10F0500064F4BC01CD016C197D098E099F090E94E1
:10F06000D541C60ED71EE81EF91E2BE038E7B701C2
:10F07000A6018091870E9091880E0E943C4C90933F
:10F080007F0E80937E0EFF90EF90DF90CF900895DB
:10F09000CF92DF92EF92FF9280917D0E882381F1D3
:10F0A00061E08DE090E031DF60917B0E70917C0E2D
:10F0B000CB01A0E0B0E0C090790ED0907A0EE12CA8
:10F0C000F12CC816D906EA06FB0664F4BC01CD0192
:10F0D0006C197D098E099F090E94D541C60ED71E65
:10F0E000E81EF91E28E438E7B701A6018091870ED3
:10F0F0009091880E0E943C4C9093780E8093770EEE
:10F10000FF90EF90DF90CF900895CF92DF92EF9233
:10F11000FF928091760E882381F161E08CE090E08F
:10F12000F4DE6091740E7091750ECB01A0E0B0E03A
:10F13000C090720ED090730EE12CF12CC816D90637
:10F14000EA06FB0664F4BC01CD016C197D098E0949
:10F150009F090E94D541C60ED71EE81EF91E25E85C
:10F1600038E7B701A6018091870E9091880E0E9422
:10F170003C4C9093710E8093700EFF90EF90DF9057
:10F18000CF90089580916F0E882341F08091760E84
:10F19000811104C081E08093760EB7DF80916E0EFE
:10F1A000882341F080917D0E811104C081E080931D
:10F1B0007D0E6EDF80916D0E882341F08091840E6C
:10F1C000811104C081E08093840E25CF08950F93B0
:10F1D0001F93CF93DF932091CE0F21111BC0C091BD
:10F1E000E405D091E505088119819C01AFEFB0E0FD
:10F1F0000E9450AD2FEF33E040E050E00E9402AD9E
:10F20000D801ED91FC91B901CE01DF91CF911F9111
:10F210000F911994DF91CF911F910F9108950C9444
:10F22000D38C80913E0E81110C94D6630C94D38CB8
:10F230000C94D66364DB8091560690915706DC01EE
:10F24000ED91FC9104A0F5A1E02D1994FCD98091D9
:10F25000560690915706DC01ED91FC9102A0F3A1B6
:10F26000E02D19940F931F93CF93DF930091960E87
:10F270001091970EC091C305D091C405B801CE017D
:10F280000E94D54B882379F0B801CE010E94ED4B46
:10F290008091C5059091C605DC01ED91FC9100A01F
:10F2A000F1A1E02D19950091940E1091950EC09149
:10F2B000C305D091C405B801CE010E94D54B882367
:10F2C00021F0B801CE010E94ED4B729880915C064E
:10F2D000882361F068E277E180915A0690915B069D
:10F2E000DF91CF911F910F910C947143DF91CF91DA
:10F2F0001F910F910895CF93DF93C091C305D091D3
:10F30000C4056091960E7091970ECE010E94D54B68
:10F31000811129C04091920E50E060E070E02BE82E
:10F320003CE6CE010E94444C9093970E8093960E3B
:10F330008091C5059091C605DC01ED91FC91068C8C
:10F34000F78DE02D19958091DC05882361F060919F
:10F35000940E7091950E8091C3059091C4050E9402
:10F36000D54B882371F080915C068823E9F06FE12A
:10F3700077E180915A0690915B06DF91CF910C94D2
:10F3800071430E947F6F2FE73FE644E650E060E064
:10F3900070E08091C3059091C4050E94444C909305
:10F3A000950E8093940EDFCFDF91CF9108950E9448
:10F3B000697180915C06882341F064EF76E1809169
:10F3C0005A0690915B060C9471430895E091900E5B
:10F3D000F091910E82810E94494F80915C068823B2
:10F3E00041F066ED76E180915A0690915B060C94AF
:10F3F0007143089580913F0E882319F00E94D271C5
:10F4000002C00E94BC7180915C06882379F0209133
:10F41000C00F80915A0690915B06222319F06AE989
:10F4200076E102C063EB76E10C94714308950C948D
:10F430005F61CF938091630A882309F452C020DC76
:10F440009091610A882339F091114BC08091E705B2
:10F45000882381F146C0911144C080915C068823C5
:10F4600041F06BE776E180915A0690915B060E942D
:10F4700071439DDC81E08093E2058091060281303A
:10F4800081F58091FA0F882361F14091C20F50916C
:10F49000C30F141615065CF4052E000C660B770BD3
:10F4A00029EC3FE58CE89AE0CF910C943C4CCF914D
:10F4B0000C94C95F82E08093E70580915C06882305
:10F4C00041F067E876E180915A0690915B060E94D0
:10F4D0007143C1E0C093E6050E945F6168DCC093A0
:10F4E000E205CF9108950C947460809153068111C8
:10F4F0000C945F610C9474600C9400620C949462A0
:10F500000E94CB598091BB0581110C9400620C9430
:10F510009462CF939C01A4E6B0E00E9450AD2FEF1F
:10F5200033E040E050E00E9402ADC22F30E0809115
:10F53000930E281B310937FF03C0319521953109FE
:10F54000233031053CF1C33020F0C23618F0C4E658
:10F5500001C0C0E08091560690915706DC01ED9104
:10F56000FC91E25BFF4F0190F081E02D6C2F19952B
:10F57000C093930E80915C06882361F062E676E189
:10F5800080915A0690915B060E9400428C2FCF9189
:10F590000C946D84CF9108959C010197849710F489
:10F5A000822F0895C901845691098438934040F40C
:10F5B000C90164E670E00E9478A7822F94E61BC020
:10F5C000283E43E03407D8F0C90168EE73E00E949A
:10F5D00078A748E15CEF649FC001659F900D749F20
:10F5E000900D1124280F391FC9016AE070E00E94B4
:10F5F0008CA7822F9AE0699F80191124089580E0DA
:10F6000008956FE676E180915A0690915B060C941E
:10F6100000428091560690915706DC01ED91FC91D5
:10F620000484F585E02D60E0199480915606909150
:10F630005706DC01ED91FC910484F585E02D61E035
:10F640001994CF93DF938091CE0F882349F1809155
:10F650000102882329F1C091E405D091E50589A133
:10F660009AA1892B11F01AA219A28B8D9C8D9B87D0
:10F670008A872FEF30E03D872C879F878E87E88130
:10F68000F9810190F081E02D60E070E0CE011995E4
:10F690001F8A1E8A0E9426476D8F7E8F8F8F98A3A8
:10F6A000DF91CF910895CF93DF938091CE0F882380
:10F6B00049F180910102882329F1C091E405D0919C
:10F6C000E50589A19AA1892B11F01AA219A2898DA9
:10F6D0009A8D9B878A872FEF30E03D872C879F8705
:10F6E0008E87E881F9810190F081E02D60E070E083
:10F6F000CE0119951F8A1E8A0E9426476D8F7E8F24
:10F700008F8F98A3DF91CF9108951F93CF93DF93AD
:10F710009091CE0F9923C9F0182FC091E405D09194
:10F72000E505CE010E94EF868E899F89892B49F4D9
:10F73000112319F0898D9A8D02C08B8D9C8D9F8B22
:10F740008E8B81E090E09AA389A3DF91CF911F91E6
:10F750000895809101028823B9F0109201028091EE
:10F760005C06882341F062E576E180915A0690912B
:10F770005B060E9471430E94CB598091BB05882390
:10F7800019F080915306C1CF089580910102811133
:10F790001AC081E08093010280915C06882341F0C9
:10F7A00063E476E180915A0690915B060E94714372
:10F7B0000E94CB598091BB05882329F08091530684
:10F7C000811171CF3ECF089590D30E9440638CE8A1
:10F7D0009AE00E944C4C0E948A520E94CB59809120
:10F7E000ED0F8230C1F01CF48130A9F02FC08330BE
:10F7F00011F1843059F580914C0690914D06DC0151
:10F80000ED91FC910680F781E02D199580914A06D3
:10F8100090914B0614C08091500690915106DC01E6
:10F82000ED91FC910680F781E02D199580914E06AF
:10F8300090914F0604C080914C0690914D06DC01DA
:10F84000ED91FC910680F781E02D19958091540689
:10F8500090915506DC01ED91FC910680F781E02D39
:10F8600019958091580690915906DC01ED91FC9113
:10F870000680F781E02D19958091E4059091E505CA
:10F88000DC01ED91FC910680F781E02D19940F9336
:10F890001F93CF93DF93EC01AB0160E070E02AE0AF
:10F8A0000E9439428C01CE010E945E43800F911F5D
:10F8B000DF91CF911F910F9108958F929F92AF92F8
:10F8C000BF92CF92DF92EF92FF920F931F93CF934D
:10F8D000DF931F921F92CDB7DEB7082E000C990B55
:10F8E000AA0BBB0BFC013197ED30F10508F033C2D8
:10F8F0008827ED5AFE4F8F4F0C949FA784E080938A
:10F9000096098AE08093970986E28093990981E0BD
:10F9100080939C0980939D0980939B0948E757E158
:10F9200020E030E08091960990E0281739070CF02C
:10F9300059C1FA0185919491A0E0B0E0880F991F18
:10F94000AA1FBB1FF901EE0FFF1FEE0FFF1FE35DA4
:10F95000F64F80839183A283B3832F5F3F4F4E5F27
:10F960005F4FE0CF84E0809396098AE08093970907
:10F9700086E28093990981E080939C0980939D0998
:10F9800082E080939B0940E757E120E030E08091DE
:10F99000960990E0281739070CF024C1FA018591E7
:10F9A0009491A0E0B0E0880F991FAA1FBB1FF90136
:10F9B000EE0FFF1FEE0FFF1FE35DF64F8083918375
:10F9C000A283B3832F5F3F4F4E5F5F4FE0CF84E052
:10F9D0008093970985E28093990981E080939C093F
:10F9E00088E080939D0983E080939B0980E090E00C
:10F9F000FC01E859F84EE491DC01A256B64FEC93B5
:10FA0000019688309105A1F70E94213CEBC088E067
:10FA10008093960986E08093970986E280939909FE
:10FA200081E080939C0980939D0984E080939B09E9
:10FA300048E557E120E030E08091960990E02817F2
:10FA400039070CF0CFC0FA0185919491A0E0B0E0A5
:10FA5000880F991FAA1FBB1FF901EE0FFF1FEE0FA2
:10FA6000FF1FE35DF64F80839183A283B3832F5FF3
:10FA70003F4F4E5F5F4FE0CF88E08093960986E06E
:10FA80008093970986E28093990981E080939C098D
:10FA900080939D0985E080939B0948E457E120E02D
:10FAA00030E08091960990E0281739070CF09AC051
:10FAB000FA0185919491A0E0B0E0880F991FAA1FE8
:10FAC000BB1FF901EE0FFF1FEE0FFF1FE35DF64FA7
:10FAD00080839183A283B3832F5F3F4F4E5F5F4F3D
:10FAE000E0CFE091CE09F091CF09729780819181AA
:10FAF00040E550E060E070E08253964F0E94783D10
:10FB00002AC182E18093960985E08093970982E279
:10FB10008093990981E080939C0980939D0987E0F7
:10FB200080939B0980E993E3A0E0B0E080932D09E6
:10FB300090932E09A0932F09B0933009F2E08F2EF5
:10FB4000912C01E010E080E090E0A0E0BBE54CE407
:10FB500054E060E070E024EEC22E2CE0D22EE12CC6
:10FB6000F12C9801220F331F220F331F5401AA0CCE
:10FB7000BB1CAA0CBB1C235D364FF901B7FF0DC09F
:10FB8000C082D182E282F3829501235D364FF90172
:10FB900040835183628373830CC0408351836283AB
:10FBA00073839501235D364FF901C082D182E282D1
:10FBB000F382880F991FAA1FBB1F0E5F1F4FF2E031
:10FBC0008F0E911C22E18216910459F688E79FEF6F
:10FBD000A0E0B0E08093710990937209A09373093B
:10FBE000B09374090E94903CB6C0CE0101960E9469
:10FBF0000D3C23E040E150E060E070E072C084E042
:10FC00008093960982E38093970986E2809399090D
:10FC100081E080939C0980939D098AE080939B09F1
:10FC200040E457E120E030E08091960990E0281709
:10FC30003907C4F6FA0185919491A0E0B0E0880FED
:10FC4000991FAA1FBB1FF901EE0FFF1FEE0FFF1F29
:10FC5000E35DF64F80839183A283B3832F5F3F4F91
:10FC60004E5F5F4FE1CF84E08093960980E28093FE
:10FC7000970986E28093990981E080939C0980939B
:10FC80009D098BE080939B0948E357E120E030E039
:10FC90008091960990E0281739070CF0A3CFFA015C
:10FCA00085919491A0E0B0E0880F991FAA1FBB1F17
:10FCB000F901EE0FFF1FEE0FFF1FE35DF64F80838C
:10FCC0009183A283B3832F5F3F4F4E5F5F4FE0CF9F
:10FCD000CE0101960E940D3C21E040E154E060E03D
:10FCE00070E0CE0101960E94EC3C35C084E0809328
:10FCF000960983E08093970986E28093990981E0D1
:10FD000080939C0980939D098DE080939B0940E33B
:10FD100057E120E030E08091960990E028173907FC
:10FD20000CF060CFFA0185919491A0E0B0E0880FCB
:10FD3000991FAA1FBB1FF901EE0FFF1FEE0FFF1F38
:10FD4000E35DF64F80839183A283B3832F5F3F4FA0
:10FD50004E5F5F4FE0CF0F900F90DF91CF911F91DB
:10FD60000F91FF90EF90DF90CF90BF90AF909F905A
:10FD70008F9008950F931F93CF93DF93EC01462F3D
:10FD800050E060E070E02AE00E9439428C01CE0130
:10FD90000E945E43800F911FDF91CF911F910F91C1
:10FDA00008952FB7F894882381F08091C411909121
:10FDB000C5119093D3118093D2118091D411909159
:10FDC000D51118161906ACF00FC08091C61190918C
:10FDD000C7119093D3118093D2118091D411909137
:10FDE000D511181619062CF48091D4119091D511C3
:10FDF00007C08091D4119091D51191958195910969
:10FE00009093D5118093D4112FBF0895AF92BF92D4
:10FE1000CF92DF92EF92FF920F931F93CF93DF93D6
:10FE20001F921F92CDB7DEB78C017A836983CE0112
:10FE300001966C01580192E0A90EB11CE12CF12C45
:10FE4000C8010E94E2ACF60161916F01861731F0A2
:10FE5000C8010E94F4ACFFEFEF1AFF0A0F5F1F4FBB
:10FE60000A151B0569F781E0EF2809F480E00F907F
:10FE70000F90DF91CF911F910F91FF90EF90DF9046
:10FE8000CF90BF90AF900895EF92FF920F931F9382
:10FE9000CF93DF931F921F92CDB7DEB78C017B010A
:10FEA0008AEA8A8341E050E0BE016E5F7F4FC8015D
:10FEB0000E942E69D701ED91FC910284F385E02D1B
:10FEC000C701199582E8898341E050E0BE016F5F68
:10FED0007F4FC8010E942E690F900F90DF91CF9144
:10FEE0001F910F91FF90EF900895CF92DF92EF92C4
:10FEF000FF920F931F930E9426476B017C01609332
:10FF00004012709341128093421290934312809159
:10FF1000780A0E94504580933F1290917A0A992363
:10FF200029F091E0811190E090933F128091820A34
:10FF30009091830AA091840AB091850A9701860165
:10FF4000081B190B2A0B3B0B4091860A5091870A1C
:10FF50006091880A7091890A90917B0A04171507AD
:10FF60002607370760F4C0927E0AD0927F0AE0929B
:10FF7000800AF092810A10927D0A892F1EC0909308
:10FF80007C0A80913F1280937B0AC0927E0AD092B5
:10FF90007F0AE092800AF092810A891761F0C0928C
:10FFA000820AD092830AE092840AF092850A91E054
:10FFB00090937D0A02C010927D0A1F910F91FF90CD
:10FFC000EF90DF90CF900895462F50E060E070E012
:10FFD0002AE00C9439420F931F93CF93DF93EC01E7
:10FFE0002AE00E9439428C01CE010E945E43800FBC
:10FFF000911FDF91CF911F910F910895CF92DF92C2
:020000021000EC
:10000000EF92FF920F931F93CF93DF936B01770FC4
:10001000EE08FF08F7FE1BC0EC016DE20E94F941FB
:100020008C0144275527BA014C195D096E097F09D7
:100030002AE0CE010E943942800F911FDF91CF91BB
:100040001F910F91FF90EF90DF90CF9008952AE0DD
:10005000B701A601DF91CF911F910F91FF90EF9013
:10006000DF90CF900C943942CF92DF92EF92FF92C3
:100070000F931F93CF93DF938C016B01770FEE08E3
:10008000FF08F7FE12C06DE20E94F941EC0144271F
:100090005527BA014C195D096E097F092AE0C8018C
:1000A0000E943942C80FD91F06C02AE0B701A60135
:1000B0000E943942EC01C8010E945E438C0F9D1FD3
:1000C000DF91CF911F910F91FF90EF90DF90CF9034
:1000D00008950F931F93CF93DF931F92CDB7DEB791
:1000E0008C0169830E94E2AC6981861729F0C801FE
:1000F0000E94F4AC81E001C080E00F90DF91CF91CD
:100100001F910F910895CF930E94A15284E090E037
:100110009093750A8093740A89E99EE09093631125
:100120008093621110925D118091730A9091990EE3
:10013000891718F091E090935A1122EA3EE030932B
:100140006D1120936C11109267119091A20E891776
:1001500018F091E0909364112BEA3EE03093771110
:1001600020937611109271119091AB0E891718F0AF
:1001700091E090936E1124EB3EE030938111209337
:10018000801110927B119091B40E891718F091E0B4
:10019000909378111092720A20E030E0F901E75C48
:1001A000F04F40815181415051094432510520F4B2
:1001B00091E09093720A05C02D5F3F4F28373105BB
:1001C00069F79091720A992341F12091AC0E309118
:1001D000AD0E2D5D3F4F3093AD0E2093AC0E2091B0
:1001E000AE0E3091AF0E235231093093AF0E2093F3
:1001F000AE0E2091B50E3091B60E2D5D3F4F30936F
:10020000B60E2093B50E2091B70E3091B80E235242
:1002100031093093B80E2093B70E9091B20F9F30F2
:1002200049F49091B30F9F3029F410925911109214
:10023000581108C0209101103091021030935911CB
:100240002093581122E130E030935611209355113C
:100250002091740A3091750AADEBBEE0E1E0F1E166
:1002600041E0B683A5839C91992329F0891718F062
:1002700040832F5F3F4F1A96379691E1E535F90796
:1002800081F73093750A2093740A2131310534F0D7
:1002900080E190E09093750A8093740A0E948C52DA
:1002A0008EE591E1909364108093631080916211C8
:1002B0009091631190936210809361108BE591E1AE
:1002C00090936610809365108CE591E1909368108F
:1002D000809367108AE591E190936A10809369108A
:1002E00088E691E190936E1080936D1080916C116F
:1002F00090916D1190936C1080936B1085E691E155
:100300009093701080936F1086E691E19093721035
:100310008093711084E691E1909374108093731030
:1003200082E791E190937810809377108091761115
:100330009091771190937610809375108FE691E1EC
:1003400090937A108093791080E791E190937C10DC
:1003500080937B108EE691E190937E1080937D10C8
:100360008CE791E1909382108093811080918011AD
:10037000909181119093801080937F1089E791E193
:1003800090938410809383108AE791E19093861074
:100390008093851088E791E190938810809387106F
:1003A0002091740A3091750A2450310960E07AE096
:1003B000C7E0462F50E04217530724F5CA010496C0
:1003C000789FF001799FF00D1124EF59FF4EC49FE3
:1003D000C001C59F900D1124AC014D5F5E4E53834B
:1003E0004283DC01AF5FBE4E15964D915C9116972E
:1003F000518340838E5F9E4E95838483B187A0870F
:100400006F5FD7CF81E08093760ACF9108950F93E5
:100410001F93CF93DF93FC01248135812115310592
:1004200019F4FB01108211C0EA0121972C173D0736
:1004300008F4E9018B01FC0160817181AE01C80102
:100440000E94E9AAC00FD11F1882DF91CF911F919E
:100450000F91089580915D0680935C060895209128
:100460006C12222369F0A0916A12B0916B12ED9187
:10047000FC9111970190F081E02DBC01CD01199400
:10048000089520916912222369F0A0916712B0911A
:100490006812ED91FC9111970190F081E02DBC0163
:1004A000CD011994089520916612222369F0A0913C
:1004B0006412B0916512ED91FC9111970190F08159
:1004C000E02DBC01CD0119940895209163122223DF
:1004D00069F0A0916112B0916212ED91FC911197B7
:1004E0000190F081E02DBC01CD0119940895209177
:1004F0006012222369F0A0915E12B0915F12ED911B
:10050000FC9111970190F081E02DBC01CD0119946F
:10051000089520915D12222369F0A0915B12B091A1
:100520005C12ED91FC9111970190F081E02DBC01DE
:10053000CD011994089520915A12222369F0A091B7
:100540005812B0915912ED91FC9111970190F081E0
:10055000E02DBC01CD01199408952091571222235A
:1005600069F0A0915512B0915612ED91FC9111973E
:100570000190F081E02DBC01CD01199408952091E6
:100580005412222369F0A0915212B0915312ED91AE
:10059000FC9111970190F081E02DBC01CD011994DF
:1005A00008958091560690915706DC01ED91FC91DB
:1005B000EC5AFF4F0190F081E02D1994809156067E
:1005C00090915706DC01ED91FC91EE5AFF4F01909E
:1005D000F081E02D19948091560690915706DC0128
:1005E000ED91FC91E05BFF4F0190F081E02D1994BB
:1005F0008091CE0F81110DC08091E4059091E505A9
:10060000DC01ED91FC910190F081E02D60E070E063
:10061000199408958091CE0F81110DC08091E40549
:100620009091E505DC01ED91FC910190F081E02DC8
:100630006FEF70E01994089580915D06882361F052
:100640000E94CC52029741F067E278E180915A060D
:1006500090915B060C9471430895CF93DF932091A2
:100660006F123091701228173907C9F090937012E9
:1006700080936F1220915C06222389F0EC0168EFD1
:1006800077E180915A0690915B060E940042BE017C
:1006900080915A0690915B06DF91CF91F8C8DF9167
:1006A000CF910895CF93DF9320916D1230916E1208
:1006B00028173907C9F090936E1280936D1220911C
:1006C0005C06222389F0EC016EED77E180915A06F9
:1006D00090915B060E940042BE0180915A06909163
:1006E0005B06DF91CF91D3C8DF91CF910895209120
:1006F0006612222339F0BC01809150129091511260
:100700000C94C739089520916312222339F0BC015B
:1007100080914E1290914F120C94C73908952091F8
:100720006012222339F0BC0180914C1290914D123D
:100730000C94C739089520915D12222339F0BC0131
:1007400080914A1290914B120C94C73908952091D0
:100750005A12222339F0BC0180914812909149121B
:100760000C94C739089520915712222339F0BC0107
:1007700080914612909147120C94C73908952091A8
:100780005412222339F0BC018091441290914512F9
:100790000C94C7390895CF92DF92EF92FF92209187
:1007A0000002213019F42091DA0F04C02230C1F583
:1007B0002091E00F2223A1F19C01211584E038074C
:1007C00010F02FEF33E0ADE0B0E00E9450AD2FEF1E
:1007D00033E040E050E00E9402AD69017A018FEF02
:1007E000C81AD80AE80AF80A80917C128C15C1F060
:1007F000C0927C1280915C06882391F067E977E1D2
:1008000080915A0690915B060E9400426C2D809167
:100810005A0690915B06FF90EF90DF90CF90AACAA6
:10082000FF90EF90DF90CF900895CF92DF92EF92FC
:10083000FF9220910002213019F42091D70F04C0BB
:100840002230C1F52091DD0F2223A1F19C01211559
:1008500084E0380710F02FEF33E0ADE0B0E00E9405
:1008600050AD2FEF33E040E050E00E9402AD69014F
:100870007A018FEFC81AD80AE80AF80A80917A122A
:100880008C15C1F0C0927A1280915C06882391F099
:1008900060E877E180915A0690915B060E940042E1
:1008A0006C2D80915A0690915B06FF90EF90DF903F
:1008B000CF9060CAFF90EF90DF90CF900895682F9F
:1008C00080915A0690915B067FDB65E278E180912A
:1008D0005A0690915B060C940042F1DF80915A0613
:1008E00090915B060C945E43CF92DF92EF92FF9261
:1008F0009C01A3E6B0E00E9450AD2FEF33E040E052
:1009000050E00E9402AD69017A018FEFC81AD80A3F
:10091000E80AF80A8091B7058C15A1F0C092B705D6
:1009200080915C06882371F067EC77E180915A062C
:1009300090915B060E9400428C2DFF90EF90DF901B
:10094000CF90CBCFFF90EF90DF90CF900895CF92D4
:10095000DF92EF92FF929C01A3E6B0E00E9450ADBF
:100960002FEF33E040E050E00E9402AD69017A01D0
:100970008FEFC81AD80AE80AF80A8091B8058C15D2
:10098000A1F0C092B80580915C06882371F06EEAF0
:1009900077E180915A0690915B060E9400428C2D6F
:1009A000FF90EF90DF90CF9098CFFF90EF90DF9087
:1009B000CF90089520915A0630915B06882319F054
:1009C00067EB76E002C06BEB76E0C9010C94004265
:1009D000F1DF80915A0690915B060C945E43209162
:1009E0005A0630915B06882319F06AE178E102C06B
:1009F0006FE178E1C9010E94004280915A0690910E
:100A00005B060C945E4368E178E180915A06909110
:100A10005B060C94004264E178E180915A06909163
:100A20005B060C940042CF93CDE262E178E18091C5
:100A30005A0690915B060E940042C150B1F7809126
:100A40005A0690915B060E945E4380915A069091EF
:100A50005B06DC01ED91FC910284F385E02DCF91E2
:100A6000199408950895089508950895623039F00D
:100A7000633041F0613041F440936F0E089540932C
:100A80006E0E089540936D0E0895623069F06330E4
:100A9000A1F06130D1F45093730E4093720E3093F5
:100AA000750E2093740E089550937A0E4093790E2C
:100AB00030937C0E20937B0E08955093810E4093CB
:100AC000800E3093830E2093820E08950895FC01CA
:100AD00062830895FC0164830895FC016383089593
:100AE00008950C946648089580E008950895089547
:100AF00008950895089508958FE090E00C944A7742
:100B0000633091F028F4613049F0623051F008957B
:100B1000653081F060F0663081F0089589E090E002
:100B20000EC08AE090E00BC08BE090E008C08CE043
:100B300090E005C08DE090E002C08EE090E00C9463
:100B40004A77FC018481882321F082E090E00C94B4
:100B50004A770895FC018381882321F081E090E0A9
:100B60000C944A7708958BE090E00C944A7784E0E7
:100B700090E00C944A7760E080E190E00C948577F7
:100B800060E08FE090E00C9485776330A1F028F46A
:100B9000613049F0623059F008956530A1F078F085
:100BA0006630A9F0089560E089E090E013C060E04D
:100BB0008AE090E00FC060E08BE090E00BC060E066
:100BC0008CE090E007C060E08DE090E003C060E062
:100BD0008EE090E00C9485776330A1F028F46130CA
:100BE00049F0623059F008956530A1F078F0663030
:100BF000A9F0089561E089E090E013C061E08AE027
:100C000090E00FC061E08BE090E00BC061E08CE011
:100C100090E007C061E08DE090E003C061E08EE00D
:100C200090E00C948577FC018281882329F061E0B3
:100C300088E090E00C9485770895FC0184818823F6
:100C400029F061E082E090E00C9485770895FC0142
:100C50008381882329F061E081E090E00C9485771E
:100C6000089561E086E090E00C94857760E08BE089
:100C700090E00C94857760E084E090E00C948577B8
:100C800061E087E090E00C94857761E085E090E09A
:100C90000C94857761E083E090E00C948577609117
:100CA000700E7091710E8091870E9091880E0E9447
:100CB000ED4B1092760E6091770E7091780E8091C8
:100CC000870E9091880E0E94ED4B10927D0E6091E0
:100CD0007E0E70917F0E8091870E9091880E0E94FB
:100CE000ED4B1092840E109275120895809175123A
:100CF000811113C022EC38E748EB5BE060E070E064
:100D00008091870E9091880E0E943C4C9093710EBA
:100D10008093700E81E08093751208958091890E02
:100D20008823B9F068EE73E081E00E94FB4E1092D8
:100D3000890E26E638E448E95AE360E070E08091E5
:100D4000870E9091880E0E943C4C9093860E809363
:100D5000850E08956CED75E080E00C94FB4E24EF59
:100D600031E0DB010E94ADA72FEF30E040E050E022
:100D70000E9402ADCA01B90164527A4F8F4F9F4F52
:100D800080E00C94FB4E8091890E81110C94327797
:100D900008958091890E81110C943277089580E036
:100DA0000E94224F81E00E94224F82E00E94224F47
:100DB0006CED75E080E00E94FB4E6CED75E081E02B
:100DC0000E94FB4E88EE94E7A1E0BB27ABBFFC017D
:100DD0006791769182E00E94FB4E0C945448FC018E
:100DE000808991899387828782899389958784876F
:100DF0008489958997878687089526E00C94EB442B
:100E00004115510521F06115710509F000CB0895D8
:100E1000EF92FF920F931F93CF93DF931F921F9236
:100E2000CDB7DEB78C018CE789831A82F801E480A4
:100E3000F580FFEFEF1AFF0AB701C8010E94F040EA
:100E4000882381F0F8012081318184819581BE0160
:100E50006F5F7F4F820F931F0E94E2AAF801F58215
:100E6000E48281E00F900F90DF91CF911F910F915D
:100E7000FF90EF900895AF92BF92CF92DF92EF92E2
:100E8000FF920F931F93CF93DF9300D01F92CDB7A4
:100E9000DEB78C0149835A836B837C83CE01019634
:100EA0006C01580194E0A90EB11CE12CF12CC80191
:100EB0000E94E2ACF60161916F01861731F0C80122
:100EC0000E94F4ACFFEFEF1AFF0A0F5F1F4F0A15E5
:100ED0001B0569F781E0EF2809F480E00F900F907F
:100EE0000F900F90DF91CF911F910F91FF90EF9096
:100EF000DF90CF90BF90AF900895CF92DF92EF92A6
:100F0000FF920F931F93CF93DF93EC010091871211
:100F1000E0E0F0E020E030E0A90110E0CE17DF07CC
:100F20001CF1309711F40D32E1F0DF01A957BD4EED
:100F3000FC9080ED8F0D8A30A8F4AAE0B0E00E940A
:100F40001EAD2F2DFF0C330B205331096901330FD8
:100F5000EE08FF089B01AC012C0D3D1D4E1D5F1DD1
:100F600001C011E03196DACFCA01B901112339F07D
:100F700090958095709561957F4F8F4F9F4FDF9132
:100F8000CF911F910F91FF90EF90DF90CF90089538
:100F900080917B0A811105C081E090917D0A9111B9
:100FA00001C080E00895CF93DF932091A70930918D
:100FB000A809E9012697A881B981A955B64F1296CB
:100FC0001C92082E000C990BAA0BBB0BFC0131974D
:100FD000EE30F10508F057C18827E05AFE4F8F4FD9
:100FE0000C949FA7F9013A97808191818955964F7A
:100FF0000E947EA5882309F44BC1E091A709F091D6
:10100000A80936970190F081E02DE955F64F81E06F
:10101000A0C0F9013C97808191818955964F0E942B
:10102000BBA4882309F434C1E091A709F091A80971
:1010300036970190F081E02DE955F64F82E089C0A6
:10104000F9013E97808191818955964F0E94FEA3B8
:10105000882309F41DC1E091A709F091A8093697EA
:101060000190F081E02DE955F64F83E072C0F9015F
:101070007097808191818955964F0E9481A3882322
:1010800009F406C1E091A709F091A80936970190EB
:10109000F081E02DE955F64F84E05BC0F9017297CD
:1010A000808191818955964F0E943CA3882309F441
:1010B000EFC0E091A709F091A80936970190F0815F
:1010C000E02DE955F64F85E044C0F9017497808121
:1010D00091818955964F0E94C3A2882309F4D8C0F4
:1010E000E091A709F091A80936970190F081E02DD1
:1010F000E955F64F86E02DC0F90176978081918100
:101100008955964F0E943DA2882309F4C1C0E09101
:10111000A709F091A80936970190F081E02DE955D3
:10112000F64F87E016C0F901789780819181895543
:10113000964F0E942FA2882309F4AAC0E091A70924
:10114000F091A80936970190F081E02DE955F64F0E
:1011500088E082839DC0F901B09780819181895593
:10116000964F0E94519F882309F492C0E091A709ED
:10117000F091A80936970190F081E02DE955F64FDE
:1011800083819481A581B6814097A105B10509F0BD
:101190007FC08EC0F9017A97808191818955964FE1
:1011A0000E9464A1882309F473C0E091A709F0911B
:1011B000A80936970190F081E02DE955F64F8AE0B5
:1011C000C8CFF9017C97808191818955964F0E9403
:1011D00099A0882309F45CC0E091A709F091A809BF
:1011E00036970190F081E02DE955F64F8BE0B1CFB5
:1011F000F901B097808191818955964F0E94519F46
:10120000882309F445C0E091A709F091A809369711
:101210000190F081E02DE955F64F83819481A581FD
:10122000B68180319440A105B10591F543C0F90123
:101230007E97808191818955964F0E94CA9F88230D
:1012400039F1E091A709F091A80936970190F08152
:10125000E02DE955F64F8DE07CCFF901B097808104
:1012600091818955964F0E94519F882389F0E09182
:10127000A709F091A80936970190F081E02DE95572
:10128000F64F8EE066CFE881F981E955F64F12827C
:10129000E091A709F091A80936970190F081E02D1F
:1012A000E955F64F81E09281911106C080E004C0BB
:1012B00089E04FCF8CE04DCFDF91CF910895EF9231
:1012C000FF920F931F93CF93DF931F921F92CDB77F
:1012D000DEB741110AC07C0197FF03C0F194E1948D
:1012E000F108E616F70664F402C0E12CF12C81E067
:1012F0008093680A8FEF633371059CF425E012C078
:101300006E157F0534F01092680A81E091E021E0CB
:101310000AC06D337105BCF381E08093680A23E055
:1013200001C024E092E03091680A332379F03FB79E
:10133000F894899F902D112490936C0A2093861223
:1013400000918412109185123FBF0AC09FB7F89494
:1013500010926C0AF0928512E09284129FBF87016E
:101360004A8389835DD24A818981442319F017FF1A
:1013700019C014C0813031F417FD10C0E016F10619
:101380008CF40FC08F3F71F40E151F0554F00F3F02
:10139000110541F03CF00FEF10E004C000E010E058
:1013A00001C08701C8010F900F90DF91CF911F916D
:1013B0000F91FF90EF900895CF92DF92EF92FF92FE
:1013C0000F931F93CF93DF93042FE22E433049F006
:1013D000453039F0443041F4F92EFF1CFF24FF1C46
:1013E00004C0FF24F39401C0F12CFC0197FF03C05B
:1013F000F195E195F109EF011092690A013009F4C4
:1014000031C1053009F06EC080919612811118C06B
:10141000C0918312D0E0D0939512C093941281E0D2
:101420008093690A21E030E0309393122093921266
:1014300030938212209381128093961211E0B9C0EA
:10144000809181129091821281159640E8F581E099
:101450008093690A80918112909182122091921258
:1014600030919312821B930BC0919412D0919512DC
:10147000089720F1BE0180E090E00E94BDAB209172
:101480007D1230917E1240917F12509180120E9405
:101490001EAC20E030E040E05FE30E94B4A70E9471
:1014A00080A8EB0170939512609394128091811241
:1014B000909182129093931280939212CF31D10522
:1014C0000CF075C0E1E001C0E0E01092690A1092F2
:1014D000951210929412109296128E2F11E0C0E085
:1014E000D0E061C0EE20E1F0023029F48091640A7E
:1014F0009091650A04C08091660A9091670AE81786
:10150000F9070CF0B2C081E08093690A80917C12E7
:1015100094E0F595E7959A95E1F7EE5F1FEF43C0EC
:10152000DB0177FF03C0B195A195B109AE17BF07E5
:10153000C4F480917B12882309F49BC081E08093DE
:10154000690A80917A12909179129130A1F5EA1B83
:10155000FB0BFD970CF0845011E054976CF5E4E020
:101560002CC0EA17FB070CF084C080917812882306
:1015700009F47FC0043009F47CC081E08093690ADB
:1015800080917C1290917712913009F07BC0E23308
:10159000F10514F48E5F76C0AE1BBF0BD3970CF42D
:1015A00071C082506FC01E1644F0E1E006C011E029
:1015B00081E0E1E006C011E0E2E0181614F06E01EF
:1015C0005FC06E019091690A9923D9F02FB7F89402
:1015D0001E9F902D112490936D0A809376121C16F5
:1015E0001D063CF48091811290918212892B09F49E
:1015F0004BC0053021F0C0918112D09182122FBFD3
:1016000009C08FB7F89410926D0AD0938212C093DC
:1016100081128FBF05D1EE2019F0D7FF1DC018C071
:10162000113031F4D7FD14C0CC16DD06ACF413C074
:101630001F3F91F4023011F0033071F4CC15DD0539
:1016400054F0CF3FD10541F03CF0CFEFD0E004C0E3
:10165000C0E0D0E001C0E601FF2001F1D195C195C5
:10166000D1091CC090E080E006C090E080E01FEF50
:1016700003C09E2F8F2F11E06F01C92FD82FE1E0FB
:1016800081E0A0CF1FEF98CF80916D0A082E000C4B
:10169000990B9093821280938112ABCFCE01DF9190
:1016A000CF911F910F91FF90EF90DF90CF90089511
:1016B000CF92DF92EF92FF9297FF26C0CC24DD24D9
:1016C000C61AD70A0D2C000CEE08FF08092E000CD4
:1016D000AA0BBB0B9C01AD0121503F4F4F4F5F4FF9
:1016E000C701B60160957095809590950E9469A795
:1016F0002EEF30E040E050E00E9402ADC20ED31E5B
:10170000E41EF51EC60126C0009711F1092E000C3B
:10171000AA0BBB0B9C01AD012150310941095109B4
:10172000CB01770FAA0BBB0BBC01CD016150710936
:10173000810991090E9469A72EEF30E040E050E056
:101740000E9402ADDA01C9010196A11DB11D02C0BE
:1017500080E090E0FF90EF90DF90CF90089580912F
:10176000C00D9091C10D892B89F08091C60D882301
:1017700081F00E9426476093C20D7093C30D809341
:10178000C40D9093C50D1092C60D089581E080930D
:10179000C60D08951F920F920FB60F9211242F932A
:1017A0008F939F93109295001092940080916B0AF2
:1017B0008F5F80936B0A90917612891784F0109254
:1017C0006B0A20916D0A8091811290918212820F92
:1017D000911D27FD9A95909382128093811280919A
:1017E0006A0A8F5F80936A0A90918612891784F043
:1017F00010926A0A20916C0A80918412909185124D
:10180000820F911D27FD9A959093851280938412E3
:101810009F918F912F910F900FBE0F901F90189551
:101820008091690A811104C08091680A882321F09F
:1018300080917100826003C0809171008D7F8093E0
:10184000710008951F93CF93DF931F92CDB7DEB73A
:1018500010E0181729F08983D6D81F5F8981F9CF46
:101860000F90DF91CF911F910895CF93DF9360E0A8
:1018700088E00E94784510929A12C0919812D091F7
:101880009912BE018CE89AE00E94D54B882329F07A
:10189000BE018CE89AE00E94ED4B81E080939712A4
:1018A00080915C06882341F06FE778E180915A06C9
:1018B00090915B060E947143DF91CF910C94257249
:1018C00060914B1070914C1080E090E00E94BDAB95
:1018D00020E030E04AE754E40E9418A8AB01BC01C4
:1018E00021E080915A0690915B060C94814260E75A
:1018F00078E180915A0690915B060E9400426091C7
:10190000001080915A0690915B060E94E47F9091AE
:1019100000108091B705981781F060E678E180911A
:101920005A0690915B060E9400426091B705809133
:101930005A0690915B060E94E47F6EE578E1809103
:101940005A0690915B060C9400426FE478E1809116
:101950005A0690915B060E9400426091FE0F8091B2
:101960005A0690915B060E94E47F9091FE0F809151
:10197000B805981781F06FE378E180915A0690914D
:101980005B060E9400426091B80580915A069091D2
:101990005B060E94E47F6DE378E180915A069091A6
:1019A0005B060C94004281E080933E0E80915C06C1
:1019B000882379F02091C00F80915A0690915B06A0
:1019C000222319F069E978E102C06BEA78E10C940E
:1019D00071430895CF93DF93CDB7DEB72F970FB63E
:1019E000F894DEBF0FBECDBF789484B5826084BD0D
:1019F00084B5816084BD85B5826085BD85B5816013
:101A000085BD80916E00816080936E001092810090
:101A1000809181008260809381008091810081604B
:101A2000809381008091800081608093800080910C
:101A3000B10084608093B1008091B0008160809398
:101A4000B00080919100826080939100809191001C
:101A500081608093910080919000816080939000DC
:101A60008091A10082608093A1008091A10081609B
:101A70008093A1008091A00081608093A00080915C
:101A800021018260809321018091210181608093F6
:101A900021018091200181608093200180917A0052
:101AA000846080937A0080917A00826080937A00CB
:101AB00080917A00816080937A0080917A008068BA
:101AC00080937A001092C1000E94980C212C312C36
:101AD00021012A948091B00681110DC0E09162111C
:101AE000F0916311818192819093AF068093AE064D
:101AF00081E08093B0068091A60681110DC0E0912F
:101B00006211F0916311838194819093A506809373
:101B1000A40681E08093A6060E9426476093A00653
:101B20007093A1068093A2069093A3068091080269
:101B3000882309F4E8C06091EB0F70E080E090E04A
:101B40000E94BDAB20E030E048EC52E40E9418A8AF
:101B500020E030E04FE753E40E941EAC0E9480A8D2
:101B600070939F0660939E066091F00F70E080E096
:101B700090E00E94BDAB20E030E048EC52E40E94CF
:101B800018A820E030E04FE753E40E941EAC0E940A
:101B900080A870939D0660939C066091EE0F64365A
:101BA000C0F470E080E090E00E94BDAB20E030E047
:101BB00048EC52E40E9418A820E030E04FE753E4DC
:101BC0000E941EAC0E9480A870939B0660939A06A8
:101BD00006C08FEF90E090939B0680939A066091E9
:101BE000EF0F6436C0F470E080E090E00E94BDAB7F
:101BF00020E030E048EC52E40E9418A820E030E0F9
:101C00004FE753EC0E941EAC0E9480A87093990687
